:100000000C943D050C9458050C9458050C94580517
:100010000C9458050C9458050C9458050C945805EC
:100020000C9458050C9474180C9458050C945805AD
:100030000C94582C0C9458050C9458050C945805A5
:100040000C9458050C9458050C9408170C945805FA
:100050000C940C0C0C9458050C94D30B0C94580570
:100060000C94881D0C9458050C94132B0C94580573
:100070000C9427680C9458050C945805361E291EBC
:100080001D1E031EE91DC51DD71D3A216E206B20C4
:10009000C51D58203E201E20FE1FAC1F5A1F421EA9
:1000A000882B7B2BC82BAC2BA02B392B4A2B4A2B14
:1000B000512B6D2B682B4D2B552B512B642B712BFA
:1000C0004D2B552B512B602B762B4D2BDA2B0A0DFC
:1000D000426174743A0020332043656C6C732020B5
:1000E0000020342043656C6C73202000204C6F7717
:1000F000207761726E696E67206C6576656C3A2058
:1001000025642E2564000A0D3D3D3D3D3D3D3D3DB0
:100110003D3D3D3D3D3D3D3D3D3D3D3D3D3D3D3D0F
:100120003D3D3D3D3D3D3D3D3D3D3D000A0D466C67
:1001300069676874436F6E74726F6C0A0D48617200
:1001400064776172653A25642E25640A0D536F66E3
:1001500074776172653A5625642E25642563200004
:100160000A0D74686520757365206F662074686970
:100170007320736F667477617265206973206F6E88
:100180006C79207065726D6974746564200A0D6FF6
:100190006E206F726967696E616C204D696B726F5A
:1001A0004B6F707465722D4861726477617265007F
:1001B0000A0D7777772E4D696B726F4B6F70746590
:1001C000722E646520286329204869537973746509
:1001D0006D7320476D6248000A0D3D3D3D3D3D3D3C
:1001E0003D3D3D3D3D3D3D3D3D3D3D3D3D3D3D3D3F
:1001F0003D3D3D3D3D3D3D3D3D3D3D3D3D000A0DCF
:1002000047656E65726174696E67206465666175C5
:100210006C74204D69786572205461626C65000AC7
:100220000D4D697865722D436F6E6669673A2027B8
:1002300025732720282575204D6F746F7273290050
:100240000A0D466F756E6420424C2D4374726C3AF1
:100250002000256420000A0D0A0D2121204D49535C
:1002600053494E4720424C2D4354524C3A2025646A
:10027000202121000A0D3D3D3D3D3D3D3D3D3D3DA3
:100280003D3D3D3D3D3D3D3D3D3D3D3D3D3D3D3D9E
:100290003D3D3D3D3D3D3D3D3D000A0D496E69748E
:1002A0002E20454550524F4D003A2047656E6572ED
:1002B0006174696E672044656661756C742D506168
:1002C00072616D65746572207573696E67206F6CFD
:1002D0006420537469636B2053657474696E67732B
:1002E000000A0D466C696768742D74696D65202578
:1002F00075206D696E2020546F74616C3A257520ED
:100300006D696E000A0D414343206E6F7420636176
:100310006C696272617465642021000A0D5573690D
:100320006E6720706172616D6574657273657420AB
:100330002564000A0D43616C6962726174696E67BD
:100340002070726573737572652073656E736F725A
:100350002E2E004F4B0A0D000A0D436F6E74726F04
:100360006C3A200048656164696E67486F6C640090
:100370004E6F726D616C20284143432D4D6F646553
:1003800029000A0D3D3D3D3D3D3D3D3D3D3D3D3D51
:100390003D3D3D3D3D3D3D3D3D3D3D3D3D3D3D3D8D
:1003A0003D3D3D3D3D3D3D0A0D002E000A0D2044E2
:1003B0004143206F7220493243204552524F52210F
:1003C00020436865636B204932432C2033567265A5
:1003D000662C2044414320616E6420424C2D4374BE
:1003E000726C005B25695D005B25695D002B204D0B
:1003F000696B726F4B6F70746572202B0048573AAF
:100400005625642E25642053573A25642E256425ED
:100410006320764D530053657474696E673A2564A2
:1004200020257300493243204552524F5221212149
:10043000004D697373696E6720424C2D4374726C72
:100440003A256421210028632920486F6C67657272
:10045000204275737300486F6568653A202020203C
:100460002025356900536F6C6C486F6568653A20CC
:10047000253569004C756674647275636B3A202586
:100480003569004F66662020202020203A2025353F
:1004900069004B65696E65200048F668656E726597
:1004A00067656C756E6700616B742E204C616765C3
:1004B000004E69636B3A20202020202025356900FA
:1004C000526F6C6C3A202020202020253569004B8B
:1004D0006F6D706173733A202020253569004B31B0
:1004E0003A25346920204B323A25346920004B33B9
:1004F0003A25346920204B343A25346920004B35A5
:100500003A25346920204B363A25346920004B3790
:100510003A25346920204B383A25346920004E6949
:100520003A2534692020526F3A25346920004773F8
:100530003A253469202047693A2534692000503132
:100540003A253469202050323A253469200050334E
:100550003A253469202050343A25346920004779FF
:10056000726F202D2053656E736F72004E69636B3E
:100570002025346920282533692E25692900526FEA
:100580006C6C2025346920282533692E25692900C3
:100590004769657220253469202825336929004E72
:1005A00069636B2025346920282533692E25782935
:1005B00000526F6C6C2025346920282533692E2564
:1005C0007829004769657220253469202825336918
:1005D00029004E69636B2025346920282533692959
:1005E000282533692900526F6C6C20253469202836
:1005F0002533692928253369290047696572202533
:100600003469202825336929282533692900414385
:1006100043202D2053656E736F72004E69636B200B
:1006200025346920282533692900526F6C6C2025F8
:10063000346920282533692900486F6368202534F0
:100640006920282533692900566F6C746167653A03
:100650002020202535690052432D4C6576656C3A83
:1006600020202535690052432D4368616E6E656C0C
:10067000733A253469004B6F6D70617373202020CD
:1006800020202020005269636874756E673A20202C
:10069000253569004D657373776572743A2020259E
:1006A00035690053746172743A202020202025356A
:1006B0006900506F7469313A202025336900506F0A
:1006C0007469323A202025336900506F7469333AD7
:1006D000202025336900506F7469343A2020253377
:1006E0006900536572766F202000536574706F69DE
:1006F0006E742020253369005374656C6C756E67C9
:100700003A202533690052616E67653A2533692DB9
:100710002533690045787465726E436F6E74726F2D
:100720006C2020004E693A2534692020526F3A250A
:100730003469200047733A253469202047693A25F7
:100740003469200048693A253469202043663A25F7
:1007500034692000424C2D4374726C204572726FD4
:100760007273200020253364202025336420202547
:100770003364202025336420002025336420202585
:100780003364202025336420202533642000202575
:100790003364202025336420202533642020253332
:1007A000642000424C2D4374726C20666F756E6439
:1007B0002000202563202020256320202025632081
:1007C0002020256320002025632020202563202071
:1007D0002025632020202563200020256320202061
:1007E0002D2020202D2020202D00313000313100FF
:1007F000313200466C696768742D54696D6520203C
:10080000002020202020202535756D696E00546F52
:1008100074616C3A2535756D696E00287265736573
:100820007429000A0D506C6561736520636F6E6EEC
:10083000656374205370656B7472756D20726563A7
:10084000656976657220666F722062696E64696E92
:1008500067204E4F572E2E2E006F6B2E0A0D005420
:10086000696D656F75742E0A0D00000102030404A2
:1008700005060708090A0B0B0C0D0E0F10111112BB
:100880001314151516171818191A1B1B1C1D1D1EDD
:100890001F1F202121222323242425252627272822
:1008A0002829292A2A2B2B2C2C2D2D2D2E2E2F2F8B
:1008B0003030303131323232333333343434353511
:1008C0003536363637373737383838393939393AAF
:1008D0003A3A3A3B3B3B3B3C3C3C3C3C3D3D3D3D5E
:1008E0003E3E3E3E3E3F3F3F3F3F3F404040404018
:1008F00040414141414141424242424242424343DE
:1009000043434343434444444444444444454545A9
:10091000454545454545464646464646464646477C
:100920004747474747474747474748484848484851
:10093000484848484849494949494949494949492C
:100940004949494A4A4A4A4A4A4A4A4A4A4A4A4A0A
:100950004A4B4B4B4B4B4B4B4B4B4B4B4B4B4B4BE8
:100960004B4B4C4C4C4C4C4C4C4C4C4C4C4C4C4CC9
:100970004C4C4C4C4C4D4D4D4D4D4D4D4D4D4D4DAC
:100980004D4D4D4D4D4D4D4D4D4D4D4E4E4E4E4E92
:100990004E4E4E4E4E4E4E4E4E4E4E4E4E4E4E4E77
:1009A0004E4E4E4E4E4F4F4F4F4F4F4F4F4F4F4F5C
:1009B0004F4F4F4F4F4F4F4F4F4F4F4F4F4F4F4F47
:1009C0004F4F4F4F00008F001E01AD013B02CA0286
:1009D0005803E603740402058F051B06A7063307B8
:1009E000BE074808D2085B09E3096B0AF20A780BD4
:1009F000FD0B810C040D860D070E870E060F840F6C
:100A000000107B10F5106E11E5115B12CF1242132E
:100A1000B31323149214FE146A15D3153B16A116B2
:100A200005176717C81727188318DE1837198E1986
:100A3000E319361A871AD61A231B6E1BB61BFD1B29
:100A4000411C831CC31C001D3C1D751DAB1DE01DFE
:100A5000121E421E6F1E9A1EC31EE91E0D1F2E1F60
:100A60004D1F691F841F9B1FB01FC31FD31FE11F92
:100A7000EC1FF51FFB1FFF1F002011241FBECFEF2F
:100A8000D0E1DEBFCDBF13E0A0E0B1E0E4ECF9EDD2
:100A900002C005900D92A63DB107D9F71AE0A6ED68
:100AA000B3E001C01D92A931B107E1F70C948906AA
:100AB0000C940000282FFB018150853008F023E0C2
:100AC000842F9927332721503040829FD001839F64
:100AD000B00D929FB00D1124AC59BF4F019724F077
:100AE0000E94C46C0192FACF0E947F6608958630FE
:100AF00038F085E0A2E0B0E0082E0E94D16C0895A5
:100B00008823C1F70895582F863048F155E0842F87
:100B10009927252F332721503040829FD001839F72
:100B2000B00D929FB00D1124AC59BF4FFB0101973E
:100B300024F001900E94D16CFACFA2E6B0E0042E1E
:100B40000E94D16CA0E5B0E088E0FB01182E0E9465
:100B5000DD6C852F0E9477050E947F6608958823AB
:100B6000B1F60895CF93A2E0B0E00E94C46C802D4E
:100B7000C82F8150853020F0C3E08C2F0E9477056C
:100B80008C2F9927CF9108958091E108E82FFF27B6
:100B9000EE0FFF1FE155F74F808191818D5E9F4FD2
:100BA00014F010920301808191818A5B9F4F24F49D
:100BB00080910301882319F020917E0717C081E0FE
:100BC0008093030120917E07280F20937E07253014
:100BD00038F088EE93E09093FC038093FB0306C00B
:100BE00066E970E0822F0E94C131E6CF822F9927FB
:100BF00090934C0880934B0808951F93CF93DF93F5
:100C0000182F882351F48091FF088233A0F080933D
:100C10000001112309F479C038C08EEC90E09F9355
:100C20008F931F920E9473140F900F900F908091DA
:100C3000FF08823360F784EF91E00E94F217EC0125
:100C4000112309F042C08091270390912803823834
:100C500091050CF046C08091FF0823E0829FC001FF
:100C60001124809300011123A1F268EC70E0822F1F
:100C70000E94C13186ED90E09F938F931F920E9456
:100C800073140F900F900F90C4CF809100016AE011
:100C90000E94546C892F99279F938F938091000114
:100CA0000E94546C99279F938F938CEE90E09F93B2
:100CB0008F931F920E9473148DB79EB707960FB63D
:100CC000F8949EBF0FBE8DBF20C0CE010E94FB17BF
:100CD000882309F0B8CFCE010E94FB178823A9F31F
:100CE000B2CF8091FF089927880F991F880F991F0D
:100CF00080930001112309F48CCF68EC70E084E04C
:100D00000E94C13181EE90E0B7CFDF91CF911F916A
:100D10000895CFEFD0E1DEBFCDBFEE24FF2414B89D
:100D200015B8C7EED3E0E297D7FFFDCF189B6FC190
:100D3000199B78C12DE02093020181E887B93E9A82
:100D40008FEF88B98BE184B981E085B98EE38AB9E8
:100D500087E48BB9469A84B7877F84BF809160000F
:100D60008861809360001092600080ED97E090931E
:100D7000FC038093FB031092D8041092D7041092C6
:100D8000B4081092B3081092DA041092D9041092A9
:100D9000DC041092DB04243108F43FC188E894E0BD
:100DA000A0E0B0E08093860390938703A09388032C
:100DB000B09389032A3009F465C1243109F462C172
:100DC000289A0E945D180E942E180E9448110E94C5
:100DD000432C0E94561C0E94D22A0E94B46278942E
:100DE00086E091E09F938F931F920E9473140F905F
:100DF0000F900F9087E690E09F938F938CE490E0A4
:100E00009F938F931F921F92809102016AE00E942C
:100E1000546C892F99279F938F93809102010E9490
:100E2000546C99279F938F938CE291E09F938F93BB
:100E30001F920E9473148DB79EB70D960FB6F8944B
:100E40009EBF0FBE8DBF80E691E09F938F931F9250
:100E50000E9473140F900F900F9080EB91E09F937E
:100E60008F931F920E9473140F900F900F9088ED34
:100E700091E09F938F931F920E9473148091C800FA
:100E80000F900F900F90803209F4F4C0809102010E
:100E90008C3008F0C0C0299A49E061EE78E083E028
:100EA0000E945A05C8EED3E0DE010E94C46C802D7A
:100EB000813009F4B9C08EEF91E09F938F931F9218
:100EC0000E9473140F900F900F9023ED35E0F901FD
:100ED0008FE0158616861786108A8150349687FF14
:100EE000F8CF80E48093E0058093E1051092E2055D
:100EF0008093E3058093E40590EC9093E5051092D0
:100F0000E6058093E7058093E8051092E905909344
:100F1000EA059093EB058093EC051092ED05809324
:100F2000EE059093EF0581E08093D30544ED55E005
:100F30008BE0E4E0F1E0DA0101900D928A95E1F7AF
:100F40008DE4DE01F901182E0E94DD6C809185038D
:100F500099279F938F935F934F938FE192E09F9395
:100F60008F931F920E9473148DB79EB707960FB68A
:100F7000F8949EBF0FBE8DBF80E492E09F938F9345
:100F80001F920E947314109247041092FF030E9454
:100F9000AE3F0F900F900F908091FF038823E1F3F5
:100FA0001092470480ED97E00E94F217EC01CC24E8
:100FB000DD2472E5A72E72E0B72E1092FF030E9487
:100FC000AE3F8091FF038823E1F3F601EE0FFF1F90
:100FD000EE0FFF1FED52FA4F858518160CF054C026
:100FE00086010E55174FCE010E94FB17882309F08A
:100FF0004EC0D8018C91882309F049C08093FF032B
:101000000E94AE3F8091FF038823E1F3ECCF199B50
:101010002FC024E190CE29983FCF8BE095E0A0E04F
:10102000B0E0C0CE2BE087CEA1E0B0E00E94C46C5F
:10103000802D8F3F09F43FCF1092850323ED35E0DB
:101040008DE4DE01F901182E0E94CC6C909185038D
:10105000F9013D962FE08081349618160CF49F5FBD
:10106000215027FFF8CF9093850344ED55E06ECFD4
:101070002AE061CE8091CA00863009F007CF0E9435
:101080002E6704CF28989DCE86010E55174FF80184
:101090008081882309F03FC086010F5F1F4F6801E0
:1010A0000C30110508F489CFCC24DD2456E5A52E9B
:1010B00052E0B52EC1E025C0F601EE0FFF1FEE0F86
:1010C000FF1FED52FA4F858518160CF586010F5F4C
:1010D0001F4F1F930F93BF92AF929F930E94731461
:1010E000C093F9030F900F900F900F900F9086E828
:1010F00098E0C80ED91ED6011C9268010C3011056B
:10110000D0F4F601EE55F74F90819923A9F28601AC
:101110000F5F1F4FECCF86010F5F1F4F1F930F9381
:10112000BF92AF921F920E9473140F900F900F9076
:101130000F900F90B4CF84E792E09F938F931F920C
:101140000E9473140E94AE3F0F900F900F90A1E089
:10115000B0E00E94C46C802D803509F029C20EE0F9
:1011600010E0D8010E94C46C802D9927582F442785
:1011700048010894811C911CD4010E94C46C802DEC
:10118000480F511DECEFAE2EEFEFBE2EA00EB11E9C
:10119000D5010E94C46C802D9927382F22276DEF2E
:1011A000C62E6FEFD62EC00ED11ED6010E94C46C83
:1011B000802D280F311DEFEF2F3F3E0709F4B9C2F4
:1011C000FFEF4F3F5F0709F4B4C23093D70320937A
:1011D000D6035093D9034093D8038091D6039091BE
:1011E000D7039F938F938091D8039091D9039F93B6
:1011F0008F9381EE92E09F938F931F920E947314BE
:101200008DB79EB707960FB6F8949EBF0FBE8DBFE1
:10121000A4E0B0E00E94C46C802D853008F0B8C214
:101220000E94B20545E661EE78E00E945A050E94F0
:10123000B20599279F938F938BE193E09F938F93B0
:101240001F920E9473148091E9080F900F900F90E5
:101250000F900F9080FD7BC20E94083D809102019B
:101260008A3009F472C2843109F46FC2289A80ED81
:1012700097E09093FC038093FB0385E580938007C0
:1012800088E593E09F938F931F920E94731480913F
:10129000E9080F900F900F9082FF54C284E693E00C
:1012A0009F938F931F920E9473140F900F900F9033
:1012B0000E941D2288E893E19093AD038093AC03D4
:1012C00081E080937F070E94FD0582E893E09F9371
:1012D0008F931F920E94731480ED97E00E94F21783
:1012E000EC010F900F900F908091FF03882309F479
:1012F000A1C080911903882309F49CC01092FF03B8
:1013000080917E07882309F4D0C00E94C4050E9402
:10131000AE3F209102012A3009F4D0C0243109F4F3
:10132000CDC0289A8091DE04882309F4CDC0809135
:10133000DE0481508093DE048091C205882369F029
:1013400081508093C205882341F41092C005109209
:10135000BF051092BE051092BD058091AC0390911F
:10136000AD0301979093AD038093AC038091AC03E0
:101370009091AD03892B29F080914604882309F4CC
:10138000D7C08091AC039091AD03892B09F4D6C0EE
:1013900080911203909113038F5F9F4F09F4E7C070
:1013A0008091FF03882321F08091D404882311F4D5
:1013B0000E9484110E946D0ECE010E94FB178823AB
:1013C000B9F1649680910F03882309F489C0815094
:1013D00080930F0380910001282F332780912703EA
:1013E00090912803821793070CF074C08091AD048C
:1013F00080628093AD0480911203909113038F5FFC
:101400009F4F09F4C8C00E94A66584E08093FA0348
:101410008091D404882321F45AEAE52E55E0F52E74
:101420000894E11CF11CF2E7EF16FBE0FF0651F017
:101430000E948E668091FA03882309F055CF0E949E
:10144000EA6552CFEE24FF242091D8033091D903CE
:101450002F5F3F4F3093D9032093D8038091D60359
:101460009091D70301969093D7038093D603832F4F
:101470009927D801082E0E94D16C8091D803D401FD
:10148000082E0E94D16C8091D703D501082E0E94AE
:10149000D16C8091D603D601082E0E94D16C84E1D4
:1014A00090E00E94F217EC01C3CF0E94C7430E9454
:1014B000AE3F209102012A3009F030CF2898809168
:1014C000DE04882309F033CF80916F00806280931F
:1014D0006F0032CF8091AD048F7D8093AD0493CFA8
:1014E00080938A071092B9041092B8041092B7043E
:1014F0001092B6041092B5041092B40480911203B5
:10150000909113038F5F9F4F09F064CF8091DE04A9
:10151000882309F05FCF88E99AE39093FC038093D6
:10152000FB0380E09CE0909313038093120352CF5F
:101530002A3079F1243169F1289A32CF0E94E82AC1
:1015400085E090E09093AD038093AC0380915D08BB
:1015500090915E08019690935E0880935D0880915B
:101560001203909113038F5F9F4F09F019CF809161
:10157000D404882309F414CF80E197E29093FC030C
:101580008093FB0380E890E0909313038093120311
:1015900007CF289805CF80E797E19093FC038093CD
:1015A000FB0380E093E090931303809312032BCF0F
:1015B0000E94E42E8AE992E09F938F931F920E94EB
:1015C000731431E0932E0F900F900F90C0E5D0E090
:1015D0008E010F5F1F4F22E0C22ED12CCC0EDD1EDC
:1015E00093E0A92EB12CAC0EBD1E84E0682E712CA8
:1015F0006C0E7D1EB5E04B2E512C4C0E5D1EA6E0F0
:101600002A2E312C2C0E3D1EE2E09E1609F48BC0D2
:10161000F3E09F1609F48AC023E0291508F483C07B
:1016200080910201843168F085E08093FC0810927B
:101630001A098BE18093F8088EE480931709809350
:101640001809DE010E94C46C802D8C3008F068C03F
:10165000D8010E94C46C802D8C3008F061C0D60186
:101660000E94C46C802D8C3008F05AC0D5010E94B5
:10167000C46C802D8C3008F053C0DE010E94C46C15
:10168000802D8093E108D8010E94C46C802D809346
:10169000E208D6010E94C46C802D8093E308D50136
:1016A0000E94C46C802D8093E408D3010E94C46C16
:1016B000802D8093E508D2010E94C46C802D809318
:1016C000E608D1010E94C46C802D8093E708A7E54D
:1016D000B0E00E94C46C802D8093E80881E09816E9
:1016E00051F4A9EAB2E0BF93AF931F920E94731422
:1016F0000F900F900F9045E661EE78E0892D0E94E3
:1017000083059394B5E0B91508F07ECF83E00E947D
:10171000770580E5A1E0B0E0082E0E94D16C1FCDD6
:101720000E94CB2EE8CF0E94B12F7ACF0E947C304E
:1017300077CF1092D9031092D8031092D70310924A
:10174000D6034BCD80E793E0ABCD289890CD83E3D3
:1017500093E09F938F931F920E94731488EE93E0FF
:101760000E94F217EC010E945C1C0F900F900F90EA
:10177000CE010E94FB178823D9F383E593E09F9362
:101780008F931F920E9473140F900F900F9064CD4F
:1017900084E093E09F938F931F920E9473140F90A5
:1017A0000F900F903DCD1F920F920FB60F92112404
:1017B0008F939F93EF93FF93809111038823A9F454
:1017C0008091ED039091EE030196FC01E05DF94FED
:1017D000E081ED3079F08639910561F09093EE0368
:1017E0008093ED03E093C6000EC01092EE031092BA
:1017F000ED0309C01092EE031092ED0381E0809397
:101800001103E093C600FF91EF919F918F910F908C
:101810000FBE0F901F9018951F920F920FB60F9248
:1018200011242F933F934F935F938F939F93AF9385
:10183000BF93EF93FF9390E08091C6008093E50300
:101840005091F303563910F09093F4038091E5031F
:101850008D3091F02091F403822F992781309105EA
:1018600009F46CC0823091050CF48EC0029709F423
:101870007FC01092F403A8C02091F403223061F7D6
:101880009093F403852F99278357984FFC01329743
:1018900040812091EF033091F003241B3109DC01DA
:1018A00011978C91281B3109C9019F709093F00307
:1018B0008093EF030024880F991F001C880F991F45
:1018C000001C892F902D982F935C9093F1032F7318
:1018D0003070235C2093F2038081891709F46EC075
:1018E00090E08091E2038F5F8093E2033091E40304
:1018F000332309F069C0992309F466C081E080931D
:10190000E403580F5093E1035150E52FFF27E357AD
:10191000F84F8DE0808380918F07823509F054C0A5
:1019200088E190E02CE00FB6F894A89580936000D1
:101930000FBE209360003093F90346C02F5F2093C1
:10194000F403E52FFF27E357F84F8091E5038083E9
:101950005F5F5093F3032091E5038091EF03909133
:10196000F003820F911D9093F0038093EF032CC03E
:10197000E52FFF27E357F84F8091E5038083563921
:1019800038F31092F403E7CF892B09F072CF8091DE
:10199000E503833259F08091E50380938D0781E060
:1019A0008093F3038091E5039927DDCF8091E403D1
:1019B000882389F781E08093F403EDCF8C9182171F
:1019C00009F08ECF91E092CFFF91EF91BF91AF914F
:1019D0009F918F915F914F913F912F910F900FBEEB
:1019E0000F901F901895AC01A0E0B0E09D01A817E2
:1019F000B90748F4E0E3F6E08191280F311D119614
:101A0000A417B507C8F33F70FD01E05DF94FC901A8
:101A10000024880F991F001C880F991F001C892F14
:101A2000902D835C80831196FD01E05DF94F2F734B
:101A30003070822F835C8083AF5CB94F8DE08C93D4
:101A400010921103809130068093C6000895BF92D2
:101A5000CF92DF92EF92FF920F931F93CF93DF937A
:101A6000CDB7DEB72C859D857E85BB2483E2809330
:101A700030069F59909331062093320603E010E020
:101A8000772309F4ADC0CF84D88843E1E42EF12C4C
:101A9000EC0EFD1EA989BA897150109709F4A0C0F7
:101AA000109709F43CC0F601EB0DF11DB394908141
:101AB000119789F47723A1F1F70122E030E0E20EDB
:101AC000F31ED701C080D180E20EF31E0D90BC91B1
:101AD000A02DBB247150109719F1F601EB0DF11DEB
:101AE000B3944081119709F466C01097D1F0F601C4
:101AF000EB0DF11DB39460811197A1F4772391F060
:101B0000F7013296D701CD90DC9032E0E32EF12C34
:101B1000EE0EFF1EA081B181BB24715003C090E086
:101B200040E060E0F801E05DF94F892F86958695E9
:101B3000835C80830F5F1F4FF801E05DF94F892FB1
:101B400099278370907082959295907F9827807FD7
:101B5000982755279A01329522952F7023273F7099
:101B60002327822B835C80830F5F1F4FF801E05D8A
:101B7000F94F4F705070440F551F440F551F862F5B
:101B800099270024880F991F001C880F991F001C9B
:101B9000892F902D842B835C80830F5F1F4FF8016A
:101BA000E05DF94F6F73635C60830F5F1F4F1097A9
:101BB00009F076CF15C0772309F4B3CFF701A2E07F
:101BC000B0E0EA0EFB1ED701C080D18022E030E0F9
:101BD000E20EF31E0D90BC91A02DBB24715085CF59
:101BE000C8010E94F30CDF91CF911F910F91FF90DC
:101BF000EF90DF90CF90BF900895A3E07A2F4091AF
:101C0000E103465009F45FC0E72FFF27E357F84F81
:101C100080818D537F5FE72FFF27E357F84F2081A7
:101C20002D537F5FE72FFF27E357F84F30813D5358
:101C30007F5FE72FFF27E357F84F60816D537F5F8A
:101C40009927880F991F880F991F522F52955F70FF
:101C5000582B822F99278F70907082959295907F44
:101C60009827807F9827232F26952695282B832F2A
:101C70009927837090700024969587950794969580
:101C800087950794982F802D682B41504F3FD9F0AE
:101C9000EA2FFF27E357F84F5083AF5F41504F3F84
:101CA00091F0EA2FFF27E357F84F2083AF5F4150B1
:101CB0004F3F49F0EA2FFF27E357F84F6083AF5FAC
:101CC000442309F0A1CF80E997E09093E00380934B
:101CD000DF03A350A093DE030895CF93DF93CDB726
:101CE000DEB722970FB6F894DEBF0FBECDBF80914E
:101CF000E403882309F4AFC20E94FD0D80918E0792
:101D0000823609F471C080918F0799278436910536
:101D100009F457C08536910584F58136910509F49B
:101D20004EC1823691050CF4C2C08236910509F489
:101D30009AC183369105C1F48091DA039091DB0357
:101D4000892B09F04FC2A091DF03B091E0039C9171
:101D5000992309F03DC29C918AE0989FC00111240B
:101D60009093DB038093DA031092E4031092E00374
:101D70001092DF031092DE036EC28C36910509F4D7
:101D800010C18D3691050CF0B3C08736910509F46A
:101D90002BC18836910541F78FEF80930F03E091B7
:101DA000DF03F091E003808190913F04892B8093C1
:101DB0003F04882311F01092E60381E08093EA0348
:101DC000D3CFE091DF03F091E00390818AE0989F08
:101DD000C001112490930D0380930C03892B21F2F1
:101DE00081E08093E903C0CF80918F0799278037E6
:101DF000910509F4F2C0813791050CF485C0833751
:101E0000910509F45BC1843791050CF03CC1813721
:101E1000910509F078CFA091DF03B091E0038C9198
:101E20008F3F09F40CC28C91882309F003C281E032
:101E30008C93A091DF03B091E00345E661EE78E07A
:101E40008C910E945A05809111038823E1F3E0915F
:101E5000DF03F091E0038081898380E58A8385E652
:101E600090E09F938F9381EE98E09F938F9321E072
:101E700030E03F932F93CE0102969F938F933F9331
:101E80002F93CE01820F931F9F938F9383E08F93A5
:101E900081E08F9381E58F930E94270DADB7BEB788
:101EA0001F960FB6F894BEBF0FBEADBF2CCF8B34BC
:101EB000910509F059CFE091DF03F091E0038081B3
:101EC00091819093F0048093EF042091ED04309180
:101ED000EE04821B930B845E9D4F68E671E00E94C6
:101EE000746C845B90409093EC048093EB043CCF43
:101EF0008437910509F47CC08637910509F034CF09
:101F000081E08093E80330CF8D36910529F18E363C
:101F100091050CF093C08B34910509F0F4CEA0919B
:101F2000DF03B091E0038D919C919093F004809336
:101F3000EF042091ED043091EE04821B930B845E3C
:101F40009D4F68E671E00E94746C845B90409093B2
:101F5000EC048093EB04D7CE809111038823E1F346
:101F6000A091DF03B091E0039C91913009F43FC14F
:101F7000198281E090E09F938F93CE0101969F9309
:101F80008F9381E08F938F938DE48F930E94270D21
:101F90008DB79EB707960FB6F8949EBF0FBE8DBF44
:101FA000B2CE8FEF80930F03E091DF03F091E00357
:101FB00080818093400481E08093EB03D5CEE09153
:101FC000DF03F091E003E081E03258F08FE180938D
:101FD00010038FEF80930F03C7CE81E08093E70358
:101FE00092CEE0931003F5CF81E08093EC03BCCE5A
:101FF0008091E103853108F4DAC0E091DF03F091CC
:10200000E00380E1A8E6B7E001900D928A95E1F740
:10201000809111038823E1F31F9280910E038F9327
:1020200084E58F930E94270D8AEF8093DC038FEF66
:1020300080930F030F900F900F9096CE8E369105E0
:1020400009F061CE809111038823E1F38DE490E0E3
:102050009F938F9383ED95E09F938F9381E08F9370
:102060008F938EE492CFA091DF03B091E0038BE0D9
:10207000E0E8F7E00D9001928A95E1F780918907F9
:1020800080936508A6CF8437910509F03CCE8091F6
:10209000E103853108F4BCC0A091DF03B091E003F7
:1020A00080E1E8E6F7E00D9001928A95E1F780EF94
:1020B0008093DC038FEF80930F0325CE2091DF0305
:1020C0003091E003F90180818150853018F48181DD
:1020D0008035E9F01982809111038823E1F381E0D2
:1020E00090E09F938F93CE0101969F938F9381E011
:1020F0008F938F9383E58F930E94270DEDB7FEB7E3
:1021000037960FB6F894FEBF0FBEEDBFFCCD61EE63
:1021100078E085E62E5F3F4FDB01F901982F0190B3
:102120000D929A95E1F722503040482FD9018C91B9
:102130000E948305809117099927AA27BB27BC0114
:10214000CD0124EC39E040E050E00E94356CDC0128
:10215000CB018093A6039093A703A093A803B09309
:10216000A903809118099927AA27BB27BC01CD0193
:102170000E94356CDC01CB018093A2039093A303F2
:10218000A093A403B093A503E091DF03F091E003D3
:1021900080810E9477050E94B205898380E00E94B9
:1021A000FD056EE670E089810E94C13194CFE09117
:1021B000DF03F091E00380819181A281B38180935C
:1021C000680790936907A0936A07B0936B0720CFC5
:1021D0008AE0989FC00111240E94F21790932F0665
:1021E00080932E06A091DF03B091E003B4CD43EDC0
:1021F00055E08DE4FA01282F0D9001922A95E1F720
:10220000A8EEB3E0FA01182E0E94DD6C9983B1CEDE
:10221000A091DF03B091E0038D919D910D90BC9151
:10222000A02D8093680790936907A0936A07B093E5
:102230006B073DCF863008F400CE85E0F9CD0E94D3
:10224000B205E091DF03F091E0038083A091DF030A
:10225000B091E003E8CD22960FB6F894DEBF0FBE32
:10226000CDBFDF91CF910895CF93C82F8A3029F049
:102270008091C00085FFFCCF04C08DE00E94341126
:10228000F7CFC093C60080E090E0CF910895089505
:1022900088E18093C1008091C00082608093C0007B
:1022A0008091C10080688093C1008091C1008064EA
:1022B0008093C1008AE28093C40080910C039091C6
:1022C0000D030E94F21790935D0780935C078CEDDD
:1022D00090E00E94F21790938C0780938B071092E6
:1022E0005E078CE480935F0786E0809362078AE054
:1022F0008093600781E0809361071092E003109261
:10230000DF031092DE030895EF92FF920F931F9365
:1023100080911103882309F478C28091EA0388230D
:1023200009F082C08091EB03882329F0809111038A
:10233000882309F07FC18091E803882329F08091E8
:102340001103882309F05BC18091EC03882329F0F5
:1023500080911103882309F036C180918B079091F9
:102360008C070E94FB17882329F080911103882392
:1023700009F0C8C080910C0390910D03892B09F0DE
:1023800084C18091E903882329F080911103882377
:1023900009F00FC28091DA039091DB03892B09F0D9
:1023A0007EC1209110032F3F59F180E190E09F936F
:1023B0008F93822F992782959295907F9827807F7F
:1023C0009827845F9E4F9F938F9381E090E09F9327
:1023D0008F9380E193E09F938F9382E08F9381E0CE
:1023E0008F9381E48F930E94270D8FEF80931003CA
:1023F0008DB79EB70B960FB6F8949EBF0FBE8DBFDC
:1024000080916508882329F080911103882309F0C1
:102410005EC08091E703882309F4F7C1809111031E
:10242000882309F4F2C139C080911103882309F48B
:1024300079CF0E94262284E190E09F938F93909120
:10244000E60384E1989FC0011124865D9C4F9F9311
:102450008F9381E090E09F938F9386EE93E09F931C
:102460008F9382E08F9381E08F9388E48F930E9413
:10247000270D8091E6038F5F2DB73EB7255F3F4F55
:102480000FB6F8943EBF0FBE2DBF843008F4B8C11C
:102490001092E6031092EA0345CF86E190E09F9305
:1024A0008F938FEA98E09F938F9381E08F938F9320
:1024B00080E58F930E94270D1092E7038DB79EB79A
:1024C00007960FB6F8949EBF0FBE8DBF9EC181E0E8
:1024D00090E09F938F9385E698E09F938F9381E0A0
:1024E0008F938F9382E48F930E94270D109265083B
:1024F0002DB73EB7295F3F4F0FB6F8943EBF0FBED2
:102500002DBF87CF8091F8089927880F991F880FD2
:10251000991F7C010027F7FC0095102F8091290559
:1025200090912A05A0912B05B0912C05BC01CD01FD
:10253000A80197010E94A96C30937907209378072E
:102540008091210590912205A0912305B091240549
:10255000BC01CD01A80197010E94A96C30937B07B3
:1025600020937A078091C10480937C078091C004F6
:1025700080937D0788E090E09F938F9388E797E0B2
:102580009F938F9381E08F9383E08F9387E78F935F
:102590000E94270D80917E072DB73EB7295F3F4FE0
:1025A0000FB6F8943EBF0FBE2DBF853018F086E001
:1025B00080937E0783E690E00E94F21790938C0749
:1025C00080938B07D7CE8BE090E09F938F9380E82A
:1025D00097E09F938F9381E08F9380910E038F9369
:1025E00087E48F930E94270D1092EC038DB79EB75E
:1025F00007960FB6F8949EBF0FBE8DBFAECE8AE091
:1026000090E09F938F938EE597E09F938F9381E067
:102610008F938F9386E58F930E94270D1092E80386
:102620002DB73EB7295F3F4F0FB6F8943EBF0FBEA0
:102630002DBF8ACE0E94262280E590E09F938F9343
:102640008AE293E09F938F9321E030E03F932F93B2
:1026500089E293E09F938F933F932F9380E494E0DC
:102660009F938F9383E08F9381E08F938CE48F937C
:102670000E94270D1092EB038DB79EB70F960FB6F1
:10268000F8949EBF0FBE8DBF56CE80915C0790918F
:102690005D070E94FB17882309F077CE72CE8091E8
:1026A0002E0690912F060E94FB17882309F479CEFD
:1026B00080911103882309F474CE8091F80899273A
:1026C000880F991F880F991F7C010027F7FC009540
:1026D000102F8091290590912A05A0912B05B0918A
:1026E0002C05BC01CD01A80197010E94A96C309373
:1026F0002106209320068091210590912205A0912A
:102700002305B0912405BC01CD01A80197010E94C9
:10271000A96C30932306209322062091AB093091B7
:10272000AC094091AD095091AE09DA01C90103E04D
:10273000880F991FAA1FBB1F0A95D1F7820F931FFD
:10274000A41FB51F820F931FA41FB51F20918603DE
:10275000309187034091880350918903BC01CD01DA
:102760000E94A96C30932506209324068EE090E009
:102770009F938F9380E296E09F938F9381E08F9356
:102780008F9383E48F930E94270D8091DA039091B9
:10279000DB030E94F21790932F0680932E062DB72D
:1027A0003EB7295F3F4F0FB6F8943EBF0FBE2DBF17
:1027B000F8CD82E490E09F938F9383E298E09F931B
:1027C0008F9381E08F938F9384E48F930E94270DE2
:1027D0001092E9038DB79EB707960FB6F8949EBF87
:1027E0000FBE8DBF80910C0390910D03009709F4EB
:1027F000D1CD0E94F21790935D0780935C07CACDFC
:102800008093E6031092EA038DCD1F910F91FF9004
:10281000EF900895982F80916608813031F0892FCC
:102820000E943411282F33270CC080914104E82FD7
:10283000FF27E65DFC4F90838F5F8093410421E08A
:1028400030E0C90108950F931F93CF93DF938C015C
:10285000EB01672B71F0F80181918F010E940A143E
:10286000219739F0F80181918F010E940A14219774
:1028700091F7DF91CF911F910F9108950F931F93BF
:10288000CF93DF938C01EB01672B81F0F8010F5F91
:102890001F4F84910E940A14219741F0F8010F5FA5
:1028A0001F4F84910E940A14219781F7DF91CF91E5
:1028B0001F910F910895CF93C82F181634F480E21A
:1028C0000E940A14C1501C16D4F3CF910895CF93DF
:1028D000C82F181634F480E30E940A14C1501C1645
:1028E000D4F3CF9108952F923F924F925F926F92BF
:1028F0007F928F929F92AF92BF92CF92DF92EF9290
:10290000FF920F931F93CF93DF93CDB7DEB7E0977E
:102910000FB6F894DEBF0FBECDBF26968FAD2697BB
:102920002896EEADFFAD2897882499245401809312
:10293000660848E4C42ED12CCC0EDD1E7F01C701F1
:10294000F7011491112331F0153221F00894E11CA4
:10295000F11CF6CFB701681B790B09F095C0112364
:1029600009F43DC20894E11CF11C1FA63FA4232CCE
:102970000FEF39A6F7010894E11CF11C14911537EB
:10298000C9F1812F80628837A9F1103209F440C063
:10299000133209F48DC01A3209F479C01D3209F4DA
:1029A00076C01B32C9F11E32C9F1103309F48AC056
:1029B000812F8153893008F07EC060E070E0CB0148
:1029C000880F991F880F991F880F991F860F971FCF
:1029D000680F791F610F711D60537040F7010894F3
:1029E000E11CF11C1491812F80538A3040F3262E74
:1029F000153739F630FE3DC0F60184E090E0C80E90
:102A0000D91E80809180A280B380103209F0C0CF9F
:102A100089A5882309F0AECF19A7ACCFF701089498
:102A2000E11CF11C14911A3209F451C060E070E00D
:102A300014C0CB01880F991F880F991F880F991F09
:102A4000860F971F680F791F610F711D60537040CB
:102A5000F7010894E11CF11C1491812F80538A30F6
:102A600040F3EFEF6F3F7E0714F46FEF7FEF062F19
:102A700086CFF60182E090E0C80ED91E8081918158
:102A80004C01AA24BB2481CF0E943E1468CF1A3285
:102A900051F4F60182E090E0C80ED91E2080222079
:102AA0000CF068CF219490E1392AEFED3E2262CFFD
:102AB00098E0392A5FCF1836C9F01C36D1F481E08E
:102AC000382A58CF34FC56CFF0E23F2A53CFF601D4
:102AD00082E090E0C80ED91E608171819FEF6F3F48
:102AE000790714F46FEF7FEF062F44CF24E0322AEA
:102AF00041CF133609F44DC1143409F41FC1143603
:102B000009F41CC1193609F419C11F3409F40FC1A5
:102B10001F3609F40CC1103709F4F9C0133709F452
:102B2000B2C0153509F4ECC0153709F4E9C0183501
:102B300009F444C0183709F441C0112309F44FC106
:102B4000CE0101969DA78CA7198381E0482E19A676
:102B5000632C7724042D5FA4541857FC2DC029A59D
:102B6000222331F10F5F050DC30180739070892B13
:102B700009F42FC1222309F027C166FC1BC1C30140
:102B800080739070809709F410C1852D0E9467149E
:102B9000842D992787FD9095BC018CA59DA50E9449
:102BA000231464FECCCE822D801B0E945B14C7CE02
:102BB00066FED9CF0E5FD7CF5524D1CFE0E1EEA787
:102BC00033FE07C081149104A104B10411F0F0E4B4
:102BD0003F2A19A60FA707FD02C02FED3222CE0112
:102BE00089969DA78CA781149104A104B10419F4BE
:102BF0009FA5992361F1EEA54E2E552466247724D6
:102C000018AA84149504A604B70410F0F1E0F8ABF8
:102C1000C501B401A30192010E94876CDC01CB01C4
:102C2000082F8A30F0F4005DECA5FDA50293FDA706
:102C3000ECA7C501B401A30192010E94876C490170
:102C40005A01F8A9FF23E1F62EA5283079F0632C6C
:102C50007724CE010196482EFCA54F1A28E2420E99
:102C600079CF095A183501F70F7DDECF632C772411
:102C700063FEEFCF003369F380E3ECA5FDA58293FB
:102C8000FDA7ECA7E6CFF60182E090E0C80ED91EC2
:102C90000190F081E02DFDA7ECA7EF2B81F4FE0160
:102CA0003196FDA7ECA788E289838EE6818385E7CC
:102CB0008B838CE68C838D8389E28E831F8207FD54
:102CC00015C0802F992787FD9095AC0160E070E0DA
:102CD0008CA59DA50E944E6B009731F0482EFCA557
:102CE0004F1A04150CF033CF402E31CFECA5FDA5C3
:102CF00001900020E9F731974E2E2CA5421A27CFDC
:102D0000153511F481E0382A9AE09EA762CFF601CA
:102D100082E090E0C80ED91E808191814C01AA24E6
:102D2000BB2490E19EA7E0E43E2A18E752CF1F346F
:102D300011F4E1E03E2AF8E0FEA74BCF143411F481
:102D400091E0392A30FE18C0F60184E090E0C80E08
:102D5000D91E80809180A280B380B7FE0AC0B09453
:102D6000A09490948094811C911CA11CB11C8DE2B4
:102D700089A79AE09EA72ECFF60182E090E0C80EC8
:102D8000D91E808191814C01AA2497FCA094BA2C71
:102D9000E4CFFE013196FDA7ECA7F60182E090E0BA
:102DA000C80ED91E80818983D0CE822D801B0E94BF
:102DB0006714EBCE80E38AA71BA762E070E0CE0128
:102DC0008A960E942314DBCE61E070E0CE018996E2
:102DD000F8CF822D801B0E945B1429A5CBCEE096F4
:102DE0000FB6F894DEBF0FBECDBFDF91CF911F911C
:102DF0000F91FF90EF90DF90CF90BF90AF909F909A
:102E00008F907F906F905F904F903F902F9008959C
:102E10001F920F920FB60F9211242F933F935F933F
:102E20006F937F938F939F93AF93BF93EF93FF9392
:102E30008091FA03882329F08091FA0381508093CE
:102E4000FA038091CE05882319F081508093CE0536
:102E50008091020481508F3F09F493C08093020453
:102E60008091FB039091FC03892B01F18091FB037E
:102E70009091FC0301979093FC038093FB03809156
:102E8000FB039091FC0320911203309113038223E2
:102E90009323892B89F0809102018A3009F48BC039
:102EA000479A8091E90883FF8DC010C08FEF9FEF94
:102EB0009093130380931203809102018A3009F4E6
:102EC00078C047988091E90883FF7CC086B1992734
:102ED000FC01E071F07084FF0AC08091FD039091C5
:102EE000FE0301969093FE038093FD036BC08091D7
:102EF000FD039091FE03892B49F18091FD03909190
:102F0000FE038A56914010F58091FD039091FE03D7
:102F100069E270E00E94606C8091FD039091FE0375
:102F2000860F971F9093FE038093FD038091FD030E
:102F30009091FE030B9708F440C08091FD0390919F
:102F4000FE030A979093F0048093EF048091EF04BE
:102F50009091F0042091ED043091EE04821B930BCC
:102F6000845E9D4F68E671E00E94746C845B9040C3
:102F70009093EC048093EB041092FE031092FD03F7
:102F800021C089E080930204809114038F5F8170D7
:102F900080931403882319F481E08093FF038091C8
:102FA0000004909101040196909301048093000421
:102FB00057CF5A9887CF5A9A85CFF093F004E09371
:102FC000EF04C4CFFF91EF91BF91AF919F918F918B
:102FD0007F916F915F913F912F910F900FBE0F9056
:102FE0001F9018952091000430910104280F391F7B
:102FF000C901019608952091000430910104821BBB
:10300000930B892F99278695807490700895CF939C
:10301000DF930E94F217EC01CE010E94FB17882378
:10302000D9F3DF91CF9108951F93CF93DF930E943F
:10303000F217EC011FEC08C080911903882321F0DE
:103040009093190310937A00CE010E94FB17982FDA
:10305000882391F3DF91CF911F9108959FB7F89442
:103060005F983E9A469A8091B0008F708093B0002E
:103070008091B00083608093B0008091B1008B7329
:103080008093B1008091B1008B608093B100109269
:10309000B2008FEF8093B3008091B000806880937E
:1030A000B000809170008A7F8093700080917000E2
:1030B0008260809370009FBF08958AE090E00E9434
:1030C000F21790930A048093090482E085BD83EA95
:1030D00084BD17BC88E788BD86E086BD80916E0000
:1030E000816080936E0008951F920F920FB60F9229
:1030F00011242F933F934F935F936F937F938F93FD
:103100009F93AF93BF93EF93FF938091020184311C
:10311000C0F480910304882309F446C0209104047C
:103120003091050441E02F37340708F49CC08FEF3D
:103130008093B3002F5F3040309305042093040444
:10314000A4C380910304882349F78091B00086FFCF
:10315000ADC08091B0008F7B8093B000E0910804F7
:10316000EE2309F0EFC080911009282F33278DED51
:1031700096E0289FA001299F500D389F500D1124E3
:10318000CA012091060430910704821B930B90938F
:103190000504809304041092070410920604469AD2
:1031A00081E080930304BACF8091B00086FFA8C06D
:1031B0008091B0008F7B8093B00089EA93E0909378
:1031C00005048093040480911503909116039C01DB
:1031D000220F331F280F391F809192039927880FE0
:1031E000991F880F991F280F391F37FD25C2C90164
:1031F00095958795959587959093160380931503DC
:103200009093F8038093F7038091380980FFDDC025
:1032100080910909682F7727882799272091290508
:1032200030912A0540912B0550912C0557FDE9C19D
:10323000A7E05595479537952795AA95D1F70E9410
:10324000356C9B01AC0197FDFAC1F6E055954795A9
:1032500037952795FA95D1F78091F7039091F80368
:10326000820F931FDCC02F3F310569F060F0A90188
:103270004F5F50404F37510588F480E88093B3008A
:103280002058304059CF809104048093B3001092AD
:1032900005041092040410920304F7C28FEF809388
:1032A000B3005093050440930404EFC28091B00032
:1032B00080648093B0008CEB90E090930504809341
:1032C0000404809106049091070484549F4F9093C6
:1032D0000704809306048091F903882329F08091E4
:1032E000DE04853B08F0F2C0469A909108049F5F87
:1032F00080911009891708F0E6C01092080450CF99
:103300008091B00080648093B00080911009282FD4
:1033100033278DED96E0289FA001299F500D389FFF
:10332000500D1124CA012091060430910704821B1C
:10333000930B90930504809304049C0181E0809397
:103340000304F0CE89EA93E090930504809304048B
:103350008E2F99278130910509F4BAC0029709F49C
:1033600078C1FF27EE0FFF1FE155F74F8081918154
:10337000880F991F2091040430910504820F931F38
:103380009093050480930404209104043091050473
:1033900055E02D3D350708F440C18CED95E0909344
:1033A0000504809304049C012C5B30403093050499
:1033B000209304048091060490910704820F931FC8
:1033C0009093070480930604EBCE80910909682F3F
:1033D0007727882799272091290530912A05409140
:1033E0002B0550912C0557FD07C1E7E055954795F2
:1033F00037952795EA95D1F70E94356C9B01AC0172
:1034000097FD22C176E055954795379527957A9592
:10341000D1F78091F7039091F803821B930B90935F
:10342000F8038093F70380910A09282F3327220F8E
:10343000331F220F331F8091F7039091F8038217F7
:1034400093077CF080910B09282F3327220F331F1D
:10345000220F331F8091F7039091F8032817390743
:1034600024F43093F8032093F7032091F70330916D
:10347000F8038091040490910504280F391F20500F
:1034800032408091F7039091F80397FDD3C0959552
:103490008795959587959093F8038093F70345E07A
:1034A0002D3D340708F4B2C08CED95E090930504EF
:1034B00080930404209104043091050430930704A0
:1034C000209306043BCF909308046ACE46980DCF14
:1034D00080911503909116039C01220F331F280F32
:1034E000391F809192039927880F991F880F991F80
:1034F000280F391F37FD99C1C90195958795959575
:10350000879590931603809315039093F803809307
:10351000F7038091380980FF30C180910909682F35
:103520007727882799272091290530912A054091EE
:103530002B0550912C0557FD85C1E7E05595479522
:1035400037952795EA95D1F70E94356C9B01AC0120
:1035500097FD73C1B6E05595479537952795BA9570
:10356000D1F78091F7039091F803820F931F909306
:10357000F8038093F70380910A09282F3327220F3D
:10358000331F220F331F8091F7039091F8038217A6
:1035900093077CF080910B09282F3327220F331FCC
:1035A000220F331F8091F7039091F80328173907F2
:1035B00024F43093F8032093F7038091F70390915C
:1035C000F8032091040430910504820F931F80506A
:1035D000924090930504809304048091F7039091A6
:1035E000F80397FD20C195958795959587959093BC
:1035F000F8038093F703C8CE21583F4F4F4F5F4FDA
:10360000F4CE21583F4F4F4F5F4F12CE51E0273736
:10361000350758F487E791E049CF81E0273738072D
:1036200008F0C2CE87E791E0BACE3093050420932C
:10363000040440CF03962BCF2D5F3F4FD8CD215CA4
:103640003F4F4F4F5F4F01CE215C3F4F4F4F5F4F7A
:10365000D9CE80911703909118039C01220F331F3C
:10366000280F391F809191039927880F991F880F80
:10367000991F280F391F37FDDBC0C9019595879524
:103680009595879590931803809317039093F6036D
:103690008093F5038091380981FF9AC080910D09CC
:1036A000682F7727882799272091210530912205B7
:1036B000409123055091240557FDE2C0A7E05595A0
:1036C000479537952795AA95D1F70E94356C9B01B0
:1036D000AC0197FDD0C0F6E05595479537952795F5
:1036E000FA95D1F78091F5039091F603820F931F1D
:1036F0009093F6038093F50380910E09282F3327CA
:10370000220F331F220F331F8091F5039091F60390
:10371000821793077CF080910F09282F3327220FFF
:10372000331F220F331F8091F5039091F603281762
:10373000390724F43093F6032093F5038091F503C1
:103740009091F6032091040430910504820F931F99
:103750008050924090930504809304048091F50377
:103760009091F60397FD67C09595879595958795F8
:103770009093F6038093F50307CE80910909682F93
:103780007727882799272091290530912A0540918C
:103790002B0550912C0557FD5FC0A7E05595479527
:1037A00037952795AA95D1F70E94356C9B01AC01FE
:1037B00097FD4DC0F6E05595479537952795FA95B5
:1037C000D1F78091F7039091F803821B930BCFCE32
:1037D00080910D09682F7727882799272091210547
:1037E00030912205409123055091240557FD3EC09C
:1037F000E7E05595479537952795EA95D1F70E94CB
:10380000356C9B01AC0197FD2CC066E05595479542
:10381000379527956A95D1F78091F5039091F60336
:10382000821B930B65CF0396DECE2D5F3F4F64CE98
:103830002D5F3F4F22CF039697CF215C3F4F4F4FD5
:103840005F4F88CE21583F4F4F4F5F4F76CE215C60
:103850003F4F4F4F5F4FAECF21583F4F4F4F5F4FBE
:103860009CCF215C3F4F4F4F5F4FCFCF21583F4FF1
:103870004F4F5F4FBDCF215C3F4F4F4F5F4F2BCF1F
:1038800021583F4F4F4F5F4F19CFFF91EF91BF919D
:10389000AF919F918F917F916F915F914F913F91E8
:1038A0002F910F900FBE0F901F90189510927C00D3
:1038B0008FEC80937A000895EF92FF920F931F93FD
:1038C000CF93DF9303E010E0D8010E94C46C802DF9
:1038D000C82FDD27C531D10508F02A97C7BD109242
:1038E000120484E690E00E94141880911D039091C8
:1038F0001E038052934010F4C0E0D0E0CA3FD105CF
:10390000E0F48AEAE82E83E0F82EC7BD82E390E077
:103910000E941418FF92EF921F920E9473148091DC
:103920001D0390911E030F900F900F9080529340B3
:1039300020F02196CA3FD10540F3D8010C2E0E94F9
:10394000D16CC09373088CE291E00E941418DF914F
:10395000CF911F910F91FF90EF900895EF92FF92FA
:103960000F931F93CF93DF9300E000930D04009318
:103970000C0400930B0480ED97E00E94F217EC0119
:103980001CE821E0F22E95EFE92E033009F4ABC0DC
:1039900000E080912204909123048C5F93400CF00E
:1039A00091C080911C03815080931C03809120045E
:1039B000909121048C5F93400CF079C080911B039F
:1039C000815080931B0380911E0490911F048C5F93
:1039D00093400CF04AC080911A03815080931A03DF
:1039E00088E0809349040E94D82A80911C038A3081
:1039F00008F055C0F0920D048AE080931C0380917A
:103A00001B038A3008F043C0F0920C048AE08093D4
:103A10001B0380911A038A3098F5F0920B048AE018
:103A200080931A0380914904882379F0CE010E9483
:103A3000FB178823B9F38CEA93E09F938F931F922F
:103A40000E9473140F900F900F90109219038FEC37
:103A500080937A00809119038823E1F31A3008F4E7
:103A600047C0115009F091CF48C080911E04909139
:103A70001F04875094408CF180911A038F5FAECF62
:103A8000863F80F2F0920B04E0921A03CBCF863F80
:103A900008F4BFCFF0920C04E0921B03BACF863F2C
:103AA00008F4ADCFF0920D04E0921C03A8CF8091F2
:103AB000200490912104875094408CF080911B0346
:103AC0008F5F7FCF80912204909123048750944090
:103AD00044F080911C038F5F67CF0F5F81CF0F5F32
:103AE00072CF01E063CF1B3008F452CF19E050CF02
:103AF0008AE090E00E941418B4CF86E490E00E941F
:103B00001418DF91CF911F910F91FF90EF900895BE
:103B10001F920F920FB60F921124AF92BF92CF92C5
:103B2000DF92EF92FF920F931F932F933F934F9348
:103B30005F936F937F938F939F93AF93BF93EF9315
:103B4000FF9320912B04822F9927AA27BB272F5F51
:103B5000FC01429740F4E25CFF4FEE0FFF1F05901F
:103B6000F491E02D099410922B0482E080932A04B2
:103B700080912A0480937C0080912B04882309F48F
:103B800043C48FEC80937A003FC420932B04809130
:103B90007800909179002091300430913104820FA7
:103BA000931F909331048093300481E0DFCF209302
:103BB0002B04809178009091790020912E0430910F
:103BC0002F04820F931F90932F0480932E0484E080
:103BD000CDCF20932B048091780090917900209193
:103BE000370530913805821B930B909372088093B0
:103BF00071088091710890917208909339048093B4
:103C0000380482E0B3CF20932B0480913505909146
:103C100036052091780030917900821B930B9093A8
:103C2000680880936708809167089091680890936E
:103C300037048093360487E099CF20932B0480913A
:103C400078009091790090932D0480932C0486E065
:103C50008DCF20932B042091780030917900309300
:103C60002F0420932E0410922A0482CF20932B0439
:103C70002091780030917900309331042093300402
:103C800081E074CF10922B0481E08093190380911E
:103C90000E0490910F04019690930F0480930E04EC
:103CA000809178009091790090931E0380931D037A
:103CB00080911D0390911E035C01CC24DD24809132
:103CC0003A0490913B04A0913C04B0913D04A80EAD
:103CD000B91ECA1EDB1E80913E048F5F823108F43C
:103CE000E8C280911F0390912003A0912103B0911D
:103CF00022037C018D0123E0EE0CFF1C001F111F2D
:103D00002A95D1F7E81AF90A0A0B1B0BEA0CFB1CDF
:103D10000C1D1D1D80911204992787FD9095A92FD8
:103D2000B92FBC01CD0126EC34E240E050E00E9406
:103D3000356CDC01CB01E81AF90A0A0B1B0BD80120
:103D4000C7010496A11DB11DB7FD23C313E0B595AE
:103D5000A795979587951A95D1F780931F03909310
:103D60002003A0932103B093220380916B089091CC
:103D70006C087C010027F7FC0095102F80911F0331
:103D800090912003A0912103B0912203E81AF90A2F
:103D90000A0B1B0BE092D004F092D1040093D204E2
:103DA0001093D3042091130430911404409115040E
:103DB0005091160457FDFDC2A4E0559547953795DF
:103DC0002795AA95D1F78091130490911404A0919E
:103DD0001504B0911604821B930BA40BB50B8093B2
:103DE000130490931404A0931504B09316048091C7
:103DF000130490911404A0911504B09116048E0D33
:103E00009F1DA01FB11F8093130490931404A093CF
:103E10001504B09316048091100490911104BC0114
:103E200062957295707F7627607F7627681B790B85
:103E300020911304309114044091150450911604FC
:103E400057FDB2C2E4E05595479537952795EA9519
:103E5000D1F78091D0049091D104821B930B880FED
:103E6000991F880F991F880F991F860F971F97FD1D
:103E7000A9C29595879595958795959587959595DB
:103E800087959093110480931004D601C501D7FC47
:103E900095C2B595A7959795879580933A04909389
:103EA0003B04A0933C04B0933D0489E080933E041E
:103EB00082E05CCE20932B04209178003091790031
:103EC00080912E0490912F04280F391F80910201B8
:103ED0008A3009F448C2220F331F220F331F309358
:103EE0002F0420932E04C90137FD73C29595879541
:103EF00095958795959587959093210480932004B7
:103F00008091340490913504820F931F97FD66C20F
:103F100095958795909335048093340420913F05BF
:103F200030914005821B930B9093240380932303CD
:103F3000209126043091270480912303909124033B
:103F4000280F391F37FD47C2359527953093270431
:103F50002093260483E00ACE20932B04209178003E
:103F6000309179008091300490913104280F391FED
:103F7000809102018A3009F407C2220F331F220FF9
:103F8000331F3093310420933004C90137FDFFC142
:103F90009595879595958795959587959093230405
:103FA000809322048091320490913304820F931FF6
:103FB00097FD0DC2959587959093330480933204B5
:103FC0002091410530914205821B930B909326036B
:103FD00080932503209128043091290480912503A2
:103FE00090912603280F391F37FDEEC1359527958F
:103FF000309329042093280481E0B8CD20932B042A
:1040000080917800909179002091370530913805A2
:10401000821B930B909372088093710880917108B2
:10402000909172082091380430913904820F931FC7
:1040300090931B0480931A0482E098CD20932B0464
:104040008091350590913605209178003091790066
:10405000821B930B90936808809367088091670890
:10406000909168082091360430913704820F931F95
:1040700090931D0480931C0487E078CD20932B043B
:10408000809102018A3009F471C1843109F4A8C118
:10409000809178009091790020912C0430912D042A
:1040A000820F931F90931F0480931E0486E05ECDC1
:1040B00020932B04809178009091790020912E0418
:1040C00030912F04820F931F90932F0480932E041E
:1040D00010922A044DCD20932B04E2CD20932B0483
:1040E0008091780090917900AA2797FDA095BA2F2A
:1040F000BC01CD010E94BB6B7B018C0180912F051F
:1041000090913005A0913105B09132059C01AD012F
:10411000C801B7010E945B6BDC01CB01BC01CD0182
:104120000E949E6BDC01CB019093190480931804CC
:10413000809118049091190402970CF4C6C08091E4
:104140002F0590913005A0913105B091320520E006
:1041500030E84BE354E4BC01CD010E94C56B8823D9
:10416000DCF580912F0590913005A0913105B0913B
:1041700032052AE037ED43EA5CE3BC01CD010E9441
:104180005C6BDC01CB0180932F0590933005A093ED
:104190003105B09332058091AE049091AF04845FF5
:1041A0009140D0F480912F0590913005A091310578
:1041B000B09132052DEC3CEC4CEC5DE3BC01CD0143
:1041C0000E945C6BDC01CB0180932F05909330053E
:1041D000A0933105B093320581E08093170480915C
:1041E00078009091790090936A0880936908809193
:1041F000180490911904AA2797FDA095BA2F209131
:10420000F1043091F2044091F3045091F404820FD0
:10421000931FA41FB51F8093F1049093F204A09301
:10422000F304B093F4042091F1043091F20440912E
:10423000F3045091F40457FDB2C00AE05595479538
:10424000379527950A95D1F78091F1049091F20462
:10425000A091F304B091F404821B930BA40BB50B53
:104260008093F1049093F204A093F304B093F404C8
:1042700083E07CCC20932B0480912703909128032A
:104280009C01220F331F280F391F809178009091D5
:10429000790063E070E00E94606C260F371F36954E
:1042A000279536952795309328032093270385E09B
:1042B0005DCC80933E04A0923A04B0923B04C0923D
:1042C0003C04D0923D0482E051CC8091180490913E
:1042D00019048F5F9F4F0CF07FCF80912F05909135
:1042E0003005A0913105B091320520E030E849E079
:1042F00054E4BC01CD010E94C86B18160CF06CCFC1
:1043000080912F0590913005A0913105B091320533
:104310002AE037ED43EA5CE3BC01CD010E945B6B10
:10432000DC01CB0180932F0590933005A0933105DC
:10433000B09332058091AE049091AF04845F9140B8
:1043400008F04ACF80912F0590913005A09131055A
:10435000B09132052DEC3CEC4CEC5DE3BC01CD01A1
:104360000E945B6B2FCF220F331FB9CD8091780055
:104370009091790020912C0430912D04820F931F8D
:104380000196969587958ECE220F331FFACD07960C
:10439000FFCDD801C7010B96A11DB11DD7CC21506F
:1043A0003C4F4F4F5F4F49CF215F3F4F4F4F5F4FC4
:1043B00049CD215F3F4F4F4F5F4FFECC0196A11D6E
:1043C000B11D67CD0F9655CD2F5F3F4F0FCE019694
:1043D000F1CD07968BCD2F5F3F4FB6CD019698CD8F
:1043E000809178009091790020912C0430912D04D7
:1043F000820F931F2FEF37E0281B390B30931F04D8
:1044000020931E0486E0B2CBFF91EF91BF91AF9154
:104410009F918F917F916F915F914F913F912F91DC
:104420001F910F91FF90EF90DF90CF90BF90AF90D2
:104430000F900FBE0F901F90189590E2EAE2F3E004
:104440008FE49193815087FFFCCF08951F93CF9302
:10445000DF938091400420912903281710F42093C2
:10446000400490913F0490FF08C08091400488234D
:1044700009F41EC181508093400491FF08C08091CF
:104480004004821709F4E4C18F5F80934004892FB0
:10449000992780FF02C081FD08C10E941D229091D2
:1044A00040049A3008F0A2C081E180934104892F32
:1044B00099279F938F9383EE93E09F938F9381E04F
:1044C0008F930E9473140F900F900F900F900F9086
:1044D00080914004C82FDD27C730D10509F4BBC146
:1044E000C830D1050CF08CC0C330D10509F455C2D9
:1044F000C430D1050CF0DFC0C130D10509F4BBC216
:10450000C230D1050CF438C31092410487EA94E01C
:104510009F938F93C1E0CF930E94731484E18093A3
:1045200041040F900F900F908091290590912A05DA
:10453000A0912B05B0912C05B7FD58C63AE0B59572
:10454000A795979587953A95D1F7BF93AF939F938A
:104550008F9381EB94E09F938F93CF930E9473147A
:1045600088E2809341048DB79EB707960FB6F89402
:104570009EBF0FBE8DBF8091210590912205A09115
:104580002305B0912405B7FD2CC62AE0B595A79563
:10459000979587952A95D1F7BF93AF939F938F9364
:1045A00080EC94E09F938F93CF930E9473148CE3DD
:1045B000809341042DB73EB7295F3F4F0FB6F89463
:1045C0003EBF0FBE2DBF8091EF049091F0049F93EA
:1045D0008F938FEC94E09F938F93CF930E947314EB
:1045E0000F900F900F900F900F90D6C780E180939F
:1045F0004104892F99279F938F9388EE93E05DCF95
:10460000CB30D10509F45DC1CC30D1050CF00FC120
:10461000C930D10509F40BC52A970CF01CC31092C0
:10462000410486E796E09F938F9311E01F930E94C9
:10463000731484E1809341040F900F900F90809148
:10464000EB049091EC049F938F9385E896E09F9301
:104650008F931F930E94731488E2809341040F90FC
:104660000F900F900F900F908091EF049091F004B5
:104670009F938F9384E996E09F938F931F930E945B
:1046800073148CE3809341040F900F900F900F9060
:104690000F908091ED049091EE049F938F9383EAA5
:1046A00096E09F938F931F9399CF10924004F5CE7D
:1046B00020934004E2CEC530D10509F403C4269707
:1046C0000CF08CC3109241048091E208E82FFF2780
:1046D000EE0FFF1FE155F74F808191819F938F93DC
:1046E0008091E108E82FFF27EE0FFF1FE155F74FFC
:1046F000808191819F938F938EE195E09F938F931B
:1047000011E01F930E94731484E1809341048DB7DC
:104710009EB707960FB6F8949EBF0FBE8DBF8091CF
:10472000E408E82FFF27EE0FFF1FE155F74F8081C8
:1047300091819F938F938091E308E82FFF27EE0FDD
:10474000FF1FE155F74F8081918188589F4F9F93BC
:104750008F938EE295E09F938F931F930E94731423
:1047600088E2809341042DB73EB7295F3F4F0FB6D3
:10477000F8943EBF0FBE2DBF8091E608E82FFF27BB
:10478000EE0FFF1FE155F74F8081918182599F4FB6
:104790009F938F938091E508E82FFF27EE0FFF1F6F
:1047A000E155F74F8081918182599F4F9F938F935D
:1047B0008EE395E09F938F931F930E9473148CE375
:1047C000809341046DB77EB7695F7F4F0FB6F89451
:1047D0007EBF0FBE6DBF8091E808E82FFF27EE0F68
:1047E000FF1FE155F74F8081918182599F4F9F9321
:1047F0008F938091E708E82FFF27EE0FFF1FE15509
:10480000F74F8081918182599F4F9F938F938EE4C0
:1048100095E09F938F931F930E9473148DB79EB75B
:1048200007960FB6F8949EBF0FBE8DBFB5C6CD30AC
:10483000D10509F447C4CD30D1050CF452C22E97EE
:1048400009F4D9C481508093290310924004A4C66E
:10485000109240041CCE84E1809341048091270390
:10486000909128039F938F9388E496E09F938F9372
:1048700011E01F930E94731488E2809341040F900B
:104880000F900F900F900F908091DE0499279F93C7
:104890008F9387E596E09F938F931F930E947314E5
:1048A0008CE3809341040F900F900F900F900F9026
:1048B0008091AE08992701979F938F9386E696E0A3
:1048C000F0CE1092410484E197E09F938F9311E022
:1048D0001F930E94731484E1809341040F900F9002
:1048E0000F9080918407992787FD90959F938F93D0
:1048F00080918307992787FD90959F938F9384E2FA
:1049000097E09F938F931F930E94731488E2809384
:1049100041048DB79EB707960FB6F8949EBF0FBEA1
:104920008DBF80918507992787FD90959F938F93E1
:104930008091860799279F938F9384E397E09F93B5
:104940008F931F930E9473148CE3809341042DB7BF
:104950003EB7295F3F4F0FB6F8943EBF0FBE2DBF45
:1049600080918A0799279F938F9380918707992732
:1049700087FD90959F938F9384E497E09F938F9307
:104980001F930E9473146DB77EB7695F7F4F0FB698
:10499000F8947EBF0FBE6DBFFFC510924104809199
:1049A000B3089091B4089F938F938091B108909130
:1049B000B2089F938F938EED94E09F938F9311E0B5
:1049C0001F930E94731484E1809341046DB77EB7F6
:1049D000695F7F4F0FB6F8947EBF0FBE6DBF8091A9
:1049E000B7089091B8089F938F938091B5089091E4
:1049F000B6089F938F938EEE94E09F938F931F93AF
:104A00000E94731488E2809341048DB79EB7079685
:104A10000FB6F8949EBF0FBE8DBF8091BB089091DA
:104A2000BC089F938F938091B9089091BA089F9387
:104A30008F938EEF94E09F938F931F930E94731434
:104A40008CE3809341042DB73EB7295F3F4F0FB6EB
:104A5000F8943EBF0FBE2DBF8091BF089091C00853
:104A60009F938F938091BD089091BE089F938F93E1
:104A70008EE095E083CF8091E90880FD1CC084E141
:104A80008093410482E994E09F938F9311E01F93F8
:104A90000E94731488E2809341040F900F900F904E
:104AA00089E994E09F938F931F930E9473140F9052
:104AB0000F900F9071C5109241048091D004909195
:104AC000D104A091D204B091D304BC01CD0125E062
:104AD00030E040E050E00E94A96C3F932F9386E5C0
:104AE00094E09F938F9311E01F930E94731484E1CD
:104AF000809341040F900F900F900F900F90809132
:104B0000CC049091CD04A091CE04B091CF04BC010F
:104B1000CD0125E030E040E050E00E94A96C3F93D9
:104B20002F9385E694E09F938F931F930E947314B5
:104B300088E2809341040F900F900F900F900F9098
:104B400080911D0390911E039F938F9384E794E0BF
:104B50009F938F931F930E9473148CE3809341045F
:104B60000F900F900F900F900F9087B599279F93FC
:104B70008F9383E894E095CD209709F063CE10924F
:104B800041048DEE93E09F938F9311E01F930E9459
:104B9000731484E1809341040F900F900F9087E687
:104BA00090E09F938F938CE490E09F938F93DF939B
:104BB000CF93809102016AE00E94546C892F99275B
:104BC0009F938F93809102010E94546C99279F9329
:104BD0008F938DEF93E09F938F931F930E94731495
:104BE00088E2809341042DB73EB7235F3F4F0FB655
:104BF000F8943EBF0FBE2DBF84ED95E09F938F9339
:104C00000E94B20599279F938F9386E194E09F932A
:104C10008F931F930E9473148091AC039091AD0306
:104C20006DB77EB7695F7F4F0FB6F8947EBF0FBE3A
:104C30006DBF069708F488C490914604992309F43F
:104C40007DC48CE380934104892F99279F938F9390
:104C500081E394E026CD1092410482EE96E09F938A
:104C60008F9311E01F930E94731484E18093410499
:104C70000F900F900F908091920399279F938F939D
:104C80008AEE96E09F938F931F930E94731488E29D
:104C9000809341040F900F900F900F900F90809190
:104CA000F7039091F8039F938F9388EF96E09F937B
:104CB0008F931F930E9473148CE3809341040F9091
:104CC0000F900F900F900F9080910B0999279F9351
:104CD0008F9380910A0999279F938F9386E097E09D
:104CE0004DCE1092410484E597E09F938F9311E09D
:104CF0001F930E94731484E1809341040F900F90DE
:104D00000F908091890899279F938F9380918808AD
:104D100099279F938F938091870899279F938F93CB
:104D20008091860899279F938F9384E697E09F93BD
:104D30008F931F930E94731488E2809341048DB770
:104D40009EB70B960FB6F8949EBF0FBE8DBF809195
:104D50008D0899279F938F9380918C0899279F9313
:104D60008F9380918B0899279F938F9380918A08C6
:104D700099279F938F9389E797E09F938F931F9332
:104D80000E9473148CE3809341042DB73EB7255FD6
:104D90003F4F0FB6F8943EBF0FBE2DBF80919108D4
:104DA00099279F938F938091900899279F938F9332
:104DB00080918F0899279F938F9380918E089927D0
:104DC0009F938F938EE897E09F938F931F930E94FA
:104DD00073146DB77EB7655F7F4FD9CD10924104D4
:104DE0008EE096E09F938F9311E01F930E947314BF
:104DF00084E1809341040F900F900F9080913705CC
:104E0000909138059F938F9380911A0490911B0481
:104E10009F938F938BE196E09F938F931F930E94B4
:104E2000731488E2809341046DB77EB7695F7F4F4A
:104E30000FB6F8947EBF0FBE6DBF8091350590917F
:104E400036059F938F9380911C0490911D049F932E
:104E50008F938AE296E09F938F931F930E9473141F
:104E60008CE3809341048DB79EB707960FB6F894F4
:104E70009EBF0FBE8DBF80912F0590913005A091F0
:104E80003105B0913205BC01CD010E949E6BDC0161
:104E9000CB019F938F9380916209909163099F93B7
:104EA0008F9389E396E09F938F931F930E947314CF
:104EB0002DB73EB7295F3F4F0FB6F8943EBF0FBEE8
:104EC0002DBF6AC3109241048EE595E09F938F93A6
:104ED000C1E0CF930E947314809102010F900F9054
:104EE0000F908A3009F4A5C28B3009F4DEC18431F9
:104EF00009F4DBC18D3009F04FC384E18093410494
:104F000080911C0399279F938F9340914105509165
:104F10004205CA0157FD39C39595879595958795A3
:104F200095958795959587959F938F939A0157FDB2
:104F300029C33595279535952795359527958091E2
:104F4000220490912304821B930B9F938F9382EDF5
:104F500095E09F938F93CF930E94731488E2809380
:104F600041046DB77EB7675F7F4F0FB6F8947EBF81
:104F70000FBE6DBF80911B0399279F938F93409124
:104F80003F0550914005CA0157FD04C3959587958B
:104F90009595879595958795959587959F938F93EB
:104FA0009A0157FDF4C23595279535952795359586
:104FB00027958091200490912104821B930B9F934D
:104FC0008F9386EE95E09F938F93CF930E947314F7
:104FD0008CE3809341048DB79EB709960FB6F89481
:104FE0009EBF0FBE8DBF80911A0399279F938F9309
:104FF00020913D0530913E05C90137FDC1C295950F
:1050000087959F938F9380911E0490911F04281B76
:10501000390B3F932F938AEF95E09F938F93CF9314
:105020000E9473142DB73EB7275F3F4F45CF1092B4
:1050300041048091E5049091E6049F938F9382EB65
:1050400096E09F938F9311E01F930E94731484E165
:10505000809341040F900F900F900F900F908091CC
:10506000E3049091E4049F938F938EEB96E09F93DB
:105070008F931F930E94731488E2809341040F90D2
:105080000F900F900F900F908091E1049091E204A7
:105090009F938F938AEC96E09F938F931F930E9428
:1050A00073148CE3809341040F900F900F900F9036
:1050B0000F908091DF049091E0049F938F9386ED91
:1050C00096E0EFCA1092410483EA97E09F938F9392
:1050D000C1E0CF930E94731484E1809341040F9048
:1050E0000F900F908091A50899278D969F938F938D
:1050F0008091A40899278D969F938F938091A30800
:1051000099278D969F938F938091A20899278D96CA
:105110009F938F9382EB97E09F938F93CF930E94FF
:10512000731488E2809341048DB79EB70B960FB637
:10513000F8949EBF0FBE8DBF8091A90899278D96C8
:105140009F938F938091A80899278D969F938F9313
:105150008091A70899278D969F938F938091A60899
:1051600099278D969F938F9386EC97E09F938F93CB
:10517000CF930E9473148CE3809341042DB73EB704
:10518000255F3F4F0FB6F8943EBF0FBE2DBF8091F5
:10519000AA0899278D969F938F938AED97E09F9306
:1051A0008F93CF930E9473140F900F900F900F90D6
:1051B0000F908091AB08882309F02DC18091AC0835
:1051C000882309F01AC18091AD08882309F4E4C14D
:1051D00088E48093410480EF97E09F938F93CF936F
:1051E00064CC81509C4FAF4FBF4FCFC981509C4F73
:1051F000AF4FBF4FA3C91092410483EF97E09F9335
:105200008F9311E01F930E94731484E180934104F3
:105210000F900F900F908091D8039091D9039F9396
:105220008F9381E098E09F938F931F930E94731454
:1052300088E2809341040F900F900F900F900F9091
:105240008091D6039091D7039F938F938EE098E03F
:105250009F938F931F930E94731489E4809341045A
:105260000F900F900F900F900F908BE198E09F930D
:105270008F931F930E94731480913F040F900F909F
:105280000F9083FF89C11092D9031092D803AEE02A
:10529000B0E080E0082E0E94D16CAFE0B0E08091D9
:1052A000D803082E0E94D16C77C184E18093410419
:1052B0004091410550914205CA0157FD57C19C01DB
:1052C00035952795359527953595279535952795C6
:1052D000C90182959295907F9827807F9827BA017F
:1052E000681B790BCB0177FD3FC1959587959F93FF
:1052F0008F933F932F939A0157FD33C1359527958F
:105300003595279535952795809122049091230412
:10531000821B930B9F938F938FE995E09F938F93BD
:10532000CF930E94731488E2809341048DB79EB797
:1053300009960FB6F8949EBF0FBE8DBF40913F05F2
:1053400050914005CA0157FD0AC19C01359527952A
:10535000359527953595279535952795C9018295DA
:105360009295907F9827807F9827BA01681B790BC8
:10537000CB0177FDF2C0959587959F938F933F93CF
:105380002F939A0157FDE6C03595279535952795BA
:10539000359527958091200490912104821B930BD1
:1053A0009F938F9381EB95E09F938F93CF930E9470
:1053B00073148CE3809341048DB79EB709960FB6A2
:1053C000F8949EBF0FBE8DBF20913D0530913E05E4
:1053D000C90137FDCDC0959587959F938F93809197
:1053E0001E0490911F04281B390B3F932F9383ECCD
:1053F00095E09F938F93CF9359CD84E4809341049C
:105400008DEE97E09F938F93CF930E9473140F902C
:105410000F900F90D8CE80E4809341048AEE97E0FD
:105420009F938F93CF930E9473140F900F900F90C0
:10543000C5CE84E1809341044091410550914205DD
:105440009A0157FD9AC0359527953595279535953D
:105450002795C901880F991F880F991F880F991FD9
:10546000481B590B5F934F933F932F9380912204D6
:1054700090912304821B930B9F938F938CE695E06E
:105480009F938F93CF930E94731488E2809341047B
:105490002DB73EB7275F3F4F0FB6F8943EBF0FBE04
:1054A0002DBF40913F05509140059A0157FD62C0C4
:1054B000359527953595279535952795C901880FF9
:1054C000991F880F991F880F991F481B590B5F93CD
:1054D0004F933F932F938091200490912104821B3E
:1054E000930B9F938F938EE795E09F938F93CF932A
:1054F0000E9473148CE3809341046DB77EB7675F9D
:105500007F4F0FB6F8947EBF0FBE6DBF80913D05F3
:1055100090913E059F938F9380913D0590913E051C
:1055200020911E0430911F04821B930B9F938F9335
:1055300080E995E09F938F93CF936EC98CE380931E
:10554000410486E494E0AECA8CE38093410484E293
:1055500094E0A8CA295F3F4F17CF01960CCF0F9652
:10556000F4CE295F3F4FCACE0196BFCE0F96A7CE8D
:10557000019631CF295F3F4F9BCF295F3F4F63CFCC
:1055800001963DCD295F3F4FD4CC0F96C5CC295F06
:105590003F4F09CD0F96FACC10923F04DF91CF9187
:1055A0001F9108951092B9008AE28093B80008957F
:1055B00085EA8093BC00089584E98093BC00089537
:1055C0001092B9008093BB0085E88093BC000895D9
:1055D0000E94DC2A109249048091BB00109248047A
:1055E00080E88093BC001092BD001092BA00109227
:1055F000BB001092B9001092B8000E94D22A0E94FB
:10560000D82A80E00E94E02A08958093BB0085E8B4
:105610008093BC00089585EC8093BC00089585E8D4
:105620008093BC0008951F920F920FB60F92112421
:105630002F933F934F935F936F937F938F939F939A
:10564000AF93BF93EF93FF9380914904282F3327A3
:10565000442755278F5F80934904F901273131058D
:10566000C8F4E05BFF4FEE0FFF1F0590F491E02DB3
:10567000099480914704E82FFF27EA58F74F90914B
:10568000BB0090838F5F8C3008F49DC0109247045C
:105690000E94DC2A10924904E0C080E80E94E02ABF
:1056A000DCC088E90E94E02AD8C00E94DC2A8AE097
:1056B00090E09093AD038093AC030E94D82ACDC0B4
:1056C00084E10E94E02AC9C082E10E94E02AC5C0AC
:1056D00080911C030E94E02AC0C080E10E94E02A61
:1056E000BCC080911B030E94E02AB7C080911A03BE
:1056F0000E94E02AB2C080914804E82FFF27EA56B2
:10570000F64F8F5F8093480480810E94E02AA5C0F5
:1057100090914804292FE92FFF27EE0FFF1FEE0F6E
:10572000FF1FED52FA4F858518160CF054C09C30BF
:1057300009F467C0990F892F8E5A0E94E02A8DC004
:1057400080914704E82FFF27EE56F74F8091BB006A
:1057500080830E940F2B81C08091B900803409F4AE
:105760006EC080914704E82FFF27EE55F74F108257
:105770008F5F8C3068F1109247040E94DC2A1092EF
:10578000490480914A048093460410924A0465C0FB
:105790008091B900803309F440C00E94DC2A8AE07D
:1057A00090E09093AD038093AC03109249040E9463
:1057B000D82A53C00E94DC2A8AE090E09093AD037F
:1057C0008093AC0367CF809347040E94DC2A62CFAA
:1057D00080934704D2CF9C3008F0A9CF922F9F5FCF
:1057E000E92FFF27EE0FFF1FEE0FFF1FED52FA4FBD
:1057F000858518161CF0292F9C3080F3909348045F
:1058000096CF1092480483E0809349048091470426
:10581000880F8D5A0E94E02A20C080914A04882374
:10582000C9F49091480490934A04E92FFF27EB575D
:10583000F74F80818F5F09F48FEF8083AECF809127
:105840004704E82FFF27EE55F74F8C5F80830E94B7
:105850000B2B97CF90914804E8CF8091BC008068D3
:105860008093BC00FF91EF91BF91AF919F918F9179
:105870007F916F915F914F913F912F910F900FBE4C
:105880000F901F90189583EC8093810080916F009A
:10589000806280936F0010923E0510923D05109239
:1058A000400510923F05109242051092410508955F
:1058B0001F920F920FB60F921124EF92FF920F9347
:1058C0001F932F933F934F935F936F937F938F9388
:1058D0009F93AF93BF93CF93DF93EF93FF93809109
:1058E000390982FD2CC0209186003091870080917B
:1058F0004C0490914D04281B390B809186009091A7
:10590000870090934D0480934C04C9018D549440BA
:10591000835F9A4108F0B5C080914E048093AE0831
:1059200080914E0490914F04049714F010928403D8
:10593000C1E0D0E0D0934F04C0934E0415C2409113
:105940008600509187008091500490915104481B2B
:10595000590B809186009091870090935104809319
:105960005004CA018D549440835F9A4138F5809168
:10597000AA0480934B0480914B04843008F00EC13C
:105980008091AB04853608F47BC18AE08093AB0438
:10599000809102018A3009F476C1843109F473C11F
:1059A000289881E08093AA048091D404882309F088
:1059B000DBC180914B048093AE08D6C10091AA044C
:1059C0000A3008F0E4C0CA018B5F9040845B9140CC
:1059D00008F05BC1425D5140E02FFF27EE0FFF1F33
:1059E000EE5AFB4F80819181FA01E81BF90BCF0140
:1059F00005960B9708F45CC1E02FFF27EE0FFF1F01
:105A0000EE5AFB4F808191819C01220F331F280F9A
:105A1000391F240F351F37FDA4C1E901D595C7955E
:105A2000D595C795CA0101968C179D070CF071C1D9
:105A300021978091DE048E3B08F462C1E02FFF279E
:105A4000EE0FFF1FDF01AE5ABB4F8D919C919E015F
:105A5000281B390BC90163E070E00E94746CCB0114
:105A6000880F991F860F971FE859FB4F91838083FA
:105A7000E02FFF27EE0FFF1FEE5AFB4FD183C083AD
:105A80000BC1C0914E04D0914F04CA30D1050CF027
:105A90006BC1C9018B5F9040845B914008F060C08E
:105AA000225D3140FE01EC0FFD1FE155F74F808173
:105AB0009181D901A81BB90BCD01B7FD0EC1069785
:105AC00054F48091DE04883C08F046C18091DE04E5
:105AD000865F8093DE04FE01EC0FFD1FE155F74F5A
:105AE00080819181AC01440F551F480F591F420F0F
:105AF000531F57FD33C17A01F594E794F594E79469
:105B0000C90101968E159F050CF013C10894E10898
:105B1000F1088091DE04833C08F403C18E010C0F70
:105B20001D1FF801E155F74F80819181F701E81BB6
:105B3000F90BCF0163E070E00E94746CCB01880F19
:105B4000991F860F971F0B53174FD80111969C93DF
:105B50008E93FE01EC0FFD1FE155F74FF182E082BD
:105B6000FE013196F0934F04E0934E04E530F105C9
:105B700009F4B9C05D98E630F10509F4BFC05C983E
:105B8000379709F4B9C05B98EFC05C9A5B98043111
:105B900008F054C00F5F0093AA04E6C09091AE08CD
:105BA00080914B04981709F0EBCE4091AB044B3039
:105BB00008F49BC0109284031092AA043AC000918A
:105BC000AA04E02FFF27EE0FFF1F9F0122583B4F33
:105BD000DF01A155B74F8D919C91D9018D939C9375
:105BE000DF01AB53B74F8D919C91EC56FB4F9183E6
:105BF0008083E02FFF27EE0FFF1F9F012155374FB6
:105C0000DF01AE5ABB4F8D919C91D90111969C93A7
:105C10008E93DF01A859BB4F8D919C91EB53F74FA9
:105C200091838083E02FEF5FEB3008F05EC0E0935C
:105C3000AA044F3120F60091AA04DBCF043109F009
:105C400093C0809102018A3009F47DC0843109F447
:105C50007AC028988EE18093AA042AE0C5ECD8E0A7
:105C6000AEE7B4E0EFEAF8E08D919D9191838083F7
:105C70003296198218822296215027FFF5CF74C0E0
:105C80001092AB0485CE289A8CCE809102018A3086
:105C900011F1843101F12898053019F15D98063031
:105CA00009F473CF5C98073009F070CF5B9A72CF1C
:105CB0008091AB048A3108F448C08091DE04865F8D
:105CC0008093DE048091DE04893C08F495CE88EC54
:105CD0008093DE0491CE289ADFCF909581959F4FD7
:105CE000EECE5D9ADFCF5D9A46CF4F3F09F459CE95
:105CF0004F5F4093AB0455CE5B9A36C05C9A40CF61
:105D0000E02FFF27EE0FFF1FE859FB4F1182108293
:105D1000AFCE41505040C417D5070CF08ACE219623
:105D200088CEFE01EC0FFD1FEB53F74F118210825E
:105D300010CF21503040E216F3060CF0EACE089462
:105D4000E11CF11CE6CE289A85CF8B3008F4BACF3F
:105D50008091DE048E5FB4CF88ECBBCE4D5F5F4F89
:105D6000CACE2D5F3F4F59CEFF91EF91DF91CF917A
:105D7000BF91AF919F918F917F916F915F914F9163
:105D80003F912F911F910F91FF90EF900F900FBEB9
:105D90000F901F90189581E08093E30882E0809334
:105DA000E20883E08093E10884E08093E40885E0E2
:105DB0008093E50886E08093E60887E08093E70813
:105DC00088E08093E80808951F938AE68093E908A5
:105DD00051E0509339094EE14093EA088BEF8093EC
:105DE000EC088AE08093ED084093EB084093EF08BD
:105DF00085E08093F00880E48093F1081092F20827
:105E000084E18093EE088EE08093F308E0E1E09374
:105E1000F4081CE01093F508F8E0F093F60886EE1D
:105E20008093F7084093F80880E88093F90830E5FC
:105E30003093FA0896E99093FB0883E08093FC087E
:105E40003093FD089093FE0881E28093FF0883E27F
:105E500080930009409301091092020960E2609367
:105E60000309109204091092050910920609109274
:105E7000070910921C0910921D0910921E09109218
:105E80001F0924E62093080998E29093090950938A
:105E9000380910920A098AEF80930B0976E0709313
:105EA000100920930C0990930D0910920E0980930C
:105EB0000F0982E3809311099AE590931209809368
:105EC00013091092370990931409309315095093D0
:105ED000160985E58093170980931809E09319093D
:105EE00060931A0920931B098FE58093200983EFA3
:105EF000809322098AEA80932409809325098FE000
:105F000080932109809323098CEF809326092093A5
:105F10002709909328099093290990932A098BE4E3
:105F200080932B0980932C0980932D0910922E09C0
:105F300070932F09F09330099093310940933209FF
:105F4000209333092093340984E080933509AEEA25
:105F5000B3E0EAE3F9E00D9001921A95E1F71F91A1
:105F600008958AE68093E90871E0709339095EE14B
:105F70005093EA088BEF8093EC089AE09093ED0839
:105F80005093EB085093EF0885E08093F00880E48D
:105F90008093F1081092F2088FE08093EE089093BE
:105FA000F30880E18093F40866E06093F508E8E088
:105FB000E093F60886EE8093F7085093F80880E89F
:105FC0008093F9082AE52093FA0898E79093FB0854
:105FD00083E08093FC082093FD089093FE0881E203
:105FE0008093FF0883E28093000950930109109287
:105FF000020940E240930309109204091092050936
:10600000109206091092070910921C0910921D099E
:1060100010921E0910921F0934E63093080998E285
:10602000909309097093380910920A098AEF8093B6
:106030000B096093100930930C0990930D0910928D
:106040000E0980930F0982E38093110920931209AE
:1060500080931309109237092093140980E58093E7
:1060600015098CE38093160985E5809317098093C1
:1060700018094093190940931A099BE490931B094E
:106080008FE58093200983EF809322098AEA809329
:1060900024098093250984E18093210980932309B1
:1060A0008CEF8093260930932709209328092093A9
:1060B000290920932A0990932B0990932C099093F6
:1060C0002D0910922E0960932F09E0933009209337
:1060D000310950933209309333093093340984E005
:1060E000809335098CE0A5EBB3E0EAE3F9E00D908D
:1060F00001928A95E1F708958AE68093E90871E0B4
:10610000709339094EE14093EA088BEF8093EC08D5
:106110008AE08093ED084093EB084093EF0885E018
:106120008093F00880E48093F1081092F2088FE0E9
:106130008093EE0868E06093F30820E12093F40870
:1061400056E05093F5086093F60886EE8093F708C2
:106150004093F80880E88093F90834E63093FA0811
:1061600098E79093FB0883E08093FC083093FD0848
:106170009093FE0881E28093FF0883E280930009F8
:1061800084E180930109109202092093030910927F
:10619000040910920509109206091092070910923D
:1061A0001C0910921D0910921E0910921F093093AC
:1061B000080998E2909309097093380910920A0926
:1061C0008AEF80930B095093100930930C09909338
:1061D0000D0910920E0980930F0992E39093110913
:1061E0002AE52093120990931309109237092093FE
:1061F000140980E58093150986E48093160985E5E6
:10620000809317098093180980E28093190980937D
:106210001A0990931B098FE58093200983EF8093DF
:1062200022098AEA80932409809325094093210951
:10623000409323098CEF80932609309327092093FC
:1062400028092093290920932A098BE480932B099C
:1062500080932C0980932D0910922E0950932F09B9
:106260006093300920933109409332093093330908
:106270003093340984E0809335098CE0ADEBB3E0D2
:10628000EAE3F9E00D9001928A95E1F70895681725
:10629000790744F4680F791F77FD09C0CB01959504
:1062A00087950895681B790B861B970B08956F5F80
:1062B0007F4FCB01959587950895681779073CF432
:1062C000680F791F77FD04C0CB01959587950895D8
:1062D0006F5F7F4FCB0195958795F9CFFC01AB019F
:1062E0008091C004873218F488E28093C0044E176E
:1062F0005F0744F4BA016E0F7F1F77FD11C07595DB
:10630000679512C064E10E94546C282F3327CA019C
:106310008E1B9F0BB9010E94746C6E0F7F1F04C00F
:106320006F5F7F4F75956795CB0108959C018091B4
:10633000C004873218F488E28093C00462177307A0
:1063400044F4620F731F77FD16C0CB0195958795B6
:106350000895621B730B77FD06C0CB019595879559
:10636000820F931F08956F5F7F4FCB01959587959F
:10637000820F931F08956F5F7F4FCB01959587958F
:106380000895EF92FF920F931F93CF93C82F8B0125
:106390008091D4048823A9F4C150CF3F91F07B01B0
:1063A000E60EF71E1093FC030093FB038091FB03A2
:1063B0009091FC03892BD1F7C7010E940718C150A7
:1063C00088F7CF911F910F91FF90EF9008952F9232
:1063D0003F924F925F926F927F928F929F92AF9275
:1063E000BF92CF92DF92EF92FF920F931F93CF93C2
:1063F000DF93CDB7DEB7ED970FB6F894DEBF0FBED3
:10640000CDBF20913D0530913E0580911E049091B5
:106410001F04281B390B3A8729873093A50920933D
:10642000A409209128043091290437FDD4C735955B
:10643000279535952795359527953AA729A73C8720
:106440002B877901209126043091270437FDC0C79E
:106450003595279535952795359527953CA72BA7F5
:106460003E872D87F0926509E092640930935B09BD
:1064700020935A098091930990919409AA2797FD36
:10648000A095BA2F7C018D01EE0CFF1C001F111F7F
:10649000E80EF91E0A1F1B1F80911A0490911B041D
:1064A0009C01442737FD4095542FDA01C901880F1C
:1064B000991FAA1FBB1F880F991FAA1FBB1F820FFE
:1064C000931FA41FB51F820F931FA41FB51FE80EB3
:1064D000F91E0A1F1B1F17FD9CC715950795F794FA
:1064E000E79415950795F794E794F0929409E09254
:1064F00093098091AF099091B009AA2797FDA095C3
:10650000BA2F7C018D01EE0CFF1C001F111FE80E3D
:10651000F91E0A1F1B1F80911C0490911D049C01F1
:10652000442737FD4095542FDA01C901880F991F80
:10653000AA1FBB1F880F991FAA1FBB1F820F931F83
:10654000A41FB51F820F931FA41FB51FE80EF91ECD
:106550000A1F1B1F17FD54C715950795F794E7945D
:1065600015950795F794E794F092B009E092AF097A
:106570008091620990916309AA2797FDA095BA2F8F
:106580009C01AD01220F331F441F551F280F391FD7
:106590004A1F5B1F8091180490911904AA2797FD48
:1065A000A095BA2F280F391F4A1F5B1F57FD16C72A
:1065B000559547953795279555954795379527953F
:1065C000309363092093620920911A0430911B04CF
:1065D000C901880F991F880F991F820F931F820F7F
:1065E000931FAA2797FDA095BA2F209119053091E6
:1065F0001A0540911B0550911C05820F931FA41F83
:10660000B51F8093190590931A05A0931B05B093AD
:106610001C0520911C0430911D04C901880F991F8D
:10662000880F991F820F931F820F931FAA2797FD30
:10663000A095BA2F209115053091160540911705A8
:1066400050911805820F931FA41FB51F8093150545
:1066500090931605A0931705B093180580916D09C6
:1066600090916E0920911A0430911B04820F931FA0
:1066700090936E0980936D098091A7099091A80964
:1066800020911C0430911D04820F931F9093A80940
:106690008093A709809133059091340501969093DA
:1066A0003405809333058091110590911205A091D6
:1066B0001305B0911405BC01CD010E94BB6B5B01B9
:1066C0006C018091690890916A08AA2797FDA095AE
:1066D000BA2FBC01CD010E94BB6B7B018C01809164
:1066E0002F0590913005A0913105B09132059C01A4
:1066F000AD01C801B7010E945B6BDC01CB019C01BD
:10670000AD01C601B5010E945C6BDC01CB01BC018F
:10671000CD010E949E6BDC01CB018093110590930B
:106720001205A0931305B09314058FEC80937A00A3
:106730001092190320900105309002054090030546
:106740005090040539E423163BE6330631E0430656
:1067500030E053060CF414C188E49BE6A1E0B0E0FD
:106760008D839E83AF83B8876090090570900A057A
:1067700080900B0590900C0539E463163BE6730698
:1067800031E0830630E093060CF4DCC488E49BE639
:10679000A1E0B0E089839A83AB83BC8349855A85A5
:1067A000CA01AA2797FDA095BA2F2091F90430912C
:1067B000FA044091FB045091FC04280F391F4A1F32
:1067C0005B1F2DA33EA34FA358A7A090AB09B09089
:1067D000AC09C090AD09D090AE09A80EB91ECA1E72
:1067E000DB1E860175013091C7043BA3332309F0FA
:1067F000DAC08091C604882309F0C2C44091E90838
:106800004CA346FF13C6EBA5FCA5CF01AA2797FD15
:10681000A095BA2FBC01CD0129813A814B815C81C1
:106820000E94356C9B01AC0197FD2CC7BBE05595D0
:10683000479537952795BA95D1F780918E03E82E25
:10684000FF2400271127C801B7010E94356C97FD6E
:1068500014C7ACE09595879577956795AA95D1F77C
:106860006F87788B898B9A8B60934D0570934E055B
:1068700080934F059093500529A53AA5C901AA27F1
:1068800097FDA095BA2FBC01CD012D813E814F818E
:1068900058850E94356C9B01AC0197FD01C7FBE058
:1068A0005595479537952795FA95D1F7C801B701C2
:1068B0000E94356C97FDEFC6DC01CB01ECE0B5958D
:1068C000A79597958795EA95D1F780935105909371
:1068D0005205A0935305B093540520914D05309176
:1068E0004E053093DC082093DB0820915105309150
:1068F00052053093E0082093DF082F8538894989B5
:106900005A89821B930BA40BB50B8AAF9BAFACAF1C
:10691000BDAF8093510590935205A0935305B0935A
:106920005405A80EB91ECA1EDB1E860175013091E2
:106930008D033DA7332309F0A3C58EA79FA7A8AB5E
:10694000B9ABB7FD61C62EA53FA548A959A9559574
:106950004795379527958DA19EA1AFA1B8A5821B1C
:10696000930BA40BB50B8DA39EA3AFA3B8A78093E5
:10697000F9049093FA04A093FB04B093FC048CC533
:1069800098EB291694E939069EEF49069FEF5906C0
:106990000CF0F1C328EB34E94EEF5FEF2D833E831B
:1069A0004F835887E1CE2DA13EA14FA158A520933A
:1069B000F9043093FA044093FB045093FC043091A3
:1069C000E9083CA31092E0081092DF081092DC085E
:1069D0001092DB081092490510924A0510924B055F
:1069E00010924C05109245051092460510924705ED
:1069F0001092480530918D033DA7809149059091F3
:106A00004A05A0914B05B0914C05BC01CD0124E68F
:106A100030E040E050E00E94A96CDA01C9014091E9
:106A2000450550914605481B590B58A34F8F80913F
:106A3000450590914605A0914705B0914805BC01D8
:106A4000CD0124E630E040E050E00E94A96CDA017C
:106A5000C9012091490530914A05821B930B9AA3E5
:106A600089A38091860390918703A0918803B091B8
:106A70008903BC01CD0128E631E040E050E00E94EE
:106A8000356CE616F7060807190744F05701680148
:106A9000A61AB70AC80AD90A8601750117FDA3C448
:106AA000A092AB09B092AC09C092AD09D092AE09E8
:106AB0002BA53CA58F8D98A1280F391F79010027A0
:106AC000F7FC0095102F8091FD049091FE04A09199
:106AD000FF04B0910005E80EF91E0A1F1B1F5701A5
:106AE00068018091CA049091CB04281B390BC9011D
:106AF000AA2797FDA095BA2F280E391E4A1E5B1EA5
:106B00002091A2033091A3034091A4035091A503C7
:106B1000221533054405550574F4A8EAEA2EA1E6CA
:106B2000FA2E012D112DE21AF30A040B150B170191
:106B300028015701680188279927DC01821B930BE4
:106B4000A40BB50B281639064A065B060CF0E9C201
:106B5000F8E52F2EFEE93F2EFFEF4F2EFFEF5F2EC1
:106B6000220E331E441E551E20920105309202054E
:106B70004092030550920405820171012092FD04A8
:106B80003092FE044092FF045092000529A53AA5D8
:106B9000A9A1BAA12A0F3B1FA901662757FD60953D
:106BA000762F8091050590910605A0910705B0917B
:106BB0000805480F591F6A1F7B1F5A016B018091FE
:106BC000C8049091C904281B390BC901AA2797FD55
:106BD000A095BA2F680E791E8A1E9B1E8091A6036F
:106BE0009091A703A091A803B091A9038EAB9FAB8E
:106BF000A8AFB9AF86159705A805B90564F448EAAA
:106C000051E660E070E0481B590B6A0B7B0B3A01C0
:106C10004B015A016B018EA99FA9A8ADB9ADB095E2
:106C2000A095909581959F4FAF4FBF4F68167906FD
:106C30008A069B060CF064C2E8E56E2EEEE97E2E15
:106C4000EFEF8E2EEFEF9E2E2EA93FA948AD59AD46
:106C5000620E731E841E951E6092090570920A05CD
:106C600080920B0590920C05B401A301609205057A
:106C70007092060580920705909208058DA19EA14D
:106C8000AFA1B8A580930D0590930E05A0930F05B5
:106C9000B09310056092290570922A0580922B0509
:106CA00090922C05209221053092220540922305D6
:106CB000509224054093250550932605609327059F
:106CC00070932805E0921D05F0921E0500931F05A4
:106CD00010932005809125039091260397FDA4C36E
:106CE0007C01F594E794F594E794F594E794FAA67B
:106CF000E9A6809123039091240397FD93C38C010F
:106D00001595079515950795159507951CA70BA73C
:106D100080912204909123040F9734F458E1E52EDA
:106D20005CEFF52EFAA6E9A6809122049091230447
:106D3000079734F440E3E42E48EFF42EFAA6E9A6D0
:106D4000209102012A3009F46BC2809122049091B3
:106D50002304815D97400CF007C28091220490913A
:106D60002304805E974034F080EDE82E87E0F82E13
:106D7000FAA6E9A680912004909121040F9724F4AB
:106D800008E11CEF1CA70BA780912004909121041F
:106D9000079724F400E318EF1CA70BA72A3009F487
:106DA00055C28091200490912104815D974024F088
:106DB00008EE13E01CA70BA78091200490912104FA
:106DC000805E974024F000ED17E01CA70BA7A09170
:106DD0009903AA2309F497C06091250370912603B3
:106DE0008091550590915605681B790B20912503DC
:106DF00030912603280F391F37FD3FC3359527955E
:106E00003093560520935505613871050CF43AC24C
:106E100060E870E070935C0560935B058A2F9927AA
:106E2000869FF001879FF00D969FF00D1124CF01F2
:106E3000F7FD21C37C01F594E794F594E794F5946C
:106E4000E794F594E79429A53AA5E20EF31EFAA675
:106E5000E9A6409123035091240380915705909116
:106E60005805481B590B2091230330912403280F08
:106E7000391F37FDFDC2359527953093580520936E
:106E80005705413851050CF4F5C140E850E05093E6
:106E90005A05409359058A2F9927849FD001859FD1
:106EA000B00D949FB00D1124AD019D01B7FDDDC261
:106EB00089011595079515950795159507951595CC
:106EC0000795EBA5FCA50E0F1F1F1CA70BA7869F00
:106ED0009001879F300D969F300D1124C90120919C
:106EE000250330912603820F931F909326038093EE
:106EF00025038091230390912403480F591F509339
:106F00002403409323034D855E85141615060CF06B
:106F1000C1C18091DB089091DC0897FDA2C2AA272D
:106F200097FDA095BA2F6DA5262F33274427552707
:106F3000BC01CD010E94356C97FD8EC2B6E09595DF
:106F4000879577956795BA95D1F7AF8DB8A1A60FBC
:106F5000B71FB0935609A09355094B855C8514164D
:106F600015060CF0C1C18091DF089091E00897FDF3
:106F70006FC2AA2797FDA095BA2F6DA5262F33279C
:106F800044275527BC01CD010E94356C97FD5BC29B
:106F9000F6E09595879577956795FA95D1F7A9A12C
:106FA000BAA1A60FB71FB0934B09A0934A093CA101
:106FB00037FDC1C11093490900934809F09258095F
:106FC000E09257098091E508E82FFF27EE0FFF1F99
:106FD000E155F74F8081918182599F4FA091E5043F
:106FE000B091E604A817B9070CF0EEC0CD010196E8
:106FF0009093E6048093E504DC018091E608E82F95
:10700000FF27EE0FFF1FE155F74F808191818259D5
:107010009F4F6091E3047091E404681779070CF0C6
:10702000C4C0CB0101969093E4048093E304BC01B7
:107030008091E708E82FFF27EE0FFF1FE155F74F7C
:107040008081918182599F4F4091E1045091E204E7
:10705000481759070CF0D5C0CA0101969093E20475
:107060008093E104AC018091E808E82FFF27EE0F40
:10707000FF1FE155F74F8081918182599F4F2091E9
:10708000DF043091E004281739070CF0ABC0C901C8
:1070900001969093E0048093DF049C01B7FD93C1B7
:1070A000AF3FB10539F034F08FEF90E09093E604F4
:1070B0008093E50477FD76C16F3F710539F034F0B8
:1070C0008FEF90E09093E4048093E30457FD70C148
:1070D0004F3F510539F034F08FEF90E09093E20488
:1070E0008093E10437FD6AC12F3F310509F00CF4AC
:1070F000EEC28FEF90E09093E0048093DF04E7C24C
:107100006092090570920A0580920B0590920C0519
:10711000A0920505B0920605C0920705D092080519
:10712000ADCD2092010530920205409203055092A8
:107130000405A092FD04B092FE04C092FF04D09218
:10714000000524CD98EB691694E979069EEF89062F
:107150009FEF99062CF528EB34E94EEF5FEF29837A
:107160003A834B835C831ACB98EEE92E93E0F92E99
:10717000FAA6E9A6F2CD2D823E824F825886F4CA45
:107180008DA19EA1AFA1B8A58093F9049093FA04B4
:10719000A093FB04B093FC049091E9089CA312CC4B
:1071A00069827A828B829C82F9CA8081918182591C
:1071B0009F4F861797070CF03BCF6115710509F4B7
:1071C00037CFCB0101972FCF8081918182599F4F7B
:1071D0008A179B070CF011CF109709F40ECFCD0141
:1071E000019706CF8081918182599F4F8217930723
:1071F0000CF054CF2115310509F450CFC901019786
:1072000048CF8081918182599F4F841795070CF058
:107210002ACF4115510509F426CFCA0101971ECF87
:107220008091220490912304835F934034F038EEE0
:10723000E32E33E0F32EFAA6E9A680912204909182
:1072400023048A5F93400CF495CD8ECD8091200469
:1072500090912104835F934024F008EE13E01CA773
:107260000BA780912004909121048A5F93400CF435
:10727000AECDA9CD3FEF403853070CF008CE40E823
:107280005FEF05CE8FEF603878070CF0C3CD60E874
:107290007FEFC0CD8091DB089091DC0897FD9BC10A
:1072A000AA2797FDA095BA2FEDA52E2F33274427A7
:1072B0005527BC01CD010E94356C97FDADC1A6E0FC
:1072C0009595879577956795AA95D1F72F8D38A1D4
:1072D000261B370B30935609209355094B855C8547
:1072E000141615060CF43FCE8091DF089091E0084B
:1072F00097FD6DC1AA2797FDA095BA2FEDA52E2F5A
:10730000332744275527BC01CD010E94356C97FDDA
:1073100088C1E6E09595879577956795EA95D1F7C9
:1073200029A13AA1261B370B30934B0920934A0918
:107330003CA137FF3FCE4BA1442309F03BCE8091C7
:10734000C604882309F036CE8B859C85A1E0813068
:107350009A070CF044C12B853C854FEF2030340751
:107360000CF0A3C189A59AA5280F391F3C872B874C
:1073700020503F4F3093580920935709AD85BE8563
:10738000E1E0A130BE070CF465C12BA53CA5A20F1E
:10739000B31FBE87AD87A050B140B0934909A093F9
:1073A000480910CE1092E4041092E30457FF90CEE7
:1073B0001092E2041092E10437FF96CE1092E0049E
:1073C0001092DF0484C11092E6041092E50472CE9C
:1073D000295F3F4F3DC8295F3F4F29C82D5F3F4F71
:1073E0004F4F5F4FE5C8E60EF71E081F191FE092CA
:1073F000AB09F092AC090093AD091093AE0958CBDC
:1074000023E030E040E050E0E20EF31E041F151FC1
:10741000A3C883E090E0A0E0B0E0E80EF91E0A1FE8
:107420001B1F5BC807966BCC07965ACC2DA13EA1BB
:107430004FA158A52093F9043093FA044093FB041C
:107440005093FC04BFCA615C7F4F8F4F9F4FA0CD0C
:10745000909581959F4F8DCD615C7F4F8F4F9F4F52
:107460006DCD909581959F4F5ACD215F3F4F20CD97
:107470002F5F3F4F00CD0F96DDCC2F5F3F4FBECC2F
:107480002DA13EA14FA158A52093F9043093FA04F1
:107490004093FB045093FC0489859A85AA2797FDA5
:1074A000A095BA2F2AAD3BAD4CAD5DAD820F931FB9
:1074B000A41FB51F8B8B9C8BAD8BBE8BBC01CD01EC
:1074C00029813A814B815C810E94356C9B01AC0122
:1074D00097FDBBC06BE055954795379527956A9505
:1074E000D1F760918F03862F9927AA27BB278F8B0F
:1074F000988FA98FBA8FBC01CD010E94356C97FD82
:107500009FC02CE095958795779567952A95D1F73B
:107510006B8F7C8F8D8F9E8F609345057093460592
:1075200080934705909348056B897C898D899E8956
:107530002D813E814F8158850E94356C9B01AC01A5
:1075400097FD79C08BE055954795379527958A9596
:10755000D1F76F89788D898D9A8D0E94356C97FD52
:1075600065C0BCE09595879577956795BA95D1F7F5
:107570006AAB7BAB8CAB9DAB6093490570934A05BE
:1075800080934B0590934C0529853A8537FD7FC044
:10759000213431050CF431CA6B8D7C8D8D8D9E8D1F
:1075A00097FD2AC0613871058105910564F46AA9C7
:1075B0007BA98CA99DA997FD82C0613871058105C1
:1075C00091050CF41ACA81E08093E90416CA9095DB
:1075D00081959F4F8FCE909581959F4F61CEE9A564
:1075E000FAA58E0F9F1F9C878B87805091409093A8
:1075F000580980935709C2CE9095809570956195F2
:107600007F4F8F4F9F4FCECF0196A11DB11D8EA7EB
:107610009FA7A8ABB9AB97C9615C7F4F8F4F9F4FB6
:107620004ECE615C7F4F8F4F9F4F73CE6150704F36
:107630008F4F9F4F96CF2150384F4F4F5F4F82CF84
:107640006150704F8F4F9F4F5CCF2150384F4F4F3D
:107650005F4F40CF4D855E856FEF4030560754F544
:107660008BA59CA5480F591F5E874D8740505F4FE3
:107670005093490940934809A5CC6150704F8F4FF2
:107680009F4FE7C82150384F4F4F5F4FCFC83095BD
:1076900021953F4F7DCF6150704F8F4F9F4F0CC949
:1076A0002150384F4F4F5F4FFAC8F0925809E0927F
:1076B000570964CE109349090093480983CC9095EB
:1076C0008095709561957F4F8F4F9F4F76CFED9648
:1076D0000FB6F894DEBF0FBECDBFDF91CF911F91E3
:1076E0000F91FF90EF90DF90CF90BF90AF909F9061
:1076F0008F907F906F905F904F903F902F90089564
:10770000809102018D3009F455C110927A00809168
:1077100022049091230490935809809357098091F3
:107720002004909121049093490980934809809105
:107730001E0490911F049093A5098093A409809141
:107740001A0490911B049C01442737FD4095542F47
:10775000DA01C901880F991FAA1FBB1F880F991F43
:10776000AA1FBB1F820F931FA41FB51F820F931F59
:10777000A41FB51F909394098093930980911C04D2
:1077800090911D049C01442737FD4095542FDA0148
:10779000C901880F991FAA1FBB1F880F991FAA1F15
:1077A000BB1F820F931FA41FB51F820F931FA41F1F
:1077B000B51F9093B0098093AF0980911804909100
:1077C000190490936309809362098FEC80937A0087
:1077D0008091E508E82FFF27EE0FFF1FE155F74FD7
:1077E0008081918182599F4FA091E504B091E60478
:1077F000A817B9070CF085C0CD0101969093E60457
:107800008093E504DC018091E608E82FFF27EE0F66
:10781000FF1FE155F74F8081918182599F4F609101
:10782000E3047091E404681779070CF096C0CB016B
:1078300001969093E4048093E304BC018091E708EF
:10784000E82FFF27EE0FFF1FE155F74F8081918151
:1078500082599F4F4091E1045091E2044817590723
:107860000CF06CC0CA0101969093E2048093E1048D
:10787000AC018091E808E82FFF27EE0FFF1FE155CC
:10788000F74F8081918182599F4F2091DF04309181
:10789000E004281739070CF042C0C9010196909303
:1078A000E0048093DF049C01B7FD7FC0AF3FB105CA
:1078B00011F00CF061C077FD67C06F3F710539F0C2
:1078C00034F08FEF90E09093E4048093E30457FD4D
:1078D00061C04F3F510539F034F08FEF90E0909345
:1078E000E2048093E10437FD5BC02F3F310509F0CE
:1078F0000CF463C08FEF90E09093E0048093DF047A
:107900005CC08081918182599F4F8A179B070CF040
:107910007ACF109709F477CFCD0101976FCF80818F
:10792000918182599F4F821793070CF0BDCF21158B
:10793000310509F4B9CFC9010197B1CF8081918197
:1079400082599F4F841795070CF093CF411551052D
:1079500009F48FCFCA01019787CF80819181825925
:107960009F4F861797070CF069CF6115710509F4D1
:1079700065CFCB0101975DCF8FEF90E09093E60448
:107980008093E50477FF99CF1092E4041092E3040A
:1079900057FF9FCF1092E2041092E10437FFA5CF6A
:1079A0001092E0041092DF0408C01092E6041092D6
:1079B000E50481CF0E94AE1CA8CE809117099927BB
:1079C000AA27BB27BC01CD0124EC39E040E050E000
:1079D0000E94356CDC01CB018093A6039093A70332
:1079E000A093A803B093A903809118099927AA2707
:1079F000BB27BC01CD010E94356CDC01CB0180931B
:107A0000A2039093A303A093A403B093A5030895A6
:107A10006F927F928F929F92AF92BF92CF92DF929E
:107A2000EF92FF920F931F93CF9300E010E0780145
:107A30006801469A10933805009337051093360570
:107A40000093350580E090E0A0E0B0E080932F0542
:107A500090933005A0933105B09332051093420501
:107A6000009341051093400500933F0510933E0598
:107A700000933D05109375090093740910928F03CC
:107A800010928E03109212040E94803B84E690E0D4
:107A90000E9414180E94803B8091E90880FF10C06A
:107AA00080911D0390911E03875B934008F0FBC1FA
:107AB00080911D0390911E038E5E924008F4F3C1E5
:107AC000CFE18AE090E00E94141880911E0490910A
:107AD0001F04080F191F8091220490912304E80EBF
:107AE000F91E8091200490912104C80ED91EC15026
:107AF000C7FFE7CFA701405F5F4F56954795569563
:107B0000479550934205409341059601205F3F4FB2
:107B100036952795369527953093400520933F0558
:107B2000C801409696958795929582958F70892782
:107B30009F70892790933E0580933D05909375092A
:107B40008093740930933C0520933B0550933A058C
:107B50004093390544E050E0DA010E94C46C802D66
:107B6000853008F4A3C18091AF099091B00997FDC9
:107B7000D2C16CE070E00E94746C70933605609323
:107B80003505809193099091940997FDD5C16CE0DA
:107B900070E00E94746C7093380560933705809193
:107BA000690890916A08AA2797FDA095BA2FBC0191
:107BB000CD010E94BB6BDC01CB0180932F0590931C
:107BC0003005A0933105B0933205109258091092F8
:107BD000570910924909109248091092A50910926C
:107BE000A40984E690E00E94141880911A049091F0
:107BF0001B04AA2797FDA095BA2F9C01AD01220F67
:107C0000331F441F551F220F331F441F551F280FBA
:107C1000391F4A1F5B1F280F391F4A1F5B1F3093F4
:107C200094092093930980911C0490911D04AA2724
:107C300097FDA095BA2F7C018D01EE0CFF1C001F53
:107C4000111FEE0CFF1C001F111FE80EF91E0A1F6A
:107C50001B1FE80EF91E0A1F1B1FF092B009E092CD
:107C6000AF098091F808682E772488249924C901E7
:107C70009C01442737FD4095542FC401B3010E9455
:107C8000356C5B016C016093290570932A05809324
:107C90002B0590932C059701442737FD4095542FD1
:107CA000C401B3010E94356CDC01CB018093210536
:107CB00090932205A0932305B0932405A092050577
:107CC000B0920605C0920705D09208058093FD0486
:107CD0009093FE04A093FF04B09300051092F90462
:107CE0001092FA041092FB041092FC0480911F037E
:107CF00090912003A0912103B091220390936C08EE
:107D000080936B0810921104109210041092F104E9
:107D10001092F2041092F3041092F4048091EF0494
:107D20009091F0049093EE048093ED040E948A6297
:107D300082E390E09093FC038093FB03809117090A
:107D40009927AA27BB27BC01CD0124EC39E040E0EC
:107D500050E00E94356CDC01CB018856954CAF4F4A
:107D6000BF4F8093A6039093A703A093A803B0935B
:107D7000A903809118099927AA27BB27BC01CD0127
:107D80000E94356CDC01CB018856954CAF4FBF4F3C
:107D90008093A2039093A303A093A403B093A5039D
:107DA00010928B0310928A038091EF049091F0045B
:107DB000AA2797FDA095BA2F2091860330918703BB
:107DC0004091880350918903BC01CD010E94356C1C
:107DD000DC01CB018093AB099093AC09A093AD0972
:107DE000B093AE091092E8041092E70481E080930A
:107DF00001010E947F668091AD0484608093AD0490
:107E00008FEF8093140A1092150A80E28093160A6D
:107E10008091E508E82FFF27EE0FFF1FE155F74F90
:107E20008081918182599F4F9093E6048093E5046D
:107E30008091E608E82FFF27EE0FFF1FE155F74F6F
:107E40008081918182599F4F9093E4048093E30451
:107E50008091E708E82FFF27EE0FFF1FE155F74F4E
:107E60008081918182599F4F9093E2048093E10435
:107E70008091E808E82FFF27EE0FFF1FE155F74F2D
:107E80008081918182599F4F9093E0048093DF0419
:107E900084E68093DE048091F903882309F450C0BE
:107EA000469A579A4DC00E945C1C0ACEDA010E9485
:107EB000C46C802D9927982F8827DA0111960E948B
:107EC000C46C202D820F911D909338058093370547
:107ED000DA0112960E94C46C802D9927982F88276A
:107EE000DA0113960E94C46C202D820F911D90938D
:107EF000360580933505DA0114960E94C46C802DF6
:107F00009927982F8827DA0115960E94C46C202D96
:107F1000820F911D48CE909581959F4F6CE070E047
:107F20000E94746C709336056093350580919309B7
:107F30009091940997FF2BCE909581959F4F27CED6
:107F4000CF911F910F91FF90EF90DF90CF90BF9056
:107F5000AF909F908F907F906F9008959091D404F0
:107F6000992381F58091AD048C7F8093AD0410C07E
:107F7000A92FBB27FD01E859F84F8083FD01E8597F
:107F8000F84F8081AA56B64F8C939F5F9C3080F447
:107F90008091DC03882361F3A92FBB27FD01E859F9
:107FA000F84F8081AA56B64F8C939F5F9C3080F328
:107FB0008091DC03882359F08091DC038150809309
:107FC000DC0305C08091AD0481608093AD04809195
:107FD0009609992790933E0880933D0880919709D0
:107FE00099279093400880933F0880919909992799
:107FF0009093420880934108809198099927909323
:1080000044088093430810924904109248040E9447
:10801000D82A08958091EC088B3F68F08B3F09F4D3
:10802000D5C28C3F09F474C38D3F09F4F6C28E3F6C
:1080300021F48091DF0480939E038091EB088B3FB5
:1080400008F439C28B3F09F434C28C3F09F448C3A9
:108050008D3F09F4D9C28E3F09F478C380919F0304
:10806000882309F02DC280939F038091ED088B3FF8
:1080700008F42DC28B3F09F428C28C3F09F442C397
:108080008D3F09F4C4C28E3F09F45AC380919D0309
:10809000882309F021C280939D038091EF088B3FD4
:1080A00068F08B3F09F495C28C3F09F42EC38D3FD5
:1080B00009F4B0C28E3F21F48091DF0480939C03C9
:1080C0008091F1088B3F68F08B3F09F479C28C3FB7
:1080D00009F4E2C28D3F09F4BEC28E3F21F48091C3
:1080E000DF0480939A038091F9088B3F68F08B3FFF
:1080F00009F469C28C3F09F4FCC28D3F09F490C2B7
:108100008E3F21F48091DF0480939B038091FA08D5
:108110008B3F08F4E8C18B3F09F4E3C18C3F09F4BD
:10812000EEC28D3F09F494C28E3F09F412C38091D0
:1081300098038B3008F4DCC18F3F11F480939803CF
:108140008091FB088B3F68F08B3F09F427C28C3F7E
:1081500009F4D2C28D3F09F466C28E3F21F48091AA
:10816000DF04809397038091FC088B3F68F08B3F7E
:1081700009F417C28C3F09F489C28D3F09F46EC21D
:108180008E3F21F48091DF04809399038091FD0854
:108190008B3F68F08B3F09F407C28C3F09F479C22A
:1081A0008D3F09F452C28E3F21F48091DF04809309
:1081B00096038091FE088B3F68F08B3F09F4F7C16E
:1081C0008C3F09F4ABC28D3F09F43CC28E3F21F4D1
:1081D0008091DF0480939503209103092B3F08F4DD
:1081E0008BC12B3F09F486C12C3F09F47CC22D3F83
:1081F00009F404C22E3F09F4A6C220919303809192
:1082000004098B3F08F07FC18093C1048091050968
:108210008B3F68F08B3F09F4D0C18C3F09F466C2F4
:108220008D3F09F4EEC18E3F21F48091DF048093ED
:10823000C004809106098B3F68F08B3F09F484C12C
:108240008C3F09F471C28D3F09F4D2C18E3F21F4F5
:108250008091DF048093BF04809107098B3F68F011
:108260008B3F09F474C18C3F09F461C28D3F09F45E
:10827000C2C18E3F21F48091DF048093BE048091BF
:108280001C098B3F68F08B3F09F464C18C3F09F4F3
:1082900054C28D3F09F4A3C18E3F21F48091DF04C5
:1082A0008093BD0480911D098B3F68F08B3F09F4DA
:1082B00054C18C3F09F42FC28D3F09F493C18E3F06
:1082C00021F48091DF048093BC0480911E098B3FD0
:1082D00068F08B3F09F444C18C3F09F4ECC18D3F39
:1082E00009F4C5C18E3F21F48091DF048093BB0463
:1082F00080911F098B3F68F08B3F09F434C18C3F9C
:1083000009F4DCC18D3F09F4B5C18E3F21F48091A1
:10831000DF048093BA04809108098B3F68F08B3F9B
:1083200009F424C18C3F09F4CFC18D3F09F484C105
:108330008E3F21F48091DF048093920380910C0999
:108340008B3F68F08B3F09F414C18C3F09F4BFC127
:108350008D3F09F474C18E3F21F48091DF04809336
:108360009103809111098B3F68F08B3F09F404C1A0
:108370008C3F09F4AFC18D3F09F458C18E3F21F401
:108380008091DF0480939003809114098B3F68F003
:108390008B3F09F4F4C08C3F09F49FC18D3F09F471
:1083A00048C18E3F21F48091DF0480938F03809138
:1083B00015098B3F68F08B3F09F4E4C08C3F09F44A
:1083C0006EC18D3F09F44DC18E3F21F48091DF04D1
:1083D00080938E03809116098B3F68F08B3F09F4E0
:1083E000D4C08C3F09F464C18D3F09F43DC18E3F78
:1083F00021F48091DF0480938D0380911B098B3FD2
:1084000068F08B3F09F4C4C08C3F09F45AC18D3F1A
:1084100009F433C18E3F21F48091DF0480938C03F3
:10842000809121098B3F08F47FC08B3F09F47AC00B
:108430008C3F09F437C18D3F09F422C18E3F09F406
:108440008BC180916F09823008F473C08F3F11F4A3
:1084500080936F09809123098B3F08F46EC08B3F96
:1084600009F469C08C3F09F420C18D3F09F40BC1A8
:108470008E3F09F474C18091A209823008F462C071
:108480008F3F11F48093A209809136098B3F70F0E1
:108490008B3F09F480C08C3F09F44CC18D3F09F437
:1084A0009BC08E3F09F05EC18091DF048093B209CA
:1084B00059C18091E50480939F03882309F4D3CDAB
:1084C000843608F4D2CD84E6CECD8091E504809345
:1084D0009D03882309F4DFCD843608F4DECD84E6DD
:1084E000DACD8091E504809398038B3008F024CE98
:1084F0008AE024CE2091E50420939303809104091F
:108500008B3F08F481CE8B3F09F454C08C3F09F4B3
:1085100008C18D3F09F469C08E3F09F077CE809184
:10852000DF0472CE8091E50480936F09823008F0F9
:108530008DCF81E08DCF8091E5048093A2098230B8
:1085400008F09ECF81E09ECF8091E50483CE80919C
:10855000E50493CE8091E504A3CE8091E504B3CEEB
:108560008091E504C3CE8091E504D3CE8091E504EB
:10857000E3CE8091E504F3CE8091E50403CF8091B2
:10858000E50413CF8091E50423CF8091E50433CF38
:108590008091E50443CF8091E50488CF8091E50484
:1085A000E0CD8091E504F0CD8091E50400CE80918E
:1085B000E50410CE8091E50427CE8091E50437CE06
:1085C0008091E5048ECD8091E5049ECD8091E504F7
:1085D00032CD8091E50472CD8091E10467CF809126
:1085E000E1045ECE8091E1046ECE8091E1040CCE78
:1085F0008091E1042FCE8091E1043FCE2091E104EF
:108600007BCF8091E10413CE8091E10454CF80911F
:10861000E1045DCF8091E10451CD8091E1040BCD67
:108620008091E10471CD8091E1049BCD8091E104C2
:10863000A9CE8091E104B9CE8091E1047DCE8091F4
:10864000E1048DCE8091E104C5CD8091E104AFCDF0
:108650008091E10448CF8091E10443CD8091E10411
:1086600093CD8091E104B4CE8091E104C4CE809199
:10867000E1043CCE8091E1044CCE8091E104CECE69
:108680008091E10451CF8091E10457CF8091E304C0
:108690007BCD8091E3048BCD8091E30422CD80914A
:1086A000E30496CE8091E3043FCF8091E30445CF6D
:1086B0008091E304A0CE8091E30418CE8091E3047E
:1086C00028CE8091E304AACE8091E30435CE809138
:1086D000E30445CE8091E30455CE8091E30465CE5A
:1086E0008091E304E8CE2091E30406CF8091E30477
:1086F0009ECD8091E30408CD8091E30432CD80913A
:10870000E304F1CE8091E304E2CE8091E304D6CC81
:108710008091E30490CC8091E304D5CD8091E30473
:1087200059CD8091E30470CD8091E30493CD809185
:10873000E304A3CD8091E304B9CE8091E304B0CDEE
:108740008091DF04C4CE2091DF04D6CE8091DF0477
:10875000B2CE8091DF04C7CE8091DF04E5CE809158
:10876000DF04EBCE33272F5F3F4F8CE398E2B90154
:108770000E94746C7093A1036093A0038091F7082A
:108780008093A3098091F60880935C0908952F9245
:108790003F924F925F926F927F928F929F92AF9291
:1087A000BF92CF92DF92EF92FF920F931F93CF93DE
:1087B000DF93CDB7DEB7EC970FB6F894DEBF0FBEF0
:1087C000CDBF8091AC04815009F485E08093AC0466
:1087D0000E94E731209102012C3008F0BAC2299A98
:1087E000A090D504B090D604BC82AB8280915C0985
:1087F00099270A96A816B90614F49C838B83809156
:10880000DE04843608F0A7C28091790590917A053C
:10881000009709F081C41092D4048091AD048F7E3A
:108820008093AD042A3009F47FC4243109F47CC458
:1088300028988091AE049091AF04895E934008F42B
:108840007CC480910009282F33273C832B8380919F
:10885000AD0480618093AD048091E108A82FBB270F
:10886000AA0FBB1FFD01EB53F74F118210828091BD
:10887000E208282F3327220F331FC9018B53974F4C
:10888000FC0111821082A155B74F11961C921E92C5
:108890002155374FD90111961C921E928091E40800
:1088A000E82FFF27EE0FFF1FE155F74F11821082CF
:1088B00080918403815080938403809184038F3F4F
:1088C00021F08091AD0484FF3BC40E940A40809156
:1088D000880590918905AC01440F551F480F591F19
:1088E0000091E108A02FBB27AA0FBB1FFD01E15596
:1088F000F74FE090F308CE2CDD24808191818C9D90
:1089000050018D9DB00C9C9DB00C11244A0D5B1D37
:1089100057FF02C00C94FD585595479555954795BE
:10892000AB53B74F8091F408682F77278D919C91B6
:10893000869F9001879F300D969F300D1124240F44
:10894000351F30938905209388058091BF0590914C
:10895000C0054091BB055091BC05840F951F281B95
:10896000390B3093DC042093DB0480918A059091CD
:108970008B05AC01440F551F480F591F1091E20899
:10898000A12FBB27AA0FBB1FFD01E155F74F808127
:1089900091818C9D90018D9D300D9C9D300D1124F9
:1089A000420F531F57FF02C00C94F9585595479535
:1089B00055954795AB53B74F8D919C91869F9001EC
:1089C000879F300D969F300D1124240F351F309353
:1089D0008B0520938A058091BD059091BE0540913D
:1089E000B9055091BA05840F951F281B390B309398
:1089F000DA042093D9048091E408E82FFF27EE0FD2
:108A0000FF1FE155F74F80819181909581959F4F90
:108A10008330910514F40C94744F02979093D8040A
:108A20008093D7048091E308E82FFF27EE0FFF1F04
:108A3000E155F74FC080D18048E750E0C40ED51E05
:108A4000809198039927AA2797FDA095BA2FBC017A
:108A5000CD010E94BB6BDC01CB0120E030E040E2A5
:108A600051E4BC01CD010E945C6BDC01CB01BC0177
:108A7000CD010E949E6BDC01CB018093A909F0908F
:108A80009703809196039927AA2797FDA095BA2F5F
:108A9000BC01CD010E94BB6BDC01CB0120E030E0CA
:108AA00040E251E4BC01CD010E945C6BDC01CB01D2
:108AB000BC01CD010E949E6BDC01CB0180934F096C
:108AC000509195035093660980918A0780FF06C0F4
:108AD0008091B209813810F00C94D74FD092D6040F
:108AE000C092D5048091D5049091D60497FF02C01E
:108AF0000C94F358F091E908FE8BF2FD02C00C943F
:108B0000BE4F109276094091DB045091DC04CA01FB
:108B100057FF02C00C94C94F9595879595958795F9
:108B200097FF02C00C94D24F2091B2043091B3044D
:108B30002817390714F00C947C4FCA0157FF02C064
:108B40000C94C15C97FF02C00C94C65CBC01759587
:108B50006795759567956536710514F40C947F4F8C
:108B600064E670E04091D9045091DA04CA0157FDDF
:108B700002C00C94884F0396959587959595879597
:108B800097FD02C00C94904F909581959F4F209136
:108B9000B0043091B1042817390714F40C94994F9C
:108BA000215030408091AD0484FD02C00C94B44F3C
:108BB0001092B3041092B2041092B1041092B00457
:108BC000E12FFF27EE0FFF1FE155F74F40911209EC
:108BD000242F3327808191812817390734F480911D
:108BE000370982FF02C00C944B50E12FFF27EE0F94
:108BF000FF1FE155F74F842F992720911309821BFE
:108C00009109208131812817390714F41092C50485
:108C1000E12FFF27EE0FFF1FE155F74F842F992714
:108C200022273327281B390B8081918182179307D4
:108C300034F48091370983FF02C00C944650809130
:108C4000C404882391F0E12FFF27EE0FFF1FE155A9
:108C5000F74F809113099927841B91092081318155
:108C60008217930714F40C947750E02FFF27EE0F30
:108C7000FF1FE155F74F242F33278081918128175B
:108C8000390734F48091370980FF02C00C944050BA
:108C90005091C204552399F0E02FFF27EE0FFF1FDC
:108CA000E155F74F842F992720911309821B9109D1
:108CB000208131812817390714F40C947250E02F69
:108CC000FF27EE0FFF1FE155F74F842F992722272B
:108CD0003327281B390B808191818217930734F445
:108CE0008091370981FF02C00C943B508091C304EE
:108CF000882391F0E02FFF27EE0FFF1FE155F74F7C
:108D0000809113099927841B910920813181821751
:108D1000930714F40C947B508091C504882331F49C
:108D20008091C404882311F40C94385091E05523A9
:108D300031F48091C304882311F40C94565081E0DF
:108D40008093C7041092C6041092C5041092C40404
:108D5000FAC1299845CD8091DE048D3808F4A8CD5C
:108D60008091AD048F7E8093AD049091010982E3E0
:108D7000989FC001112490937A0580937905EB8127
:108D8000FC81B99714F00C945B508091AE049091E3
:108D9000AF048F3F910519F010F00C94EC5810922D
:108DA0005D0510925E0510925F05109260051092AD
:108DB00061051092620510926305109264058A3F66
:108DC000910511F40C94245E3091E308E32FFF2702
:108DD000EE0FFF1FE155F74F80819181813591059D
:108DE0000CF4E9C04091D404442309F0E4C080911C
:108DF000E408E82FFF27EE0FFF1FE155F74F8081B2
:108E000091818C34910514F40C94555D80917B050F
:108E10008F5F893C10F40C94665E2C3010F00C943B
:108E20005C5F29981092D40410927B051092AF04D5
:108E30001092AE040091E108E02FFF27EE0FFF1F14
:108E4000E155F74F808191818734910514F00C949E
:108E5000585F1091E208E12FFF27EE0FFF1FE15549
:108E6000F74F808191810190F081E02DF7FF02C0E2
:108E70000C941F62E734F1050CF470C021E0A12FBF
:108E8000BB27AA0FBB1FA155B74F8D919C9111977E
:108E90008734910544F0E02FFF27EE0FFF1FE155C7
:108EA000F74F808191818D919C918734910564F079
:108EB000E02FFF27EE0FFF1FE155F74F80819181D3
:108EC000873491050CF022E0E12FFF27EE0FFF1F02
:108ED000E155F74F808191818634910564F4E02F4C
:108EE000FF27EE0FFF1FE155F74F808191818734F7
:108EF00091050CF023E0E12FFF27EE0FFF1FE15556
:108F0000F74F808191818A5B9F4F64F4E02FFF27A8
:108F1000EE0FFF1FE155F74F808191818734910556
:108F20000CF024E0E12FFF27EE0FFF1FE155F74F74
:108F3000808191818A5B9F4F64F4E02FFF27EE0FC1
:108F4000FF1FE155F74F80819181863491050CF424
:108F500025E0822F0E9477051091E208E12FFF277C
:108F6000EE0FFF1FE155F74F808191810190F08155
:108F7000E02DF7FF02C00C941F617E9714F00C9453
:108F8000EE5E8091E108E82FFF27EE0FFF1FE1550D
:108F9000F74F808191818A5B9F4F14F00C94EE5EB5
:108FA00081E080937E0788EE93E09093FC038093AA
:108FB000FB033091E308E32FFF27EE0FFF1FE1557E
:108FC000F74F808191818B5A9F4F0CF071CC90901C
:108FD000E408E92DFF27EE0FFF1FE155F74F8081D1
:108FE0009181855B9F4F14F00C940F5A80917C0502
:108FF0008F5F893C10F40C94525D88EC80937C0563
:1090000081E090E09093AF048093AE0481E0809380
:10901000D4041092650510926605109267051092AF
:1090200068051092F9041092FA041092FB04109251
:10903000FC041092F5041092F6041092F7041092BA
:10904000F8048091F808A82EBB24CC24DD2480915C
:109050009309909194099C01442737FD4095542F22
:10906000C601B5010E94356CDC01CB018093090576
:1090700090930A05A0930B05B0930C058091AF095E
:109080009091B0099C01442737FD4095542FC601AB
:10909000B5010E94356CDC01CB01809301059093F2
:1090A0000205A0930305B0930405809129059091D2
:1090B0002A05A0912B05B0912C058093050590936E
:1090C0000605A0930705B0930805809121059091AE
:1090D0002205A0912305B09124058093FD0490936F
:1090E000FE04A093FF04B093000510925D0510925A
:1090F0005E0510925F051092600510926105109256
:10910000620510926305109264058091AD04886039
:109110008093AD040C94115A019790937A05809333
:1091200079052A3009F081CB289A8091AE0490917C
:10913000AF04895E934008F084CB1092D404B8CB7E
:10914000A090E908AE8A0091C6040FA3002321F481
:109150008091C704882369F08091110999272B8198
:109160003C818217930714F49C838B8381E0809366
:10917000E9048091AD0484FFB3C61092D804109224
:10918000D7041092DC041092DB041092DA041092DF
:10919000D9049AE59093A90988E78093760990937A
:1091A0004F0988A7809366091092C6041092C704DD
:1091B0001FA22091690930916A0940916B09509171
:1091C0006C096091290570912A0580912B05909179
:1091D0002C056D8F7E8F8F8F98A3260F371F481F0A
:1091E000591F8091700990917109A0917209B091F5
:1091F0007309A0902105B0902205C0902305D0905E
:109200002405AA8ABB8ACC8ADD8A8A0D9B1DAC1DE7
:10921000BD1DC0905E09D0905F09E0906009F0909C
:109220006109CDAADEAAEFAAF8AEE0902505F0907C
:1092300026050091270510912805EAA2FBA20CA3A0
:109240001DA3ADA8BEA8CFA8D8ACAE0CBF1CC01E35
:10925000D11EADAABEAACFAAD8AEC0905009D09058
:109260005109E0905209F0905309C9AADAAAEBAA71
:10927000FCAAE0901D05F0901E0500911F051091BD
:109280002005E9A6FAA60BA71CA7A9A8BAA8CBA8EF
:10929000DCA8AE0CBF1CC01ED11EA9AABAAACBAABC
:1092A000DCAAB090C704BB8EBB2009F0B8C50FA1E3
:1092B000002309F0B4C58093700990937109A093BD
:1092C0007209B09373092093690930936A09409336
:1092D0006B0950936C098091690890916A088150DC
:1092E00092400CF066C48091D404882309F061C4D4
:1092F00080910E0490910F048F3F910509F008F4BE
:1093000067C5BB8DBB2309F0FFC6EFA1EE2309F0B3
:10931000FBC6F091E904FEA3FF2309F0F5C6A09077
:109320001A09AC8EAA2009F4EFC6CDA8DEA8EFA8D2
:10933000F8ACC0925E09D0925F09E0926009F092A9
:109340006109E9A8FAA80BA91CA9E0925009F092BA
:109350005109009352091093530980916909909122
:109360006A09A0916B09B0916C09B7FF02C00C9417
:109370005260292E3A2E4B2E552447FC5A942092A7
:10938000690930926A0940926B0950926C09809188
:10939000700990917109A0917209B0917309B7FF9A
:1093A00002C00C947D60892F9A2FAB2FBB27A7FD9D
:1093B000BA9588879987AA87BB878093700990930D
:1093C0007109A0937209B09373098091F808E82E8F
:1093D000FF24002711272091190530911A0540918B
:1093E0001B0550911C05C801B7010E94356C97FF01
:1093F00002C00C947760672E782E892E992487FC02
:109400009A942091150530911605409117055091B9
:109410001805C801B7010E94356C97FF02C00C9473
:109420008960A72EB82EC92EDD24C7FCDA94D2019C
:10943000C10186199709A809B90920911909222E95
:10944000332444245524BC01CD01A20191010E9482
:10945000A96C39014A012DA73EA74FA758AB8885B3
:109460009985AA85BB858A199B09AC09BD09BC01F0
:10947000CD01A20191010E94A96CD401C30197FE04
:1094800002C00C948360892F9A2FAB2FBB27A7FDB6
:10949000BA95BC01DA01C90157FF02C00C948F6074
:1094A000892F9A2FAB2FBB27A7FDBA955C0180911E
:1094B000B2049091B30481349105D4F48091B00446
:1094C0009091B104813491059CF48091E408E82FD7
:1094D000FF27EE0FFF1FE155F74F8081918101902B
:1094E000F081E02DF7FF02C00C9416627A9734F0F9
:1094F0008091140A8F3F11F40C94285F0AA11BA1DC
:109500002CA13DA18D8D9E8DAF8DB8A1081B190B8F
:109510002A0B3B0B09AF1AAF2BAF3CAF0093690589
:1095200010936A0520936B0530936C0529A43AA427
:109530004BA45CA4CA88DB88EC88FD882C183D0805
:109540004E085F0820926D0530926E0540926F05BF
:109550005092700500937105109372052093730566
:109560003093740520927505309276054092770508
:10957000509278058091050590910605A091070508
:10958000B0910805801B910BA20BB30B80930505CE
:1095900090930605A0930705B09308058091FD04FC
:1095A0009091FE04A091FF04B091000582199309E7
:1095B000A409B5098093FD049093FE04A093FF04D1
:1095C000B0930005DC8CDD2071F12091E70430912F
:1095D000E8042138310594F080913D0590913E05D5
:1095E000019690933E0580933D058091740990917A
:1095F00075090196909375098093740920583F4F1F
:1096000094F480913D0590913E05019790933E051D
:1096100080933D058091740990917509019790930D
:109620007509809374091092E8041092E70401E030
:10963000C02ED12C89AD9AADABADBCADB7FF02C089
:109640000C946E6081509240A040B0401CF014E039
:10965000C12ED12C8091920590919305A0919405F3
:10966000B0919505E0906909F0906A0900916B0945
:1096700010916C098E199F09A00BB10B815E914B63
:10968000AF4FBF4F8F539C49A040B04010F40C9493
:109690007D5E3091150A39A3393114F40C943E5F84
:1096A000D0928D05C0928C0589AD9AADABADBCADA5
:1096B00081509041A040B04014F40C94B25E80916F
:1096C0008E05882311F40C94A6607093C9046093EE
:1096D000C80489AD9AADABADBCADB7FF02C00C9468
:1096E000C5619C01AD01B7FF02C00C94BF61B9E038
:1096F0005595479537952795BA95D1F780918C0563
:1097000090918D05820F931F90938D0580938C050A
:1097100029AD3AAD4BAD5CAD57FF02C00C94D4619E
:1097200039014A01A3E09594879477946794AA95A8
:10973000D1F76DA67EA68FA698AAF9E86F16F3E179
:109740007F06F0E08F06F0E09F0654F0F8E86F2EF9
:10975000F3E17F2E812C912C6DA67EA68FA698AA70
:10976000D401C30197FE02C00C94CE61892F9A2FB9
:10977000AB2FBB27A7FDBA95680F791F29AD3AAD6E
:109780004BAD5CAD203080EF38078FEF48078FEF8F
:10979000580714F00C94A25E80918F05882311F471
:1097A0000C9495607093C9046093C804DA01C901F0
:1097B00057FF02C00C94EC619C01AD01B7FF02C0E1
:1097C0000C94E66169E055954795379527956A951C
:1097D000D1F780918C0590918D05820F931F909306
:1097E0008D0580938C0529AD3AAD4BAD5CAD57FF2F
:1097F00002C00C94E06139014A0143E095948794DA
:10980000779467944A95D1F798E769169CEE7906A4
:109810009FEF89069FEF990644F438E7632E3CEEEC
:10982000732E3FEF832E3FEF932E60928005709250
:1098300081058092820590928305D401C30197FE31
:1098400002C00C94DA61892F9A2FAB2FBB27A7FD9A
:10985000BA956091C8047091C904680F791F9C8DF6
:10986000292F332780918C0590918D052817390772
:1098700024F430938D0520938C05A9A1AA2379F0B7
:109880002A2F332727FD309580918C0590918D05E7
:109890002817390724F430938D0520938C0529ADC2
:1098A0003AAD4BAD5CAD213831054105510574F041
:1098B000809141059091420520918C0530918D0554
:1098C000820F931F909342058093410589AD9AAD15
:1098D000ABADBCAD80589F4FAF4FBF4F74F480917C
:1098E00041059091420520918C0530918D05821B98
:1098F000930B9093420580934105B1E0CB2ED12C80
:10990000D201C10157FE02C00C94586081509240B0
:10991000A040B0401CF0A4E0CA2ED12C20E030E0E2
:1099200040E050E08091960590919705A0919805B0
:10993000B0919905609070097090710980907209DA
:109940009090730986199709A809B909815E914B0E
:10995000AF4FBF4F8F539C49A040B04028F0F9A1B2
:10996000F93114F40C94125FD0928D05C0928C05DD
:1099700081E0281680E1380680E0480680E058063D
:1099800014F40C94965E80919005882311F40C9445
:109990006160B092CB04A092CA04D201C10157FE0B
:1099A00002C00C94B661B7FF02C00C94B061F9E03C
:1099B000B595A79597958795FA95D1F7C80ED91EB5
:1099C000D0928D05C0928C05A201910157FE02C074
:1099D0000C94AA61E3E05595479537952795EA954C
:1099E000D1F7293893E1390790E0490790E059070A
:1099F00014F40C94A06188E893E1A0E0B0E08093B7
:109A0000840590938505A0938605B0938705809182
:109A1000840590918505A0918605B0918705B7FFD3
:109A200002C00C941062892F9A2FAB2FBB27A7FD81
:109A3000BA95A090CA04B090CB04A80EB91EA0E0BD
:109A40002A16A0EF3A06AFEF4A06AFEF5A0614F017
:109A50000C94B65E80919105882311F40C94AF604C
:109A6000B092CB04A092CA04D201C10157FE02C039
:109A70000C9424629C01AD01B7FF02C00C94FB6101
:109A8000B9E05595479537952795BA95D1F78091C7
:109A90008C0590918D05820F931F90938D05809377
:109AA0008C05A201910157FE02C00C94F561A3E060
:109AB0005595479537952795AA95D1F72837BCEE48
:109AC0003B07BFEF4B07BFEF5B0714F00C949661A9
:109AD00088E79CEEAFEFBFEF8093840590938505F8
:109AE000A0938605B09387058091840590918505A4
:109AF000A0918605B0918705B7FF02C00C94016262
:109B0000892F9A2FAB2FBB27A7FDBA95A090CA0427
:109B1000B090CB04A80EB91EEC8D2E2F3327809168
:109B20008C0590918D052817390724F430938D0505
:109B300020938C05F9A1FF2379F02F2F332727FDE0
:109B4000309580918C0590918D052817390724F464
:109B500030938D0520938C0521E8221631044104B1
:109B6000510474F080913F059091400520918C053F
:109B700030918D05820F931F9093400580933F0590
:109B800030E823163FEF33063FEF43063FEF53061F
:109B90000CF0D0C280913F059091400520918C053A
:109BA00030918D05821B930B9093400580933F0568
:109BB000C1C25090140A6FEF561611F40C94035959
:109BC0008091F808A82EBB24CC24DD246D8D7E8DD9
:109BD0008F8D98A1A60195010E94A96C39014A01B7
:109BE0008091930990919409AA2797FDA095BA2F87
:109BF000681A790A8A0A9B0A6A897B898C899D89F5
:109C0000A60195010E94A96C59016A018091AF09D2
:109C10009091B009AA2797FDA095BA2FA81AB90A62
:109C2000CA0ADB0A252C332427FC3094432C532CFE
:109C3000C201B101A40193010E94356C97FD5FC27E
:109C40003B014C01F9E09594879477946794FA95D9
:109C5000D1F7C201B101A60195010E94356C97FFB1
:109C600002C00C941B5D5B016C01E9E0D594C794C4
:109C7000B794A794EA95D1F78091B2049091B30478
:109C8000813491053CF48091B0049091B104813409
:109C90009105C4F0D401C30197FE02C00C941A5E72
:109CA0003C014D019594879477946794D601C50142
:109CB000D7FE02C00C941F5E5C016D01D594C79461
:109CC000B794A7948091E408E82FFF27EE0FFF1FB9
:109CD000E155F74F808191810190F081E02DF7FFF0
:109CE00002C00C94165D7A97A4F0C401B30123E07E
:109CF00030E040E050E00E94A96C39014A01C60101
:109D0000B50123E030E040E050E00E94A96C590129
:109D10006A018091160A282F332727FD3095432F9B
:109D2000532F261537054805590514F439014A0102
:109D3000992787FD9095909581959F4FAA2797FD2C
:109D4000A095BA2F681679068A069B0614F43C0182
:109D50004D012A153B054C055D0514F459016A01B6
:109D6000A816B906CA06DB0614F45C016D018091E1
:109D7000090590910A05A0910B05B0910C05861973
:109D80009709A809B9098093090590930A05A0933A
:109D90000B05B0930C058091010590910205A091EF
:109DA0000305B09104058A199B09AC09BD0980938C
:109DB000010590930205A0930305B09304058091DB
:109DC0000E0490910F048F3F910511F008F099CA8D
:109DD0004DA95EA96FA978AD40935E0950935F09C4
:109DE000609360097093610969A97AA98BA99CA9FC
:109DF00060935009709351098093520990935309CD
:109E00007091E9047EA3A090D704B090D804C50156
:109E1000B7FEF1C1882799278A199B09ECC11092D6
:109E2000190510921A0510921B0510921C0510922C
:109E3000150510921605109217051092180510922C
:109E4000690910926A0910926B0910926C091092BC
:109E5000700910927109109272091092730919AA6F
:109E60001AAA1BAA1CAA20E030E040E050E02DAB6B
:109E70003EAB4FAB58AF8091090590910A05A09178
:109E80000B05B0910C058093050590930605A093F2
:109E90000705B09308058091010590910205A091F6
:109EA0000305B09104058093FD049093FE04A093F4
:109EB000FF04B093000510920F0410920E0410924C
:109EC000C9041092C8041092CB041092CA043B8DAE
:109ED000332309F00DCA4FA1442309F009CAFBC975
:109EE0003091660938A765C93FEF8E3F93070CF0A4
:109EF000D7C002960C940E45B90161507040409154
:109F0000D9045091DA04CA0157FF02C00C94BB4532
:109F1000959587959595879597FF02C00C94C445B4
:109F20002091B0043091B1042817390714F00C9433
:109F3000D045CA0157FF02C00C94CC5C97FF02C009
:109F40000C94C95C9C013595279535952795253648
:109F5000310514F40C94D24524E630E08091AD0430
:109F600084FF02C00C94D8453093B1042093B00410
:109F70007093B3046093B2040C94E045F0927609B8
:109F80004091DB045091DC04CA0157FD02C00C94DF
:109F90008C450396959587959595879597FD02C075
:109FA0000C949445909581959F4F0C949445809185
:109FB0008307992787FD90954E2D5527849FB001E3
:109FC000859F700D949F700D1124CB012091DB04AF
:109FD0003091DC04820F931F9093DC048093DB04A8
:109FE00080918407992787FD9095849FD001859F54
:109FF000B00D949FB00D1124CD012091D904309162
:10A00000DA04820F931F9093DA048093D90480912D
:10A010008507992787FD90952091D7043091D80422
:10A02000820F931F9093D8048093D7048091870761
:10A03000282F332727FD30958091EE089927289FF8
:10A04000F001299FF00D389FF00D1124F0938B0340
:10A05000E0938A038091860799278C159D0514F05B
:10A060000C946E459093D6048093D5040C9472455D
:10A07000982F0C94974681E08093C3040C948C46EF
:10A0800081E08093C204582F0C945F4681E0809356
:10A09000C4040C94354681E08093C5040C940846B2
:10A0A0001092D8041092D7040C9412459093C604D1
:10A0B0008093C70448C88091D404882311F40C9479
:10A0C000C5468091AE049091AF04FFEF8F3F9F078C
:10A0D00011F40C94C94601969093AF048093AE049A
:10A0E0000C94C9461092C20450E00C945F46109242
:10A0F000C4040C9435461092C3040C948C466150F1
:10A100007E4F8F4F9F4F9CCD60E070E05B011092BF
:10A11000E9041EA2E0906909F0906A0900916B09B8
:10A1200010916C09609070097090710980907209AB
:10A130009090730980917609882311F00C94A958A6
:10A140001092CB041092CA041092C9041092C80451
:10A15000E0929205F0929305009394051093950573
:10A160006092960570929705809298059092990555
:10A170001092190510921A0510921B0510921C05D9
:10A1800010921505109216051092170510921805D9
:10A1900010921105109212051092130510921405D9
:10A1A0001092690910926A0910926B0910926C0959
:10A1B000109270091092710910927209109273092D
:10A1C00010925E0910925F09109260091092610965
:10A1D000109250091092510910925209109253098D
:10A1E00010920F0410920E04A090D704B090D804DF
:10A1F000C501B7FC0FCE409774F068EEC62E63E041
:10A20000D62ED092AB03C092AA038E8984FD03C0E0
:10A2100081E080937F05D090F508ED2CFF24002786
:10A220001127B501882777FD8095982F9501B7FCF8
:10A23000CEC7442737FD4095542F0E94356C9B01B3
:10A24000AC01C801B7010E94356C97FDBBC759E04E
:10A2500095958795779567955A95D1F79B018D2DA3
:10A2600099278A9DD0018B9DB00D9A9DB00D112428
:10A27000CD01B7FD98C79595879595958795280F3A
:10A28000391FC901AA2797FDA095BA2F80936505AC
:10A2900090936605A0936705B0936805E090F90474
:10A2A000F090FA040091FB041091FC04E81AF90AFA
:10A2B0000A0B1B0BB1E5EB16B3ECFB06B0E00B078A
:10A2C000B0E01B070CF43CC780E593ECA0E0B0E0E5
:10A2D0008093F9049093FA04A093FB04B093FC04D8
:10A2E0008091F9049091FA04A091FB04B091FC04D0
:10A2F000805B9C43AF4FBF4F64F480EB9CE3AFEFB8
:10A30000BFEF8093F9049093FA04A093FB04B093F9
:10A31000FC042090EF043090F0042114310409F47F
:10A320000AC6FE89F3FF07C68D8D9E8DAF8DB8A13D
:10A33000B7FF02C00C94E35C09E0B595A79597952B
:10A3400087950A95D1F79AAF89AF97FF02C00C9411
:10A35000EF5C8A899B89AC89BD89B7FF02C00C94E8
:10A36000E95C19E0B595A795979587951A95D1F76A
:10A37000BC0197FF02C00C94DE5CC9ACDAACC61617
:10A38000D70614F47AAF69AF69AD7AAD77FF02C032
:10A390000C94DA5C759567957595679575956795D5
:10A3A0006F5F7F4F7D876C87ACE1EA2EA2E0FA2ECB
:10A3B0002E0C3F1C5101CC24B7FCC094DC2C04EEC5
:10A3C0001DEF200E311E4090AB095090AC096090FB
:10A3D000AD097090AE0920918603309187034091BA
:10A3E0008803509189032F8B388F498F5A8FC3016F
:10A3F000B2010E94A96CA21AB30AC40AD50AC60106
:10A40000B50128E631E040E050E00E94A96CDC0193
:10A41000CB018C01045B10408090A4099090A509A9
:10A42000C40197FE02C00C94D45C8138910514F0ED
:10A4300000E010E0C090AA03D090AB03C114D10497
:10A44000A9F449AD5AAD4931510584F48091E7042E
:10A450009091E804800F911F9093E8048093E704A3
:10A4600080917F05882311F00C94E15DC801880F6D
:10A47000991F880F991F880F991F6C857D850E94F1
:10A48000746C9B01442737FD4095542F240D351DD6
:10A49000461D571D2093AB093093AC094093AD097D
:10A4A0005093AE09F0909B036F2D7727A9ADBAADFD
:10A4B0006A9FC0016B9F900D7A9F900D112497FFAA
:10A4C00002C00C94D15C9595879595958795959547
:10A4D00087959595879595958795681B790B7AAFA4
:10A4E00069AF77FF02C00C94F85CC114D10411F07D
:10A4F0000C940D5D0091B2041091B3048091B004EE
:10A500009091B104080F191F17FF02C00C94515EFF
:10A51000159507951595079515950795005C1F4F9F
:10A52000CA01B9012F89388D498D5A8D0E94A96CB5
:10A53000DA01C9012091ED043091EE04442737FD82
:10A540004095542F821B930BA40BB50B845E9D4F3B
:10A55000AF4FBF4FBC01CD0128E631E040E050E0F5
:10A560000E94A96CDC01CB01845B9040A9ACBAAC21
:10A570008A9DF0018B9DF00D9A9DF00D1124CF0165
:10A58000B8010E94746C83E0F89E60011124DAAE79
:10A59000C9AEC616D70614F00C94005DB601CB0107
:10A5A000AA2797FDA095BA2F2091F9043091FA04BB
:10A5B0004091FB045091FC04820F931FA41FB51F10
:10A5C0008093F9049093FA04A093FB04B093FC04E5
:10A5D00080917E0581508F3F09F4B6C480937E053B
:10A5E0000EA1002381F01092610510926205109275
:10A5F00063051092640510925D0510925E0510923D
:10A600005F05109260051B8D112309F096C580919E
:10A6100076099927AA27BB27BC01CD012D8D3E8D38
:10A620004F8D58A10E94356CDC01CB01BC01CD01DE
:10A6300028EF3AE240E050E00E94A96C19012FA1F6
:10A64000222309F077C5809176099927AA27BB278D
:10A65000BC01CD012A893B894C895D890E94356CFA
:10A66000DC01CB01BC01CD0128EF3AE240E050E033
:10A670000E94A96C3E832D83A0904A09B0904B099B
:10A6800039ECA316B1040CF44AC5B8ECAB2EB12CCE
:10A69000B0924B09A0924A090091550910915609B0
:10A6A000093C11050CF433C508EC10E01093560971
:10A6B000009355098091570990915809AA2797FD51
:10A6C000A095BA2F2091A909C22EDD24EE24FF24E3
:10A6D000BC01CD01A70196010E94356C9B01AC0124
:10A6E000C501AA2797FDA095BA2FF7E0880F991FFB
:10A6F000AA1FBB1FFA95D1F7280F391F4A1F5B1FEE
:10A7000057FD3FC5E6E05595479537952795EA955E
:10A71000D1F7B101620F731F7AAF69AF3B0180912E
:10A72000480990914909AA2797FDA095BA2FBC0125
:10A73000CD01A70196010E94356C9B01AC01C801B7
:10A74000AA2797FDA095BA2F77E0880F991FAA1F17
:10A75000BB1F7A95D1F7280F391F4A1F5B1F57FD82
:10A760000BC566E055954795379527956A95D1F7BE
:10A770000D811E81020F131F5801880C991CC40102
:10A78000AA2797FDA095BA2F20914F093327442778
:10A790005527BC01CD010E94356C6B017C0197FDF2
:10A7A000E2C496E0F594E794D794C7949A95D1F7CC
:10A7B000E8A58E2F9927AA27BB2720910D05309158
:10A7C0000E0540910F0550911005BC01CD010E946E
:10A7D000356CDC01CB01BC01CD0120EF35E540E05B
:10A7E00050E00E94A96C4601820E931EC40129AD5F
:10A7F0003AAD215030442CF060E070E47AAF69AF9C
:10A800003B01A9ADBAADA050B04C0CF07BC420E028
:10A8100030EC3AAF29AF309358092093570930E410
:10A82000013013071CF000E010E4580140EC003048
:10A8300014070CF062C400E010EC10934909009377
:10A84000480951E0851650E4950624F0812C80E4F7
:10A85000982EC40160E0861660EC96060CF048C4A1
:10A86000812CB0EC9B2E9092A5098092A409809136
:10A870000001482F552780912703909128034817FE
:10A88000590794F42091270330912803AB81BC81B0
:10A890004A9FC0014B9F900D5A9F900D1124B90102
:10A8A0000E94606C7C836B83EB81FC81EE0FFF1F49
:10A8B000EE0FFF1FFC83EB83FE89F0FF51C02FA139
:10A8C000222309F04DC03B8D332309F049C080910C
:10A8D0009E0590919F059093500880934F0880911A
:10A8E00010049091110490934A0880934908209194
:10A8F0004305309144052115310509F04DC580917E
:10A900001D0390911E038959934010F00C94FA5D39
:10A9100080911D0390911E038436910510F00C94D4
:10A92000605E87B58B3010F40C94545F80911204F4
:10A930008F5F809312049AE0890290011124809124
:10A940007308821B87BD8CE291E09093FC03809397
:10A95000FB038EE591E090934405809343053DC54C
:10A96000D090A30980915C09282F3327C901880F53
:10A97000991F880F991F88964B815C81481759074A
:10A9800014F49C838B838D2D9927880F991F880F32
:10A99000991F805590406B817C818617970714F42E
:10A9A0009C838B83809146048823A1F08091AE0420
:10A9B0009091AF040297C09768F48B819C81181620
:10A9C000190644F481E090E09093AF048093AE04C4
:10A9D0003C832B83AB81BC81B0933408A0933308B4
:10A9E0008091650590916605A0916705B091680515
:10A9F000880F991FAA1FBB1F880F991FAA1FBB1F73
:10AA00002401481A590AEB81FC81E13AF1050CF462
:10AA10005DC3CF01F7FDF5C3959587958415950521
:10AA20000CF42C01909581959F4F481659060CF413
:10AA30002C012D2D3327220F331F220F331FC90165
:10AA40004B815C81841B950B841595050CF42C01BE
:10AA50006B817C81621B730B461657060CF42B012D
:10AA60008091DB049091DC04A9ACBAACA81AB90AB5
:10AA7000B0926809A0926709C0907609CC2009F4C9
:10AA80001FC3281A390AC101AA2797FDA095BA2F1A
:10AA900020915D0530915E0540915F055091600504
:10AAA000820F931FA41FB51F80935D0590935E05D1
:10AAB000A0935F05B093600560915D0570915E05A0
:10AAC00080915F05909160056130AAEF7A07A0E060
:10AAD0008A07A0E09A0774F080E09AEFA0E0B0E067
:10AAE00080935D0590935E05A0935F05B09360052C
:10AAF000BC01CD016030B6E07B07BFEF8B07BFEF35
:10AB00009B0774F480E096E0AFEFBFEF80935D05A4
:10AB100090935E05A0935F05B0936005BC01CD01E5
:10AB2000E090A003F090A1039701442737FD4095E2
:10AB3000542F0E94A96CA20EB31EBA82A982D09093
:10AB40008C036D2D772788279927920157FC26C300
:10AB500037FD21C335952795EB81FC812E0F3F1FD3
:10AB6000442737FD4095542F0E94356C97FD0EC346
:10AB700056E095958795779567955A95D1F79B01FE
:10AB8000A980BA806A157B0514F47A8369833095AD
:10AB900021953F4F49815A814217530714F43A8354
:10ABA00029838091D9049091DA04081B190B109322
:10ABB000470900934609CC2009F47CC26D817E814F
:10ABC000681B790BCB01AA2797FDA095BA2F20917E
:10ABD0006105309162054091630550916405820FD3
:10ABE000931FA41FB51F8093610590936205A093E6
:10ABF0006305B09364056091610570916205809171
:10AC00006305909164056130AAEF7A07A0E08A0796
:10AC1000A0E09A0774F080E09AEFA0E0B0E08093A3
:10AC2000610590936205A0936305B0936405BC0130
:10AC3000CD016030B6E07B07BFEF8B07BFEF9B070E
:10AC400074F480E096E0AFEFBFEF809361059093DE
:10AC50006205A0936305B0936405BC01CD01970123
:10AC6000442737FD4095542F0E94A96C1801220EED
:10AC7000331E6D2D772788279927920157FC9DC297
:10AC800037FD98C235952795EB81FC812E0F3F1F2C
:10AC9000442737FD4095542F0E94356C97FD85C29F
:10ACA00026E095958795779567952A95D1F79B012D
:10ACB000621573050CF41B01309521953F4F221648
:10ACC00033060CF4190106E9602E09E0702E13ED2D
:10ACD000A12E15E0B12E88249924FBE0FF83F50115
:10ACE000258512160CF0D5C0CB80DC80C601AA27C2
:10ACF00097FDA095BA2F332727FD3095432F532F6B
:10AD0000BC01CD010E94356C97FD10C1B6E0959550
:10AD1000879577956795BA95D1F77AAF69AFE9804E
:10AD2000FA80C701AA2797FDA095BA2FF5012685BD
:10AD3000332727FD3095432F532FBC01CD010E94AF
:10AD4000356C97FDEEC0A6E095958795779567954C
:10AD5000AA95D1F7C9ACDAACC60ED71EDAAEC9AE29
:10AD6000C101AA2797FDA095BA2FF50127853327A2
:10AD700027FD3095432F532FBC01CD010E94356C28
:10AD800097FDCAC0F6E09595879577956795FA95F2
:10AD9000D1F7C9ACDAACC60ED71EDAAEC9AEC20165
:10ADA000AA2797FDA095BA2FF5012089332727FD03
:10ADB0003095432F532FBC01CD010E94356C97FD78
:10ADC000A6C0E6E09595879577956795EA95D1F7C2
:10ADD000C9ACDAACC60ED71EDAAEC9AE0091C1045A
:10ADE000033308F05DC07401E80CF91C9701295881
:10ADF000364F3F872E87D9016D917C91C6010E9405
:10AE00004731EE85FF8591838083802F8353823382
:10AE100080F497012958364F398B288BD9016D91D1
:10AE20007C9189AD9AAD0E945D31E889F989918361
:10AE30008083802F85568436B8F1093C08F049C0DC
:10AE400037E7C32E39E0D32EEC0CFD1CD7016D91F2
:10AE50007C9177FD59C075956795759567957AAF23
:10AE600069AF80915C09992768177907B4F08091E0
:10AE7000A3099927E9ADFAAD8E179F0774F0E9ADE4
:10AE8000D301EC930C946062F501258512160CF445
:10AE90002BCFD3011C920C9460629AAF89AFEFCF95
:10AEA0007401E80CF91CB1CF57E7C52E59E0D52E37
:10AEB000CE0CDF1CD6016D917C9189AD9AAD0E94BC
:10AEC0009631F601918380830091C104093C08F416
:10AED000B7CF47E7C42E49E0D42ECE0CDF1CD601F5
:10AEE0006D917C9189AD9AAD0E946E31F60191838E
:10AEF000808337E7C32E39E0D32EEC0CFD1CD7013D
:10AF00006D917C9177FFA7CF6D5F7F4FA4CF615C80
:10AF10007F4F8F4F9F4F55CF615C7F4F8F4F9F4F1C
:10AF200031CF615C7F4F8F4F9F4F0DCF615C7F4F63
:10AF30008F4F9F4FEBCE8090A4099090A5098091F0
:10AF40007E05815008F04ACB88E180937E05809190
:10AF5000F8089927880F991F880F991F5C01CC2446
:10AF6000B7FCC094DC2C6D8D7E8D8F8D98A1A601D1
:10AF700095010E94A96C30932608209325086A89C0
:10AF80007B898C899D89A60195010E94A96C3093CB
:10AF9000280820932708809193099091940997FDA0
:10AFA000EEC4959587959595879590932A088093FB
:10AFB00029088091AF099091B00997FDDEC495955D
:10AFC00087959595879590932C0880932B08909260
:10AFD0002E0880922D088091D0049091D104A091E8
:10AFE000D204B091D304BC01CD0125E030E040E0B3
:10AFF00050E00E94A96C3093300820932F08809174
:10B00000690890916A0890933208809331083092D1
:10B010003608209235088091270390912803909359
:10B020003808809337088091DE04992790933A0876
:10B03000809339088091AB099091AC09A091AD093A
:10B04000B091AE0920918603309187034091880327
:10B0500050918903BC01CD010E94A96C30933C083A
:10B0600020933B08809110049091110490934A081A
:10B070008093490880917E07992790934C0880938C
:10B080004B088091F7039091F80390934E088093BA
:10B090004D088091BF059091C00590936208809300
:10B0A00061088091BD059091BE05909364088093DE
:10B0B000630896CAC801AA2797FDA095BA2F87CD25
:10B0C000C501AA2797FDA095BA2FE2CCF1E54F164E
:10B0D00051041CF0B0E54B2E512C20EB42162FEF03
:10B0E00052060CF0A6CCA0EB4A2EAFEF5A2EA1CC04
:10B0F0009093A5098093A409BACBB0924909A09274
:10B1000048099FCB709258096092570988CB5FEF2E
:10B11000083315070CF0CECA08E31FEFC7CA48E38F
:10B12000A4164FEFB4060CF0B7CAA8E3AA2EAFEFEF
:10B13000BA2EAECA1E821D829FCA222433247FCA21
:10B14000E092F904F092FA040093FB041093FC04DB
:10B15000C7C8B092CB04A092CA047093C90460938C
:10B16000C8040C94A8508FE390E0A0E0B0E0C80EB3
:10B17000D91EEA1EFB1E15CB215C3F4F4F4F5F4F80
:10B18000F0CA215C3F4F4F4F5F4FBCCA615C7F4F9D
:10B190008F4F9F4FEDCC2F5F3F4FDCCC22273327C3
:10B1A00024193509D5CC039666C8615C7F4F8F4F53
:10B1B0009F4F76CD2F5F3F4F65CD22273327241930
:10B1C00035095ECD61507E4F8F4F9F4F40C822277B
:10B1D00033272A193B092DC88091AD0482608093E2
:10B1E000AD040C94E4461092D6041092D5040C944D
:10B1F0007A454D5F5F4F0C94D6444D5F5F4F0C9482
:10B200008C44019609CC8091F808A82EBB24CC244C
:10B21000DD246D8D7E8D8F8D98A1A60195010E94F4
:10B22000A96C39014A018091930990919409AA2748
:10B2300097FDA095BA2F681A790A8A0A9B0A6A892B
:10B240007B898C899D89A60195010E94A96C590171
:10B250006A018091AF099091B009AA2797FDA09546
:10B26000BA2FA81AB90ACA0ADB0AD401C30197FC8B
:10B270001CC53C014D0154E09594879477946794E4
:10B280005A95D1F7D601C501D7FC07C55C016D0100
:10B2900044E0D594C794B794A7944A95D1F7809188
:10B2A000B2049091B304813491050CF4CAC3C40173
:10B2B000B30123E030E040E050E00E94A96C390186
:10B2C0004A01C601B50123E030E040E050E00E94B1
:10B2D000A96C59016A018091E408E82FFF27EE0F5D
:10B2E000FF1FE155F74F808191810190F081E02DA2
:10B2F000F7FDCFC47A97A4F0C401B30123E030E096
:10B3000040E050E00E94A96C39014A01C601B50134
:10B3100023E030E040E050E00E94A96C59016A014E
:10B3200071E267167104810491042CF030E2632EFF
:10B33000712C812C912C80EE68168FEF78068FEFA0
:10B3400088068FEF980644F420EE622E2FEF722EBF
:10B350002FEF822E2FEF922E91E2A916B104C10495
:10B36000D1042CF090E2A92EB12CC12CD12CA0EE4E
:10B37000AA16AFEFBA06AFEFCA06AFEFDA0614F0BF
:10B380000C94B74E80EEA82E8FEFB82E8FEFC82EFC
:10B390008FEFD82E0C94B74E8091D0049091D104A9
:10B3A000A091D204B091D304F4E0880F991FAA1F92
:10B3B000BB1FFA95D1F78093130490931404A093C4
:10B3C0001504B09316041092110410921004215029
:10B3D000304030934405209343056E8961FF3EC0A1
:10B3E00080919E03823308F056C38091CB03815035
:10B3F00098F41092EA048091D0049091D104A09125
:10B40000D204B091D3048093CC049093CD04A09344
:10B41000CE04B093CF0481E08093CB0341C010925F
:10B420007C05E92DFF27EE0FFF1FE155F74F8081C7
:10B4300091818C3491050CF49CC280917D058F5FC5
:10B44000893C08F424C31092D40488EC80937D05D1
:10B450001092AF041092AE040C94584420919E03B5
:10B4600080918A0390918B03820F911D2091EE08A9
:10B470003327829FD001839FB00D929FB00D11247E
:10B48000CD01AA2797FDA095BA2F8093CC04909365
:10B49000CD04A093CE04B093CF0481E08093EA045E
:10B4A0006090860370908703809088039090890352
:10B4B0006D8D7E8D8F8D98A1A40193010E94A96C42
:10B4C00059016A016A897B898C899D89A40193014C
:10B4D0000E94A96CB901C5010E94246B5C01CD9743
:10B4E0001CF0ECE3AE2EB12CC5010E94CA695C01D0
:10B4F0008091EA04882309F469C18091AD049927F9
:10B500009C012071307084FD61C1C0903909C0FC7C
:10B5100004C08091E90881FD04C50B811C81309332
:10B520009B0520939A056090D0047090D104809080
:10B53000D2049090D3048091CC049091CD04A0913A
:10B54000CE04B091CF0486159705A805B90514F06F
:10B55000C0FC52C1E090D004F090D1048091CC04A2
:10B560009091CD04E81AF90A80919D0399278E9D48
:10B57000D0018F9DB00D9E9DB00D1124CD01B7FD62
:10B58000FEC59595879595958795959587959595FC
:10B590008795081B190B209110043091110437FD79
:10B5A000EBC5359527953595279535952795293000
:10B5B00031050CF4F8C328E030E0229FF001239F0E
:10B5C000F00D329FF00D11249F01F7FDD2C5359586
:10B5D0002795359527958091100490911104280F97
:10B5E000391F80919F039927AA27BB27442737FD3E
:10B5F0004095542FBC01CD010E94356C97FDB4C518
:10B60000B7E09595879577956795BA95D1F79B01A2
:10B61000FFEF61387F070CF0BEC321E83FEF021B4C
:10B62000130B6090F1047090F2048090F3049090FA
:10B63000F40497FCABC5A7E095948794779467943E
:10B64000AA95D1F780919C03282F332744275527AB
:10B65000C401B3010E94356C97FD93C5F5E0959543
:10B66000879577956795FA95D1F79B014FEF6138EC
:10B6700074070CF04BC321E83FEF021B130B65E985
:10B6800070E0E60EF71E7BE2E71671E0F706E8F4DD
:10B6900080919A0590919B05892BB9F480919E0524
:10B6A00090919F051816190684F48091A005909139
:10B6B000A105081719070CF4A6C28091C90390913F
:10B6C000CA03801791070CF49EC2809143059091A4
:10B6D0004405892B21F000919E0510919F058091D2
:10B6E0009A039927AA27BB272091180A332727FDF9
:10B6F0003095432F532FBC01CD010E94356C97FD2F
:10B700004EC5E7E09595879577956795EA95D1F7CA
:10B710009B018FEF213838070CF000C321E83FEF81
:10B72000021B130BC801AA2797FDA095BA2F5DE055
:10B73000880F991FAA1FBB1F5A95D1F7950144275F
:10B7400037FD4095542FBC01CD010E94A96C209378
:10B750006D0530936E0540936F0550937005009111
:10B760006D0510916E0580919C0590919D059C0141
:10B77000220F331F280F391F200F311F37FD14C52B
:10B78000A9015595479555954795BA018091EA08C5
:10B79000282F3327220F331F220F331F421753073F
:10B7A0000CF0E8C2A901B901D090A309C0FE81C282
:10B7B000AB81BC81A417B5070CF07BC2AD01B0937F
:10B7C0009D05A0939C055C834B8318C06091F20893
:10B7D000662309F43FC17727663471050CF020C257
:10B7E00026E430E03093C8032093C703CB80DC808D
:10B7F000D0929D05C0929C05D090A3098091AD0484
:10B8000081FF03C28091AD0484FD33C2E090A205A4
:10B81000F090A3050091A4051091A505E114F10491
:10B8200001051105B1F42B813C8179010027F7FC5A
:10B830000095102FACE0EE0CFF1C001F111FAA9505
:10B84000D1F7E092A205F092A3050093A40510930E
:10B85000A50580911004909111048091100490919D
:10B86000110497FD78C4843691050CF033C26B81C6
:10B870007C819B01442737FD4095542FC501AA27A1
:10B8800097FDA095BA2FBC01CD010E94356C97FDA4
:10B890008EC49B01AC01FDE05595479537952795E2
:10B8A000FA95D1F720936D0530936E0540936F059F
:10B8B000509370058091AE049091AF0477E0803D85
:10B8C000970708F0FCC2D801C701E9E0B695A79533
:10B8D00097958795EA95D1F7E81AF90A0A0B1B0B99
:10B8E000DA01C90173E0880F991FAA1FBB1F7A955F
:10B8F000D1F7E80EF91E0A1F1B1FE092A205F09275
:10B90000A3050093A4051093A505D801C7016CE019
:10B91000B695A795979587956A95D1F790939F05CA
:10B9200080939E054091F008442309F4E5C2552711
:10B930009C01BA010E94746CC901861B970B9093FD
:10B94000A1058093A005260F371F3093CA032093CB
:10B95000C9038090A4099090A509E0915709F0913E
:10B960005809FAAFE9AF00914809109149090C94C0
:10B97000B25410927D050C945844039620CB039644
:10B9800010CB909581959F4F0C94A24503960C94F3
:10B99000A64503960C94A24F909581959F4F0C94C9
:10B9A0009E4F4F960C9463528827992788199909BE
:10B9B0000C941552695F7F4F0C94CA517095619534
:10B9C0007F4F0C94BD5181509E4FAF4FBF4F0C9491
:10B9D0009C5181509E4FAF4FBF4F0C94B1515C01B1
:10B9E000B094A194B108B394BAAEA9AE0C94A95185
:10B9F00084EF91E09093AB038093AA030C94E852F8
:10BA000089AD9AAD909581959F4F6817790714F08D
:10BA10000C94CF52BC010C94CF520894C108D108A9
:10BA2000D092AB03C092AA030C94E852F095E19532
:10BA3000FF4F0C94734E61507E4F8F4F9F4F0C946D
:10BA4000334E8091B0049091B104813491050CF48F
:10BA500042CC2DCC40919E0550919F0557FDBBC116
:10BA600055954795559547958091270390912803C3
:10BA7000209100013327489FF001499FF00D589F06
:10BA8000F00D1124CF01B9010E94746CA5CE8093F2
:10BA90007D050C94584481E08093EA0488EC8093FF
:10BAA000CB03FECC80937C05BCCC80819181855BEF
:10BAB0009F4F0CF01AC180917B058F5F80937B05AF
:10BAC000893C10F40C94DB472C3008F0B6C329985D
:10BAD000A4E0B0E08FEF082E0E94D16C1092D40445
:10BAE00010927B051092AF041092AE040E94083DA4
:10BAF000A4E0B0E0809137059091380597FDB3C47C
:10BB0000892F990F990B082E0E94D16CA5E0B0E007
:10BB10008091370590913805082E0E94D16CA6E0DF
:10BB2000B0E0809135059091360597FD99C4892F35
:10BB3000990F990B082E0E94D16CA7E0B0E080917C
:10BB4000350590913605082E0E94D16C08E010E072
:10BB500080912F0590913005A0913105B09132056B
:10BB6000BC01CD010E949E6BDC01CB019C0197FDC5
:10BB700074C4832F992787FD9A95D801082E0E94B7
:10BB8000D16CB9E0EB2EB0E0FB2E80912F059091A7
:10BB90003005A0913105B0913205BC01CD010E9464
:10BBA0009E6BDC01CB01D701082E0E94D16C0E9454
:10BBB000B20568E770E00E94C1313091E3080C944F
:10BBC000DB47C101AA2797FDA095BA2FBC01CD0183
:10BBD0002F89388D498D5A8D0E94356C2B013C017F
:10BBE0000E94A96C3093EE042093ED0410927F051F
:10BBF0000C94365287B5853F08F07BC080911204C3
:10BC000081500C9499548C0160CD8090A40990903F
:10BC1000A509E0905709F0905809FAAEE9AEA3CE15
:10BC2000673971058CF186E990E09093C8038093A1
:10BC3000C703DCCD0196A11DB11D0C94504E019699
:10BC4000A11DB11D0C945C4E81E080937F05109284
:10BC500065051092660510926705109268051092AE
:10BC6000F9041092FA041092FB041092FC040C9454
:10BC7000E4468090A4099090A5090091570910917D
:10BC800058091AAF09AF6FCE7093C8036093C7030A
:10BC9000ADCDF095E195FF4F2DCB0F96A11DB11DB8
:10BCA000F5CA095F1F4F0C9488520F96A11DB11D54
:10BCB000E0CA70939D0560939C055C834B839ECD89
:10BCC0005B8D5093A6055093A70587CB80937B058A
:10BCD0000C94DB478090A4099090A5092091570906
:10BCE000309158093AAF29AF3ECE40937B050C9472
:10BCF000DB4781E08093A70570CBD0928D05C09281
:10BD00008C054091150A49A30C94544B6F3F710563
:10BD100009F00CF4B2CC2FEF30E0AFCC2F3F31055F
:10BD200009F00CF4FDCC2FEF30E0FACC2093840521
:10BD300030938505409386055093870510929005B2
:10BD40000C941F4D8DA59EA5AFA5B8A98093800525
:10BD500090938105A0938205B093830510928F057F
:10BD60000C942F4C10928E050C94BE4B10929105A2
:10BD70000C948C4DD090A3092D2D3327220F331F07
:10BD8000220F331F20553040241735070CF00ECDFD
:10BD9000A901B9010BCD6F3F710509F00CF43FCC3F
:10BDA0002FEF30E03CCC121613060CF406CC229F89
:10BDB000C001239F900D329F900D112497FD56C313
:10BDC000959587959595879520911004309111044C
:10BDD000281B390B06CC4D5F5F4F42CE0E94B20547
:10BDE00045E661EE78E00E945A058091E90880FFFF
:10BDF00010C080911D0390911E03875B934038F41F
:10BE000080911D0390911E038E5E924010F40E945B
:10BE10005C1C1092F9030E94083D81E08093F903B5
:10BE2000579AC5CE209384053093850540938605A7
:10BE30005093870510928D0510928C05E8EECE2E5A
:10BE4000E3E0DE2ED092AB03C092AA030C948C4D9B
:10BE50007093C9046093C804B092CB04A092CA0442
:10BE6000CB0177FDEAC2BC0175956795C501B7FCAA
:10BE7000E2C25C01B594A7940C947E4A609280055E
:10BE800070928105809282059092830510928D05B3
:10BE900010928C0588EEC82E83E0D82ED092AB038A
:10BEA000C092AA030C942F4C81E08093A60595CAFA
:10BEB0001091E2080C943E47299A0C941247AFE087
:10BEC000803A9A0708F09CC1D801C7016AE0B6958C
:10BED000A795979587956A95D1F7E81AF90A0A0BFD
:10BEE0001B0BDA01C901880F991FAA1FBB1F880FFE
:10BEF000991FAA1FBB1FFDCC1092A1051092A0058F
:10BF00008FEF93E09093CA038093C9038090A409B4
:10BF10009090A509A0905709B0905809BAAEA9AE63
:10BF200022CD8091AD0481FF47C12091C70330919C
:10BF3000C803C9010F964091D5045091D6048417C7
:10BF400095070CF084C18091A605882309F07FC174
:10BF50008091A80581FF9AC28D7F6090D004709077
:10BF6000D1048090D2049090D3046092CC0470925B
:10BF7000CD048092CE049092CF0481608093A80576
:10BF8000421B530B9A012F50304037FD91C28091D4
:10BF90009A0590919B05280F391F30939B0520939C
:10BFA0009A0520919A0530919B05C90137FF04C07D
:10BFB00088279927821B930B815092400CF438C13B
:10BFC0008091EE089927829F7001839FF00C929FC9
:10BFD000F00C1124C70160E075E00E94746CCB0185
:10BFE000AA2797FDA095BA2F2091CC043091CD04BB
:10BFF0004091CE045091CF04820F931FA41FB51F10
:10C000008093CC049093CD04A093CE04B093CF043E
:10C0100010929B0510929A05C1FE06C08BE490E039
:10C020009093FC038093FB038091F208882309F02E
:10C03000FFC000919E0510919F05A80117FD1EC22B
:10C0400055954795559547958091270390912803DD
:10C05000209100013327489FB001499F700D589FE0
:10C06000700D1124CB01B9010E94746C6634710506
:10C070000CF0FEC126E430E03093C8032093C703E0
:10C080008091430590914405892B09F454CAD40149
:10C09000C3016092CC047092CD048092CE04909241
:10C0A000CF0451CA81509F4FAF4FBF4F0C94B94935
:10C0B00088279927DC0182199309A409B5090C94F2
:10C0C000864C2093840530938505409386055093D4
:10C0D000870581E0809390050C941F4DB095A09545
:10C0E000909581959F4FAF4FBF4F0C94224B61505D
:10C0F0007F4F8F4F9F4F0C94FB4981509F4FAF4F05
:10C10000BF4F0C94D34981509F4FAF4FBF4F0C94FA
:10C11000434A61507F4F8F4F9F4F0C94114A81507B
:10C120009F4FAF4FBF4F0C94504A2DA53EA54FA532
:10C1300058A9209380053093810540938205509340
:10C14000830581E080938F050C942F4C81E08093D0
:10C150008E050C94BE4B909581959F4F84CB81E0CA
:10C16000809391050C948C4D61587F4F8F4F9F4F5A
:10C1700047CA2D5F3F4F2BCA295F3F4F12CA0F9608
:10C1800000CA615E7F4F8F4F9F4F68CA2FE730E034
:10C1900040E050E0620E731E841E951E4CCA61582A
:10C1A0007F4F8F4F9F4FADCA2D5F3F4FE9CA615000
:10C1B000704E8F4F9F4F6DCB6090D0047090D10424
:10C1C0008090D2049090D304D401C301805991404F
:10C1D000A040B0408093CC049093CD04A093CE04B3
:10C1E000B093CF042091F208222371F133273093CA
:10C1F000C8032093C70300919E0510919F05A3C912
:10C2000080549F4108F057C0D801C701EBE0B695B4
:10C21000A79597958795EA95D1F7E81AF90A0A0B39
:10C220001B0BDA01C901820F931FA41FB51F61CB3D
:10C2300000919E0510919F0523CF299A49CCF09536
:10C24000E195FF4F0C94BD4728E730E0D0CFC901FE
:10C250000F97481759070CF040C08091A705882315
:10C26000E1F58091A80580FF1AC18E7F6090D0040F
:10C270007090D1048090D2049090D3046092CC044A
:10C280007092CD048092CE049092CF04826080930D
:10C29000A805421B530B9A01215F3F4F37FD0CC18C
:10C2A00080919A0590919B05821B930B90939B051F
:10C2B00080939A0576CED801C7017CE0B695A79504
:10C2C000979587957A95D1F7E81AF90A0A0B1B0B0F
:10C2D000E20EF31E041F151F10CB2091A805822F1C
:10C2E000992783709070892B09F491C02C7F20933B
:10C2F000A80510929B0510929A056090D00470904A
:10C30000D1048090D2049090D3046092CC047092B7
:10C31000CD048092CE049092CF04C1FE42CE84EF31
:10C3200091E09093FC038093FB033BCE2093840524
:10C330003093850540938605509387050C94744D82
:10C340002093840530938505409386055093870597
:10C350000C94074D295F3F4F4F4F5F4F0C94EA4CB1
:10C3600081509E4FAF4FBF4F0C94D74C88279927D1
:10C37000DC0182199309A409B5090C94D34C21500E
:10C380003E4F4F4F5F4F0C94774BB095A0959095D3
:10C3900081959F4FAF4FBF4F0C94714B81509F4F72
:10C3A000AF4FBF4F0C94B64B295F3F4F4F4F5F4F7E
:10C3B0000C94904B81509F4FAF4FBF4F0C94234C28
:10C3C000295F3F4F4F4F5F4F0C94FB4B21503E4F27
:10C3D0004F4F5F4F0C94E24BB095A095909581958F
:10C3E0009F4FAF4FBF4F0C94DC4B295F3F4F4F4FD8
:10C3F0005F4F0C94574D21503E4F4F4F5F4F0C9461
:10C40000404D81509F4FAF4FBF4F0C94804D609077
:10C41000D0047090D1048090D2049090D304C1CD08
:10C4200081509F4FAF4FBF4F0C94134DF095E19546
:10C43000FF4F0C94764A01961CCD019614CDF095D1
:10C44000E195FF4F0C943A4788279927DC01821920
:10C450009309A409B5090C943A4D21503F4F89CB5B
:10C4600081509F4F64CB81509F4F4ACB0396A8CCFD
:10C470006739710534F026E930E0FECD4D5F5F4F3E
:10C48000DFCD7093C8036093C703FACD6090D004EA
:10C490007090D1048090D2049090D3046ECD6090BF
:10C4A000D0047090D1048090D2049090D304EECE4A
:10C4B000309521953F4F6BCD309521953F4FF0CE74
:10C4C000BF81B150BF830894811C911CE4E0F0E06F
:10C4D000AE0EBF1E0894611C711CB7FD02C00C9407
:10C4E0004457EC960FB6F894DEBF0FBECDBFDF9178
:10C4F000CF911F910F91FF90EF90DF90CF90BF9061
:10C50000AF909F908F907F906F905F904F903F90F3
:10C510002F9008958091B5059091B605A091B7052B
:10C52000B091B8058093AD059093AE05A093AF058B
:10C53000B093B0058091B1059091B205A091B3057B
:10C54000B091B4058093A9059093AA05A093AB057B
:10C55000B093AC0508951092C0051092BF051092DB
:10C56000BE051092BD05089584B1806A84B93D9AD4
:10C5700082E58CBD1DBC459A81E08093B5098AEAAD
:10C580008093B90983E88093BA099AE09093BB0934
:10C590001092BD091092BC091092BF091092BE09F9
:10C5A0001092170A1092DB091092DC098CE4809338
:10C5B000DD0986E08093DE099093DF090895EF920C
:10C5C000FF920F931F938091F8089927880F991F66
:10C5D000880F991F7C010027F7FC0095102F809190
:10C5E000290590912A05A0912B05B0912C05BC013D
:10C5F000CD01A80197010E94A96C3093BD09209339
:10C60000BC098091210590912205A0912305B0914C
:10C610002405BC01CD01A80197010E94A96C3093AB
:10C62000BF092093BE092091AB093091AC0940911C
:10C63000AD095091AE09DA01C901E3E0880F991FF5
:10C64000AA1FBB1FEA95D1F7820F931FA41FB51F26
:10C65000820F931FA41FB51F20918603309187037B
:10C660004091880350918903BC01CD010E94A96CBF
:10C670003093C5092093C409E0913305F091340546
:10C6800080916D0990916E09BF010E94746CCB017D
:10C690009B01220F331F220F331F280F391F280F32
:10C6A000391F37FD1CC13595279535952795309352
:10C6B000C1092093C0098091A7099091A809BF01E1
:10C6C0000E94746C9B01220F331F220F331F260F11
:10C6D000371F260F371F37FDFFC035952795359536
:10C6E00027953093C3092093C20910923405109204
:10C6F000330510926E0910926D091092A8091092DC
:10C70000A7098091BB0999278C30910509F4A1C034
:10C710008D3091050CF069C08A30910509F4A4C1EF
:10C720000B9709F410C18091DB09882309F4CBC071
:10C730002091E1093091E209C90181509E4F8F5F3C
:10C740009340C8F44091E3095091E409CA01815033
:10C750009E4F8F5F934078F48091E90885FF0BC06E
:10C760003093C0052093BF055093BE054093BD058F
:10C770008AEF8093C2058091E7099091E80921E052
:10C78000893692070CF056C19C019093F004809377
:10C79000EF048091ED049091EE04281B390BC90140
:10C7A000845E9D4F68E671E00E94746C845B9040EB
:10C7B0009093EC048093EB042091EB093091EC0909
:10C7C0008091FB039091FC038217930740F48091C2
:10C7D0007E07882321F43093FC032093FB03809190
:10C7E000E009873609F0ADC12AC18E30910509F400
:10C7F00076C18E3091050CF475C00F9709F093CF78
:10C80000809110098093CC09809138098093CD09DB
:10C81000809192038093CE09809109098093CF097A
:10C8200080910A098093D00980910B098093D109E6
:10C83000809191038093D20980910D098093D3094F
:10C8400080910E098093D40980910F098093D509B6
:10C850006ACF80917E07863018F010927E0785E0BF
:10C860008093CC09809135098093CD0980912F0860
:10C87000909130089093CF098093CE098091CC0499
:10C880009091CD04A091CE04B091CF04BC01CD0114
:10C8900025E030E040E050E00E94A96C3093D109DF
:10C8A0002093D00980912B098093D20980912C0983
:10C8B0008093D30980912D098093D4098091DB095D
:10C8C000882309F035CF1092C0051092BF05109251
:10C8D000BE051092BD0535C12D5F3F4FFECE2D5FC9
:10C8E0003F4FE1CE809126098093CC0980912709A2
:10C8F0008093CD09809128098093CE0980912909E0
:10C900008093CF0980912A098093D00980912E09C4
:10C910008093D10980912F098093D20980913009A9
:10C920008093D309809133098093D4098091310990
:10C930008093D509809132098093D609809134097A
:10C940008093D709F0CEF8948091E308E82FFF2771
:10C95000EE0FFF1FE155F74F0190F081E02DE03819
:10C96000F1050CF0D1C02FEFE138F20714F4E1E843
:10C97000FFEFE093CC098091E408E82FFF27EE0F4A
:10C98000FF1FE155F74F0190F081E02DE038F105F0
:10C990000CF4CDC0EFE7F0E0E093CD098091E20820
:10C9A000E82FFF27EE0FFF1FE155F74F0190F081B1
:10C9B000E02DE038F1050CF4B2C0EFE7F0E0E093D1
:10C9C000CE098091E108E82FFF27EE0FFF1FE15508
:10C9D000F74F0190F081E02DE038F1050CF497C09D
:10C9E000EFE7F0E07894E093CF098091E50480933D
:10C9F000D0098091E3048093D1098091E104809370
:10CA0000D2098091DF048093D3098091DE04809362
:10CA1000D4098091DD048093D509809133089091E9
:10CA2000340897FD8CC0959587959595879580934B
:10CA3000D60979CE2091EF043091F004AACE8091EE
:10CA4000ED098093140A8091EE098093160A809173
:10CA5000EF098093150A8091F0098093170A80915D
:10CA6000F1098093180A6DC08091C1048093CC09AC
:10CA70008091C0048093CD098091BF048093CE093A
:10CA80008091BE048093CF098091BD048093D0092A
:10CA90008091BC048093D1098091BB048093D2091A
:10CAA0008091BA048093D3098091AD048093D40916
:10CAB0008091AD04837F8093AD0480912703909192
:10CAC00028038093D509809100018093D609A2E0C4
:10CAD000B0E00E94C46C802D8093D70924CE809151
:10CAE000DC098093CC098091DD098093CD09809188
:10CAF000DE098093CE098091DF098093CF09809170
:10CB000002018093D0090FCEEFE7F0E032CF8FEF34
:10CB1000E138F8070CF066CFE1E8FFEF63CF6FEF85
:10CB2000E138F6070CF04BCFE1E8FFEF48CF4FEFCD
:10CB3000E138F4070CF030CFE1E8FFEF2DCF03969A
:10CB400072CF1F910F91FF90EF9008958091B509DA
:10CB5000882309F43BC0459889EB99E09093B70985
:10CB60008093B6098091C105E82FFF27E453FC4F5D
:10CB7000982F9F5F80818093BB09973008F027C072
:10CB80009093C1051092B5090E94DF6281E0809305
:10CB9000B8090000000000000000000000000000D4
:10CBA0000000000000000000000000000000000085
:10CBB0000000000000000000000000000000000075
:10CBC00000008091B9098093D8098EBD0895109214
:10CBD000C105D8CF2091B509222309F045C00DB475
:10CBE00007FE42C084E08093FA03459A3EB58091E7
:10CBF000C30599278130910509F437C0823091052A
:10CC00000CF451C0029709F439C02091B8092032C0
:10CC100008F030C04598000000000000000000004F
:10CC20000000000000000000000000000000000004
:10CC300000000000000000000000000000000000F4
:10CC4000000000000000E091B609F091B709E20F82
:10CC5000F11D80818EBD8091D8099081890F8093CC
:10CC6000D8092F5F2093B8090895353551F12093E5
:10CC7000C305CBCF81E08093B509F3CF8091DA096A
:10CC8000E82FFF27E650F64F30838F5F8093DA0955
:10CC90008A3100F18091C405381711F12093DB0926
:10CCA0001092C305B2CF892B09F0AFCF2093DA09D8
:10CCB0003093C405313809F0A8CF81E08093C305D3
:10CCC000A4CF8091C405830F8093C40582E0809334
:10CCD000C3059BCF8091C405830F8093C40595CF76
:10CCE0008AE1EAEFF9E0A0EEB9E001900D928A95B1
:10CCF000E1F781E08093DB091092C30586CF87B10D
:10CD00008C6087B9429843981092C60580E880935A
:10CD1000D4031092C5058093D30308958091CB0569
:10CD200081508F3F19F08093CB05089584E0809364
:10CD3000CB058091AD0485FF16C040912409409336
:10CD4000CC05609125096093CD0550913709252FB9
:10CD5000332724FF13C08091D404882379F425FF5E
:10CD600017C0429A33C08091DE04882334F7409183
:10CD700020094093CC0560912209E5CF90912109CB
:10CD80009B3FB8F080916F098D3D98F047FDE9CF4A
:10CD90004298252F332724FD1DC0909123099B3FE6
:10CDA00008F18091A209873EE8F067FD19C0439819
:10CDB00008959B3F20F080916F098A3008F180919F
:10CDC000C60581508F3F21F18093C605252F33275B
:10CDD00024FFE3CF8091D4048823F9F626FFE7CF20
:10CDE000439A08959B3F20F08091A2098A3060F019
:10CDF0008091C50581508F3FE1F08093C50508956E
:10CE000047FDC6CF429AE2CF67FDD1CF439A08953E
:10CE100080916F0981508093C6058091D403813041
:10CE2000C9F086958093D403842309F4B1CF429A44
:10CE3000CDCF8091A20981508093C5058091D30305
:10CE4000813051F086958093D303862309F4AFCFC8
:10CE5000439A089580E8E6CF80E8F5CF8091C90035
:10CE60008F778093C9008091C9008F7B8093C90020
:10CE70008091C9008F7D8093C9005A9A5298109270
:10CE8000CD0084E190E08093CC008091C800826066
:10CE90008093C80080E18093C9008091CA008F7799
:10CEA0008093CA008091CA008F7B8093CA008091D2
:10CEB000CA008F7D8093CA008091CA008F7E8093C4
:10CEC000CA008091CA00877F8093CA008091C90000
:10CED0008B7F8093C9008091CA0084608093CA00D0
:10CEE0008091CA0082608093CA008091C80087FF49
:10CEF0000CC08091CE008091C800882334F48091CA
:10CF0000CE008091C8008823A4F38091C900806876
:10CF10008093C90008951F93CF93DF9380E197E238
:10CF20000E94F217EC0110E08091C9008F77809386
:10CF3000C9008091C9008F7E8093C9005A9883E20E
:10CF400098E09F938F931F930E9473140F900F90FC
:10CF50000F90CE010E94FB17882309F066C04A9B00
:10CF6000F8CF8AE590E00E94F217EC0189E598E09D
:10CF70009F938F931F920E947314529A0F900F9059
:10CF80000F90CE010E94FB178823D9F383E690E02F
:10CF90005A9A019797FFFCCF8FE891E05A98019732
:10CFA00097FFFCCF89E090E05A9A019797FFFCCF5A
:10CFB00089E090E05A98019797FFFCCF8FE891E0C5
:10CFC0005A9A019797FFFCCF8FE891E05A98019702
:10CFD00097FFFCCF89E090E05A9A019797FFFCCF2A
:10CFE00089E090E05A98019797FFFCCF8FE891E095
:10CFF0005A9A019797FFFCCF8FE891E05A980197D2
:10D0000097FFFCCF89E090E05A9A019797FFFCCFF9
:10D0100089E090E05A98019797FFFCCF8FE891E064
:10D020005A9A019797FFFCCF0AC08FE598E09F932B
:10D030008F931F930E9473140F900F900F9052982C
:10D040005A980E942E67DF91CF911F9108951F92E9
:10D050000F920FB60F921124EF92FF920F931F932E
:10D060002F933F934F935F936F937F938F939F93F0
:10D07000AF93BF93CF93DF93EF93FF932091CE00B5
:10D080008091D503813009F44BC08091CE0588236F
:10D09000C9F040E050E08091CF058823C9F4452BCA
:10D0A00009F44AC081E08093CF058091D0058F5F5D
:10D0B0008093D00543E08091D0058031E8F440931F
:10D0C000CE0504C141E050E08091CF05882339F3BB
:10D0D000813009F44AC08230B9F1833009F44AC082
:10D0E00081E08093D5031092D0051092D20544E4DC
:10D0F0008091D005803118F38091D205882331F4D6
:10D100008091D503882311F4809384031092D00575
:10D110001092D2051092CF0584E48093CE05D6C03C
:10D120001092D50384E48093CE051092D00510921E
:10D13000CF051092D105CAC044E48093D0058093F6
:10D14000CF058093D105D4CF452B51F643E02093F2
:10D15000D1059091D005923009F492C083E080937C
:10D16000CF059F5F9093D005C3CF452B09F0B8CF73
:10D1700082E099CF452B09F0B3CF482F82E080930E
:10D18000CF058091D0058F5F8093D0059091D10518
:10D19000892F86958695E82FFF27EF70F0703196DE
:10D1A000892F9927982F88273327822B932B9370C9
:10D1B0008050924063E070E00E94746CEB30F105A7
:10D1C00008F057C07F01EE0EFF1EF701E155F74F43
:10D1D000808191819B01281B390BC90137FD6EC0ED
:10D1E000069754F48091DE04883C08F05BC080917F
:10D1F000DE04865F8093DE04F701E155F74F8081FE
:10D2000091819C01220F331F280F391F260F371FD2
:10D2100037FD51C0E901D595C795D595C795CB0187
:10D2200001968C179D07BCF521978091DE04843B05
:10D2300060F187010B53174FF701E155F74F8081DC
:10D240009181FE01E81BF90BCF0163E070E00E94C1
:10D25000746CCB01880F991F860F971FF80191837B
:10D2600080832FEA38E0E20EF31EF701D183C083FA
:10D270003FCF729708F43CCF81E08093D50338CF3D
:10D2800027FD20C01092D20569CFF701EB53F74F6D
:10D2900011821082E6CF61507040C617D7072CF676
:10D2A0002196C3CF88EC8093DE0480916F008F7D40
:10D2B00080936F00A1CF2D5F3F4FACCF90958195AC
:10D2C0009F4F8ECF81E08093D20548CFFF91EF91A1
:10D2D000DF91CF91BF91AF919F918F917F916F918E
:10D2E0005F914F913F912F911F910F91FF90EF9080
:10D2F0000F900FBE0F901F901895CF93FC0197FDD4
:10D3000021C0C1E028E631E0CF01B9010E94746C70
:10D31000FC018B35910554F08B5590408A35910571
:10D3200038F484EB90E08E1B9F0BFC0141E013C0AE
:10D33000CF01855B90408A35910548F4E45BF0406D
:10D340004FEF09C0CFEFF095E195FF4FDBCF2E1BDC
:10D350003F0BF9014FEFEE0FFF1FEC53F64F2591F6
:10D3600034918C2F992787FD9095829FB001839FE0
:10D37000700D929F700D1124842F992787FD909531
:10D38000689FA001699F500D789F500D1124CA011C
:10D39000CF9108952AE530E0281B390BC9010E947E
:10D3A0007D6908951F93CF93DF93EB01611571059C
:10D3B00019F4009709F494C097FD3EC011E020973E
:10D3C00029F48AE51802B00111248AC0AA2797FD22
:10D3D000A095BA2F26E0880F991FAA1FBB1F2A9578
:10D3E000D1F79E01442737FD4095542FBC01CD0154
:10D3F0000E94A96CF90137FD2CC081E0EA35F807DD
:10D40000ACF08CE1E73AF807CCF02AE530E01C16E6
:10D410001D061CF5812F992787FD9095829FB001ED
:10D42000839F700D929F700D11245AC0E659F74FDB
:10D430008491282F3327EBCF1FEFC1CF89E0ED3840
:10D44000F8078CF485E0EA3BF80784F028E530E043
:10D45000DECFF095E195FF4FD0CFD7FD0EC0B901DB
:10D46000645B70403DC029E530E0D1CF84E0E73116
:10D47000F80754F027E530E0CACF111684F764EBC3
:10D4800070E0621B730B2CC083E0EE32F8071CF0D7
:10D4900026E530E0BCCF82E0E939F8071CF025E54D
:10D4A00030E0B5CF82E0E233F8071CF024E530E04D
:10D4B000AECF81E0E73EF8071CF023E530E0A7CFD0
:10D4C00081E0ED3AF8071CF022E530E0A0CFEF57FD
:10D4D000F1401CF021E530E09ACF20E530E097CF15
:10D4E000CB01DF91CF911F910895EF92FF920F939F
:10D4F0001F93CF93DF937B018C0120E030E040E06D
:10D5000050E0FA01E9016FE00BC0C21BD30BE40B42
:10D51000F50B2F5F3F4F4F4F5F4F615067FD31C09D
:10D52000220F331F441F551FCC0FDD1FEE1FFF1F9F
:10D53000CC0FDD1FEE1FFF1FD801C7017EE1B6959E
:10D54000A795979587957A95D1F7C80FD91FEA1FA8
:10D55000FB1FEE0CFF1C001F111FEE0CFF1C001F19
:10D56000111F2F5F3F4F4F4F5F4FC217D307E40785
:10D57000F50758F62150304040405040615067FF59
:10D58000CFCF5695479537952795CA01B901DF91B9
:10D59000CF911F910F91FF90EF90089500242227C3
:10D5A0003327442751E0BB27EE27FF27A0E1660F72
:10D5B000771F881F991F001C221F331F441F660FEF
:10D5C000771F881F991F001C221F331F441F2AF436
:10D5D000050E2B1F3E1F4F1F04C0051A2B0B3E0BC1
:10D5E0004F0B550FBB1FEE1F587F556047FD525024
:10D5F000AA95E9F6E695B7955795E695B7955795A7
:10D60000852F9B2F08952227332741E0552768E077
:10D61000880F991F221F331F880F991F221F331F46
:10D620001AF4240F351F02C0241B350B440F551F5D
:10D63000487F456037FD42506A9551F756954795AA
:10D6400056954795842F0895AA2797FF04C0809583
:10D6500090958A1F9A1F77FF04C0609570956A1F86
:10D660007A1F669F9001779FA001679F300D411D33
:10D670005A1F300D411D5A1F889FF001999F2E0F90
:10D680003F1F401D511D899F300D411D5A1F300DF8
:10D69000411D5A1FCA01B901112480CFFC0141501C
:10D6A000504030F001900616D1F73197CF01089520
:10D6B0008827992708955058192EA6D001D08CC0DC
:10D6C000BA176207730784079507B1F188F40EF45F
:10D6D00010940B2EBA2FA02D062E622F202D072E70
:10D6E000732F302D082E842F402D092E952F502D6D
:10D6F000FF275523B9F0591B49F0573E98F046953E
:10D7000037952795A795F0405395C9F776F0BA0F4E
:10D71000621F731F841F30F4879577956795B795BF
:10D72000F040939517FA0F2E0895BF1BBB27BA0B35
:10D73000620B730B840BF6CFDEF692C097FB70D0B2
:10D740009F3738F0FEE9F91B982F872F762F6B2F24
:10D7500005C083C09695879577956795F150D0F76A
:10D760003EF490958095709561957F4F8F4F9F4FB8
:10D770000895E89403C097FB0EF4F3DFB62F672FEC
:10D78000782F892F9EE9002427C00ED05EF004C0B8
:10D790000BD026F001C008D019F020F48FEF0895C7
:10D7A00080E0089581E0089597FB092E052600F892
:10D7B00068942DD0E89407FC07C0621773078407AC
:10D7C000950721F008F400940794989408959A9589
:10D7D000BB0F661F771F881F11249923A1F0882390
:10D7E000B2F79F3F59F0BB0F48F421F4002011F429
:10D7F00060FF04C06F5F7F4F8F4F9F4F881F9795CB
:10D80000879597F9089529C0052E092607FA440F30
:10D81000551F5F3F79F0AA27A51708F051E04795FB
:10D82000880F991F9F3F31F0BB27B91708F091E08F
:10D83000879508959F919F91112414C097FB880F9D
:10D84000991F9F3F31F0BB27B91708F091E08795EA
:10D8500008959F919F91112405C0662777278827F7
:10D86000992708959FEF80EC0895629FD001739FE0
:10D87000F001829FE00DF11D649FE00DF11D929F6C
:10D88000F00D839FF00D749FF00D659FF00D9927AB
:10D89000729FB00DE11DF91F639FB00DE11DF91FCF
:10D8A000BD01CF0111240895991B79E004C0991F8F
:10D8B000961708F0961B881F7A95C9F780950895EA
:10D8C000AA1BBB1B51E107C0AA1FBB1FA617B707A6
:10D8D00010F0A61BB70B881F991F5A95A9F78095C2
:10D8E0009095BC01CD01089597FB092E07260AD01B
:10D8F00077FD04D0E5DF06D000201AF4709561951D
:10D900007F4F0895F6F7909581959F4F0895A1E276
:10D910001A2EAA1BBB1BFD010DC0AA1FBB1FEE1FA9
:10D92000FF1FA217B307E407F50720F0A21BB30BF4
:10D93000E40BF50B661F771F881F991F1A9469F770
:10D9400060957095809590959B01AC01BD01CF01CC
:10D95000089597FB092E05260ED057FD04D0D7DF7A
:10D960000AD0001C38F450954095309521953F4FD2
:10D970004F4F5F4F0895F6F790958095709561959C
:10D980007F4F8F4F9F4F0895F999FECFB2BDA1BD34
:10D99000F89A119600B40895F7DF01921A94E1F70E
:10D9A0000895F999FECFB2BDA1BD00BC11960FB686
:10D9B000F894FA9AF99A0FBE08950190F2DF1A943A
:04D9C000E1F70895EE
:10D9C4005E010A0151756164726F0000416E676CFB
:10D9D400654E69636B20202020202020416E676CF7
:10D9E40065526F6C6C202020202020204163634E00
:10D9F40069636B2020202020202020204163635273
:10DA04006F6C6C2020202020202020204779726F0A
:10DA140047696572202020202020202048696768FB
:10DA2400742056616C756520202020204163635A60
:10DA34002020202020202020202020204761732027
:10DA4400202020202020202020202020436F6D70C3
:10DA54006173732056616C7565202020566F6C7459
:10DA6400616765202020202020202020456D7066DD
:10DA7400616E672020202020202020204779726FAB
:10DA8400204B6F6D70617373202020204D6F746F75
:10DA9400722046726F6E7420202020204D6F746FA8
:10DAA4007220526561722020202020204D6F746FF7
:10DAB40072204C6566742020202020204D6F746FE6
:10DAC40072205269676874202020202020202020A2
:10DAD4002020202020202020202020202020202042
:10DAE4002020202020202020202020205661726920
:10DAF4006F4D657465722020202020204D4B334DDE
:10DB040061672043616C5374617465205365727658
:10DB14006F2020202020202020202020486F6F7696
:10DB2400657267617320202020202020202020207F
:10DB340020202020202020202020202020202020E1
:10DB440020202020202020202020202020202020D1
:10DB540020202020202020202020202020202020C1
:10DB640020202020202020202020202020202020B1
:10DB740020202020202020202020202020202020A1
:10DB84002020202020202020202020204932432D26
:10DB94004572726F72202020202020202020202017
:10DBA4002020202020202020202020204750535FA8
:10DBB4004E69636B20202020202020204750535F93
:10DBC400526F6C6C2020202020202020C80001648B
:10DBD400FF01FFFF01FC01FC0101737373FF0300EC
:10DBE4007D0000C409C40964000E48616C6C6F2098
:10DBF40057656C7400000000000000000000000085
:10DC04000000000000000000000000000000000010
:10DC14000000000000000000000000000000000000
:10DC240000000000000000000000000000000000F0
:10DC340000000000000000000000010203040506CB
:10DC44000708090A01040B050000ECFF6440415A6F
:10DC54004664640A02969696960840403A10FB3051
:10DC6400380190D0030090D00300F4016400537095
:10DC74006F727400004E6F726D616C0000426567D4
:10DC8400696E6E657200007800FF03640A0B0D0B69
:06DC94000C0E0F0101015E
:00000001FF
